:100000000C94850B0C9422B40C9453B40C9484B4CB
:100010000C94B5B40C94E6B40C9417B50C9448B594
:100020000C9479B50C94B00B0C943BAE0C94B00BC3
:100030000C94B00B0C94B00B0C94B00B0C94B37EDE
:100040000C94B00B0C94B00B0C94B00B0C94B00B44
:100050000C94E17E0C94B00B0C94B00B0C94AAB5EC
:100060000C94B00B0C94E5B70C94DEB90C94B00B67
:100070000C94B00B0C94B00B0C94B00B0C949780B8
:100080000C9404800C944A810C94B00B0C94B00B2B
:100090000C94B00B0C94B00B63557F55A955C55506
:1000A000EB552A56545678569056C156F156175766
:1000B0007357995716583C586258BF58F1581959F8
:1000C0003D5961596C597759775F9E59D759E9590C
:1000D000065A235A3C5A625A775F775F775F775F99
:1000E000775F775F815AAA5ACE5A775F775F775FDB
:1000F000775F775F775F775FF25A0A5B385B775F8E
:10010000775F775F775F775F775F775F775F775F3F
:10011000775F775F775F775F775F775F775F775F2F
:10012000775F775F775F775F775F775F775F775F1F
:10013000775F775F775F775F775F775F775F775F0F
:10014000775F775F775F775F775F775F775F775FFF
:10015000775F775F775F775F775F775FDA5B005C0A
:10016000255C4B5C715C9A5CBA5CFB5C215D405D1C
:10017000635D895DAA5DD05DF15D125E335E545EA4
:100180006F5E865EA75EBA5EE05EF85E235F4765DF
:100190006E2E004D6F742E0043616D2E004B662E47
:1001A0000056656C206F66207265717565737465A5
:1001B00064204B463A2000506F73206F66207265B2
:1001C00071756573746564204B463A200054696DFF
:1001D00065206F6620726571756573746564204B68
:1001E000463A200050726F672E202520636F6D7095
:1001F0006C6574653A20004D61782070726F67728B
:10020000616D2074696D652028696E636C2E2073A2
:10021000746172742064656C6179293A20004B46E0
:100220002043757272656E742072756E2074696DEC
:10023000653A200052756E2073746174653A20002F
:10024000436F6E742E2076696420647572617469E0
:100250006F6E3A2000416363656C2076616C69645F
:100260003A200056656C2076616C69643A20004142
:100270006363656C2061742074696D6520783A2031
:100280000056656C2061742074696D6520783A2091
:1002900000506F736974696F6E2061742074696DAA
:1002A0006520783A20004D6F746F722076656C205F
:1002B000757064617465207261746520286D73299E
:1002C0003A20004B6579206672616D6520636F7519
:1002D0006E743A200054616B696E672075702062FD
:1002E00061636B6C6173680053746F7070696E67E3
:1002F000206B662070726F6772616D00506175735C
:10030000696E67206B662070726F6772616D005254
:10031000756E6E696E672F726573756D696E672095
:100320006B662070726F6772616D005365747469DB
:100330006E6720636F6E742E207669642E206D6F59
:1003400076652074696D653A2000456E64696E6754
:10035000204B46207472616E736D697373696F6EA2
:100360000053657474696E672075647061746520EC
:10037000726174653A200053657474696E67207603
:10038000656C6F636974793A200053657474696EA3
:100390006720706F736974696F6E3A2000536574DB
:1003A00074696E672061627363697373613A2000D8
:1003B00053657474696E67206B6579206672616D30
:1003C0006520636F756E743A200053656C656374C5
:1003D000696E6720617869733A200041766F6964BD
:1003E000206F66667365743A2000496E7465727694
:1003F000616C6F6D65746572206D6F64653F203A46
:1004000020004B6565702D616C6976653F203A2050
:100410000054657374206D6F64653F203A2000536B
:10042000686F74732066697265643A2000496E745F
:10043000657276616C2074696D653A20004D697251
:10044000726F722075703F203A2000466F6375739B
:1004500020772F20736875747465723F203A2000EE
:1004600044656C61792074696D653A20004D61784E
:100470002073686F74733A2000466F63757320743D
:10048000696D653A20005472696767657220746906
:100490006D653A200042757379206578706F7369D5
:1004A0006E673F203A2000456E61626C65643F20B4
:1004B0003A200053657474696E6720696E746572C2
:1004C00076616C6F6D65746572206D6F64653A203E
:1004D0000053657474696E67206B6565702D616C7F
:1004E0006976653A200053657474696E6720746597
:1004F0007374206D6F64653A200053657474696E7F
:100500006720696E74657276616C2074696D653AF6
:10051000200053657474696E67207265706561743C
:10052000206379636C65733A200053657474696E57
:100530006720666F63757320772F206578706F73FF
:100540007572653A200053657474696E672064653E
:100550006C61792074696D653A2000536574746923
:100560006E67206D61782073686F74733A20005352
:10057000657474696E6720666F6375732074696D46
:10058000653A200053657474696E672074726967F8
:100590006765722074696D653A20004578706F73E5
:1005A000696E67206E6F77210053657420656E61F8
:1005B000626C65643A200049732073656E64696EED
:1005C000673F3A2000506C6174666F726D207261F3
:1005D00074696F3A200047656172626F78207261BA
:1005E00074696F3A2000556E697420636F64653AD0
:1005F0002000436865636B696E6720322D7074203C
:1006000076656C2076616C69646974793A20004C77
:100610006561642D6F75743A200049732070726FA4
:100620006772616D2076616C69643F203A200053E7
:100630006C6565703A200050726F6772616D20645E
:100640006563656C206C656E6774683A2000507253
:100650006F6772616D20616363656C206C656E67A6
:1006600074683A20004C6561642D696E3A2000542C
:10067000726176656C206C656E6774683A20005311
:10068000746F7020706F733A20005374617274201D
:10069000706F733A2000456173696E673A200041BC
:1006A0006363656C3A200053706565643A200052BC
:1006B000756E6E696E673F203A20004375727265F1
:1006C0006E7420706F733A2000456E6420706F73F3
:1006D0003A20004D61782073706565643A200044CB
:1006E0006972656374696F6E3A20004D6963726F59
:1006F00073746570733A20004261636B6C61736858
:100700003A2000456E61626C65643A20005365745E
:1007100074696E672073746F702D6D6F74696F6E7E
:10072000206D6F64653A200053657474696E6720AC
:10073000706C6174666F726D20726174696F3A20BB
:100740000053657474696E672067656172626F78C3
:1007500020726174696F3A200053657474696E6722
:1007600020756E6974733A200053657474696E67FE
:1007700020656E6420706F736974696F6E20746F8A
:100780003A200053657474696E67206375727265F0
:100790006E7420706F736974696F6E20746F3A2085
:1007A0000053656E64696E6720746F3A200053656C
:1007B0007474696E672073746F7020686572650069
:1007C00053657474696E6720737461727420686510
:1007D0007265004175746F2D73657474696E67205E
:1007E0006D6963726F737465707320005265736511
:1007F00074696E67206C696D69747320616E642022
:1008000073746172742F73746F7020706F696E747B
:10081000730053657474696E67206C656164206F42
:1008200075743A200053656E64696E6720746F209A
:1008300073746F70200053656E64696E6720746F07
:100840002073746172740053657474696E672064F8
:100850006563656C206C656E6774683A200053654B
:100860007474696E6720616363656C206C656E6784
:1008700074683A200053657474696E6720747261FD
:1008800076656C206C656E6774683A2000536574F9
:1008900074696E67206C6561642D696E3A2000533F
:1008A000657474696E6720656173696E67206D6F2A
:1008B00064653A200053657474696E672073746FC1
:1008C000703A200053657474696E672073746172A6
:1008D000743A2000436F6D6D616E646564207374BB
:1008E0006570733A200053657474696E67206163A4
:1008F00063656C65726174696F6E3A20005365744C
:1009000074696E6720636F6E742E20737065656402
:100910003A200053657474696E67206A6F79737446
:1009200069636B2073706565643A200053656E647B
:10093000696E6720746F20656E640053656E64692C
:100940006E6720746F20686F6D65005365747469FD
:100950006E6720656E6420686572653A2000536595
:100960007474696E6720686F6D65206865726500D4
:1009700053657474696E6720646972656374696F26
:100980006E3A200053657474696E67206D6178203B
:1009900073706565643A200053657474696E6720EE
:1009A0006D6963726F73746570733A200053657478
:1009B00074696E67206261636B6C6173683A2000D2
:1009C00053746F7070696E67206D6F746F7200532F
:1009D000657474696E6720656E61626C653A2000AB
:1009E00053657474696E6720736C6565703A200096
:1009F00052756E696E672073656C66206469616705
:100A00006E6F737469630046726565206D656D6F06
:100A100072793A20004772616666696B206D6F6477
:100A2000653A200050726F6772616D2072756E209A
:100A30007374617475733A2000436F6E74726F6CD7
:100A40006C657220636F756E743A2000456E642089
:100A5000706F7320726573746F72653A20005374FF
:100A60006172742F73746F7020706F73207265736E
:100A7000746F72653A200043757220706F73207234
:100A80006573746F72653A2000416C6C206D6F74F1
:100A90006F7220736C656570207374617465733A4E
:100AA000200050726F6772616D2076616C69643FDF
:100AB0003A2000416E79206D6F746F7273207275E9
:100AC0006E6E696E673F3A200046505320666C6137
:100AD000673A200049732070726F6772616D2063FE
:100AE0006F6D706C6574653F3A2000546F74616C73
:100AF0002070726F6772616D2074696D653A2000B5
:100B0000546F74616C2070726F6772616D207469CC
:100B10006D653A20002520436F6D706C6574653AF1
:100B200020005761746368646F67206D6F64653F70
:100B3000203A200050696E67706F6E67206D6F6499
:100B4000653A20004A6F79737469636B206D6F6436
:100B5000653A2000506C616E20747970653A20000F
:100B600053746172742064656C61793A2000416C41
:100B70007420696E7075742065646765206465749F
:100B8000656374696F6E3A2000537570706C7920DC
:100B900063757272656E743A2000537570706C796B
:100BA00020766F6C746167653A20004375727265D8
:100BB0006E742072756E2074696D653A20005275EE
:100BC0006E207374617475733A2000536574746990
:100BD0006E6720617070206D6F64653A2000536508
:100BE0007474696E67204772616666696B206D6F09
:100BF00064653A200053657474696E6720636F6E94
:100C000074726F6C6C657220636F756E743A20003D
:100C100053657474696E6720656E6420706F73200D
:100C2000726573746F72653A200053657474696EEF
:100C3000672073746172742F73746F7020706F7398
:100C400020726573746F72653A200053657474691D
:100C50006E672063757220706F7320726573746F96
:100C600072653A2000526576657273696E6720730B
:100C7000746172742F73746F7020706F696E747307
:100C80000053657474696E672046505320666C612A
:100C9000673A200053657474696E672073746F70CF
:100CA00020706F73206865726520666F7220616CBA
:100CB0006C206D6F746F72732E2E2E0053656E64F0
:100CC000696E67206D6F746F727320746F20737418
:100CD00061727420706F736974696F6E005365740C
:100CE00074696E672070696E672D706F6E67206D16
:100CF0006F6465200053657474696E67206A6F794C
:100D0000737469636B206D6F646520005365747440
:100D1000696E672070726F6772616D206D6F6465B8
:100D20003A200053657474696E672073746172743D
:100D30002064656C61793A200053657474696E674C
:100D4000207761746368646F67206D6F64653A2013
:100D50000053657474696E67206C696D69742073E3
:100D600077697463682065646765206D6F64653AB0
:100D7000200053656E64696E6720616C6C206D6F36
:100D8000746F727320686F6D650053657474696E5B
:100D90006720616464726573733A2000546F6767FB
:100DA0006C696E67206465627567204C454400532A
:100DB000746F7070696E672070726F6772616D001A
:100DC00050617573696E672070726F6772616D0034
:100DD0005374617274696E67202F20726573756D2C
:100DE000696E672070726F6772616D00536574740D
:100DF000696E67206E657720616464726573732124
:100E000000426C7565746F6F746820004D6F636F7E
:100E10004275732000537562616464723A00206306
:100E20006F6D6D616E643A00206275665B305D3A8D
:100E30002000206275665B315D3A20002062756695
:100E40005B325D3A2000206275665B335D3A2000BC
:100E5000206275665B345D3A200074696D65200020
:100E600053656E64696E67206D6F746F72200072D7
:100E7000657665727365537461727453746F70280C
:100E800029004D6F742E3133202D204175746F2D44
:100E90007374617274696E6720636F6E74696E75C6
:100EA0006F7573206D6F7665004A6F79737469632F
:100EB0006B3A20004D6F746F7273206172652072FF
:100EC000756E6E696E672C2063616E277420617584
:100ED000746F2D736574206D6963726F73746570C0
:100EE0007300526571756573746564204D69637232
:100EF0006F73746570733A2000547279696E67205D
:100F0000746F206175746F2D736574206D696372E1
:100F10006F73746570730045786365737369766584
:100F2000207370656564207265717565737465649E
:100F300000546F702073706565642072657175650B
:100F4000737465643A20004D6963726F73746570E1
:100F5000733A20004F7574206F66206C6F6F70209D
:100F6000616E64206D6F76696E67206F6E21004D33
:100F70006963726F73746570733A200047657474A7
:100F8000696E6720766964206D6F76652074696D7F
:100F9000653A200047657474696E6720544C206D73
:100FA0006F76652074696D653A20005368757474B6
:100FB000657220646F6E652C2072656164792066AD
:100FC0006F72206D6F76650054696D6520617420C5
:100FD0006578706F737572653A200054696D65208D
:100FE000617420666F6375733A20006B665F4361BE
:100FF0006D657261436865636B2829202D2042610D
:10100000696C696E672066726F6D2063616D6572D1
:1010100061206379636C6520617420706F696E7400
:101020002032006B665F43616D6572614368656382
:101030006B2829202D20536B697070696E672073AF
:10104000686F742C2077616974696E6720666F72AF
:101050002065787465726E616C207472696767656B
:10106000720053656E64696E6720746F2000416280
:101070006F757420746F2073656E6420746F206CBC
:101080006F636174696F6E20233A200053656E644C
:10109000696E67206D6F746F727320746F206E6558
:1010A00077206C6F636174696F6E73005374617243
:1010B00074696E67206E6577206B6620626F756E4F
:1010C00063652070726F6772616D0053746F70702A
:1010D000696E67206B662070726F6772616D005376
:1010E00074617274696E67206B65657020616C69EC
:1010F0007665207068617365005061757365206C5A
:10110000656E6774683A200053544F5050494E47FB
:10111000204B462050524F4752414D0053746F7040
:1011200070696E67206D6F746F7220005041555367
:10113000494E47204B462050524F4752414D0020C8
:101140004B462070726F6772616D005374617274E8
:10115000696E67206E6577207479706520002A2A91
:101160002A2056656C6F636974696573202A2A2A80
:10117000002A2A2A20506F736974696F6E73202ABF
:101180002A2A002A2A2A20416273636973736173D1
:10119000202A2A2A00207E7E7E7E7E7E007E7E7E23
:1011A0007E7E7E20415849532000436F6E742E206E
:1011B000766964656F2074696D653A200050726FBE
:1011C0006772616D206D6F64653A200050657263CF
:1011D000656E7420636F6D706C6574653A200043B2
:1011E000757272656E742072756E2074696D653AE1
:1011F000200052756E207374617475733A20004D2F
:101200006178206D6F76652074696D653A20004DB8
:1012100061782063616D6572612074696D653A2043
:10122000007E7E7E7E7E7E2047656E6572616C20CC
:1012300050726F6772616D20506172616D73207EB4
:101240007E7E7E7E7E004175746F2070617573694D
:101250006E67212121006379636C6553686F744F59
:101260004B2829202D20616C74466F72636553688A
:101270006F74206E6F7420646574656374656400B8
:101280006379636C6553686F744F4B2829202D2058
:10129000616C74466F72636553686F742064657423
:1012A0006563746564202A2A2A2A2A2A2A2A2A2A75
:1012B0002A2A006379636C6553686F744F4B282941
:1012C000202D204578742E20696E74657276616CCD
:1012D000206D6F646520616374697665006379636E
:1012E0006C6553686F744F4B2829202D20456E7410
:1012F00065722066756E6374696F6E006379636CE6
:101300006543616D6572612829202D2053746172D7
:1013100074696E67206578706F7375726520637984
:10132000636C65006379636C6543616D6572612808
:1013300029202D2043616D65726120627573793AB1
:1013400020006379636C6543616D657261282920B3
:101350002D204261696C696E672066726F6D206333
:10136000616D657261206379636C652061742070C2
:101370006F696E742033004D6F746F722000637953
:10138000636C6543616D6572612829202D20536867
:101390006F74733A20006379636C6543616D6572A5
:1013A000612829202D204261696C696E6720667270
:1013B0006F6D2063616D657261206379636C652078
:1013C000617420706F696E742032006379636C659C
:1013D00043616D6572612829202D20536B697070FF
:1013E000696E672073686F742C2077616974696E09
:1013F0006720666F722065787465726E616C207408
:10140000726967676572006379636C6543616D65D6
:1014100072612829202D204261696C696E672066FF
:10142000726F6D2063616D657261206379636C65B5
:1014300020617420706F696E742031006D73206FAD
:1014400066206C6561642D6F75742072656D6169CD
:101450006E696E67006379636C6543616D65726187
:101460002829202D2054686572652061726520004E
:101470006379636C6543616D6572612829202D2055
:10148000416C6C206D6F7420646F6E65206D6F769B
:10149000696E67006379636C6543616D657261288D
:1014A00029202D2050617573696E67006379636C24
:1014B0006543616D6572612829202D205374617226
:1014C000740063616D43616C6C4261636B28292019
:1014D0002D2053746F700063616D43616C6C4261C9
:1014E000636B2829202D20537461727400206C6571
:1014F0006164496E3A20002073686F74733A20006B
:1015000020547970653A200020656E61626C653AFE
:1015100020002072756E6E696E673A200020656E3D
:1015200064506F733A20002073746F70506F733A79
:101530002000207374617274506F733A200020622F
:1015400061636B6C6173683A200020636F6E74692D
:101550006E696F75732053706565643A200043753A
:101560007272656E742053746570732000120110DE
:101570000102000008EB03442001000102030109FD
:10158000023E00020100C032090400000102020113
:1015900000052400100104240206052406000107AA
:1015A0000582030800FF09040100020A0000000789
:1015B0000504021000050705830210000504030955
:1015C000042E03440079006E0061006D0069006321
:1015D0000020005000650072006300650070007418
:1015E0000069006F006E0020004C004C00430000BA
:1015F000003C03440079006E0061006D00690063E7
:1016000000200050006500720063006500700074E7
:101610000069006F006E002000430044004300207A
:1016200000530065007200690061006C0000000E4C
:101630000330003000340035003700330000000074
:10164000002100240027002A002D00300000002285
:1016500000250028002B002E003100000020002370
:1016600000260029002C002F0001010101010101C9
:101670000102020202020202020303030303030344
:101680000304040404040404040505050505050514
:101690000506060606060606060102040810204096
:1016A000800102040810204080010204081020403C
:1016B000800102040810204080010204081020402C
:1016C000800102040810204080000000000000009B
:1016D000000000000007030401000000000B0A09DD
:1016E00000020800000000000000000000000000F0
:1016F00000000000000000000000010203040506D5
:101700000700B01899B9C1BDA91811241FBECFEFA9
:10171000D0E2DEBFCDBF14E0A0E0B1E0E8E2F1E945
:1017200001E00BBF02C007900D92A839B107D9F7AD
:101730001BBE13E1A8E9B4E001C01D92A236B107B7
:10174000E1F717E1C8E0D7E104C02297FE010E944B
:101750004CC8C230D107C9F70E94B4BA0C9487C8EC
:101760000C940000CF93DF93BC018230910510F4FC
:1017700062E070E0A0915A13B0915B13ED01E0E0DC
:10178000F0E040E050E021C08881998186179707FA
:1017900069F48A819B81309719F09383828304C016
:1017A00090935B1380935A13FE0134C06817790736
:1017B00038F44115510519F08417950708F4AC0168
:1017C000FE018A819B819C01E9012097E9F6411580
:1017D0005105A9F1CA01861B970B049708F4BA01B9
:1017E000E0E0F0E02AC08D919C9111978417950755
:1017F000F9F46417750781F412968D919C911397F3
:10180000309719F09383828304C090935B13809385
:101810005A13FD0132964CC0CA01861B970BFD017D
:10182000E80FF91F6193719302978D939C9340C0C9
:10183000FD01828193819C01D9011097A1F68091CD
:10184000581390915913892B41F48091A4039091DE
:10185000A50390935913809358134091A603509178
:10186000A7034115510541F44DB75EB78091A2031E
:101870009091A303481B590B209158133091591391
:10188000CA01821B930B8617970780F0AB014E5F4E
:101890005F4F8417950750F0420F531F5093591311
:1018A00040935813F9016193719302C0E0E0F0E0B6
:1018B000CF01DF91CF910895CF93DF93009709F483
:1018C00050C0EC0122971B821A82A0915A13B0914A
:1018D0005B13109709F140E050E0AC17BD0708F129
:1018E000BB83AA83FE0121913191E20FF31FAE1752
:1018F000BF0779F48D919C911197280F391F2E5FA6
:101900003F4F3983288312968D919C9113979B8327
:101910008A834115510571F4D0935B13C0935A1318
:1019200020C012968D919C911397AD01009711F0F4
:10193000DC01D3CFFA01D383C28321913191E20F2D
:10194000F31FCE17DF0769F488819981280F391FAB
:101950002E5F3F4FFA01318320838A819B819383DD
:101960008283DF91CF910895A0E0B0E0EAEBFCE044
:101970000C9452C86C01009729F4CB010E94B20B61
:101980006C01C1C08EEF882E8FEF982E8C0C9D1CA1
:101990008601060F171F0815190508F4B2C0F401D7
:1019A000A081B181A617B707B8F0A530B10508F43A
:1019B000AAC0CD0104978617970708F4A4C0129710
:1019C000A61BB70BF801A193B193D4016D937C933F
:1019D000CF010E945C0C97C07B01EA1AFB0AEEEF74
:1019E000FFEFEE0EFF1E36016A0E7B1EC0915A13EA
:1019F000D0915B1344245524AA24BB244AC0C615A5
:101A0000D705E1F5488159814E155F05B8F1CA0146
:101A100004978E159F05B0F41296A40FB51FF4011C
:101A2000B183A0832A813B814114510431F0D2015A
:101A300013963C932E93129766C030935B132093BA
:101A40005A1361C08A819B81F8019383828342503B
:101A500050404E195F09518340834114510431F0C5
:101A6000D20113961C930E93129704C010935B132C
:101A700000935A13F4017183608345C08881998172
:101A8000A816B90608F45C012E018A819B819C018D
:101A9000E901209709F0B3CF809158139091591321
:101AA00086159705E9F4A616B706D0F42091A6038B
:101AB0003091A7032115310541F42DB73EB7809130
:101AC000A2039091A303281B390B02171307C8F434
:101AD0001093591300935813D4016D937C9313C042
:101AE000CB010E94B20BEC01009759F0F401408148
:101AF0005181B6010E94900DC6010E945C0C6E01DE
:101B000002C0CC24DD24C601CDB7DEB7E0E10C94E1
:101B10006EC8FB01DC0105900D920020E1F70895ED
:101B2000FB01DC0102C001900D9241505040D8F7FA
:101B30000895FB01DC0101900D920020E1F708956A
:101B4000FB019F01E8944230C4F04532B4F44A30BE
:101B500029F497FB1EF4909581959F4F642F77276A
:101B60000E94E6C7805D8A330CF0895D8193CB01CA
:101B70000097A1F716F45DE251931082C9010C940D
:101B80000310FA01CF93FF93EF932230CCF025326C
:101B9000BCF4C22F2C2F332744275527FF93EF93F4
:101BA0000E940DC8EF91FF91605D6A330CF0695D92
:101BB0006193B901CA01605070408040904051F774
:101BC00010828F919F91CF910C940310FB019F0184
:101BD000423074F0453264F4642F77270E94E6C7E0
:101BE000805D8A330CF0895D8193CB010097A1F76A
:101BF0001082C9010C940310A0E0B0E0E2E0FEE026
:101C00000C9460C89E01275F3F4F8D819E816F813C
:101C10007885A9010E94100E2096E2E00C947CC801
:101C2000ABE0B0E0E6E1FEE00C9450C83C012B01D3
:101C30005A01FC0117821682838181FD03C06FEF78
:101C40007FEFC6C19AE0892E1E010894211C311C29
:101C5000F3012381F20123FD859123FF81912F015F
:101C6000882309F4B2C1853239F423FD859123FF1D
:101C700081912F01853229F490E0B3010E94131065
:101C8000E7CF982FFF24EE249924FFE1FF15D0F031
:101C90009B3269F09C3228F4903259F0933291F4DF
:101CA0000EC09D3249F0903369F441E024C052E007
:101CB000F52A84E0F82A28C098E0F92A25C0E0E156
:101CC000FE2A22C0F7FC29C0892F80538A3070F485
:101CD000F6FE05C0989C902C1124980E15C0E89C27
:101CE000E02C1124E80EF0E2FF2A0EC09E3229F407
:101CF000F6FC6BC140E4F42A07C09C3619F450E8A6
:101D0000F52A02C0983649F4F20123FD959123FF8C
:101D100091912F01992309F0B8CF892F85548330F1
:101D200018F08052833038F444E050E0A40EB51E21
:101D30005FE359830FC0933631F0933779F09335D1
:101D400009F056C020C0F5018081898342E050E04F
:101D5000A40EB51E610101E010E012C0F501C080C3
:101D6000D180F6FC03C06FEF7FEF02C0692D70E0F9
:101D700042E050E0A40EB51EC6010E94F80F8C018F
:101D80005FE7F52214C0F501C080D180F6FC03C0E6
:101D90006FEF7FEF02C0692D70E042E050E0A40ECB
:101DA000B51EC6010E94ED0F8C0150E8F52AF3FE26
:101DB00007C01AC080E290E0B3010E941310EA94B9
:101DC0008E2D90E008171907A8F30EC0F601F7FC56
:101DD0008591F7FE81916F0190E0B3010E9413108D
:101DE000E110EA94015010400115110579F7EAC09D
:101DF000943611F0993669F5F7FE08C0F501208197
:101E000031814281538184E090E00AC0F5018081F4
:101E100091819C01442737FD4095542F82E090E04A
:101E2000A80EB91E9FE6F92257FF09C050954095AC
:101E3000309521953F4F4F4F5F4FE0E8FE2ACA0192
:101E4000B901A1012AE030E00E943F10D82ED2183B
:101E500040C0953729F41F2D1F7E2AE030E01DC0B9
:101E60001F2D197F9F3661F0903720F4983509F0C7
:101E7000ACC00FC0903739F0983709F0A6C004C045
:101E800028E030E00AC0106114FD146020E130E069
:101E900004C014FD166020E132E017FF08C0F50110
:101EA000608171818281938144E050E008C0F50136
:101EB00080819181BC0180E090E042E050E0A40E7E
:101EC000B51EA1010E943F10D82ED2188FE7F82E20
:101ED000F122F6FE0BC05EEFF522D91438F4F4FEC1
:101EE00007C0F2FC05C08FEEF82202C01D2D01C014
:101EF000192DF4FE0DC0FE01ED0DF11D8081803322
:101F000019F499EEF92208C01F5FF2FE05C003C064
:101F10008F2D867809F01F5F0F2DF3FC14C0F0FEA3
:101F20000FC01E1510F09D2C0BC09D2C9E0C911AFD
:101F30001E2D06C080E290E0B3010E9413101F5FC7
:101F40001E15C0F304C01E1510F4E11A01C0EE24E2
:101F500004FF0FC080E390E0B3010E94131002FF62
:101F60001DC001FD03C088E790E00EC088E590E049
:101F70000BC0802F867891F001FF02C08BE201C078
:101F800080E2F7FC8DE290E0B3010E94131006C0DE
:101F900080E390E0B3010E9413109A94D914C0F327
:101FA000DA94F101ED0DF11D808190E0B3010E9402
:101FB0001310DD20A9F706C080E290E0B3010E9473
:101FC0001310EA94EE20C1F743CEF30166817781C6
:101FD000CB012B96E2E10C946CC8FC01059061509A
:101FE00070400110D8F7809590958E0F9F1F08952F
:101FF000FC016150704001900110D8F780959095D8
:102000008E0F9F1F0895DC01FC01672F71917723CC
:10201000E1F7329704C07C916D9370836291AE17A3
:10202000BF07C8F308950F931F93CF93DF938C01DD
:10203000EB018B8181FF1BC082FF0DC02E813F8190
:102040008C819D812817390764F4E881F981019317
:10205000F983E88306C0E885F985802F0995892BE7
:1020600031F48E819F8101969F838E8302C00FEF92
:102070001FEFC801DF91CF911F910F910895FA01D1
:10208000AA27283051F1203181F1E8946F936E7FB7
:102090006E5F7F4F8F4F9F4FAF4FB1E03ED0B4E0A8
:1020A0003CD0670F781F891F9A1FA11D680F791FE9
:1020B0008A1F911DA11D6A0F711D811D911DA11DFA
:1020C00020D009F468943F912AE0269F112430190A
:1020D000305D3193DEF6CF010895462F4770405DA5
:1020E0004193B3E00FD0C9F7F6CF462F4F70405D54
:1020F0004A3318F0495D31FD4052419302D0A9F7AF
:10210000EACFB4E0A6959795879577956795BA95A8
:10211000C9F700976105710508959B01AC010A2E6E
:1021200006945795479537952795BA95C9F7620F45
:10213000731F841F951FA01D0895FC01108281E06C
:10214000818312820895FC01748363830E949D1031
:102150000895FC0180810895FC016183862F089514
:10216000FC016283862F08951F93CF93DF93EC01C8
:10217000162F68838981882399F085E393E160E0D5
:1021800071E00E9499BC85E393E1612F42E050E049
:102190000E940EBC85E393E167E171E00E9449BDB6
:1021A0008A81882399F08B819C8160E071E00E9494
:1021B00099BC8B819C81612F42E050E00E940EBC53
:1021C0008B819C8167E171E00E9449BDDF91CF91D5
:1021D0001F9108958091A20408958091DA041092CD
:1021E000DA040895809106041092060408958093FD
:1021F0009B04882311F010929C04089580919B0405
:10220000089580939C04882311F010929B040895F4
:1022100080919C0408958093DB048093DC040895EE
:102220008091DB04811181E0089581E08093880D25
:1022300008950F931F93CF93DF93EC018EE46132E7
:10224000780718F060E27EE405C06436710510F48A
:1022500064E670E080E090E00E9449C62FEF30E035
:10226000C29F8001C39F100DD29F100D11240157F2
:10227000124F0F501F4FF801619371938193919307
:102280008F0120E030E040E05FE30E94FFC6F801EC
:102290006083718382839383DF91CF911F910F912C
:1022A00008952F923F924F925F926F927F928F92FA
:1022B0009F92AF92BF92CF92DF92EF92FF920F93D5
:1022C0001F93DF93CF9300D000D0CDB7DEB73C0192
:1022D0008FEF90E0689EB001699E700D789E700D42
:1022E0001124FB01E157F24FDF01A751BF4FE3512A
:1022F000FF4F20813181428153818D919D910D90BD
:10230000BC91A02D281739074A075B0709F43FC184
:10231000FB01EF56F24F80E090E020E030E040E03B
:1023200050E0208331834283538320AF31AF42AFEB
:1023300053AF148E158E168E178E019634968730F5
:10234000910579F78FEF90E0689E8001699E100DEE
:10235000789E100D11240157124F05501F4FD801C0
:102360006D917D918D919C9120E030E040EA51E4A7
:102370000E94FFC62FE632E143E852E40E94B0C556
:102380006B017C0106501040D8018D919D910D90FC
:10239000BC91A02D89839A83AB83BC83F801B29052
:1023A000A29092908290C701B601A50194010E946B
:1023B000FBC6181614F4750164018FEF90E0689E57
:1023C000F001699EF00D789EF00D1124E958F14F4F
:1023D0008081882321F4F7FAF094F7F8F094C7018C
:1023E000B60129813A814B815C810E94B0C51B01F5
:1023F0002C01E89457F88FEF90E0689EF001699EF9
:10240000F00D789EF00D1124E157F24F22823382B5
:1024100044825582E751FF4F80819181A281B3812F
:10242000E95EF040868F978FA0A3B1A3C2AED3AE72
:10243000E4AEF5AEC701B60120E030E040E050E088
:102440000E94FBC618164CF489819A81AB81BC812D
:10245000B05889839A83AB83BC838FEF90E0689EEA
:102460008001699E100D789E100D11240157124FA6
:1024700086E5682E712C600E711E89819A81AB8170
:10248000BC81F30180839183A283B3830F2EF0E09C
:102490008F2EF0E09F2EF0E0AF2EF0E0BF2EF02D5B
:1024A000D80116968D929D92AD92BC9219975E9628
:1024B0006D917D918D919C9191970E944BC66B017E
:1024C0007C01C201B101F80122AD33AD44AD55AD7F
:1024D0000E94FFC69B01AC01C701B6010E9448C51E
:1024E0006B017C0169817A818B819C8120E030E0E5
:1024F00040E05FE30E94FFC6A20191010E94FFC677
:10250000A20191010E94FFC69B01AC01C701B60167
:102510000E9448C50E9418C66B017C01D8019296A2
:102520006D937D938D939C939597025C1F4FF8015B
:1025300080829182A282B382045E1F4FD8018D9265
:102540009D92AD92BC921397F3016081718182815B
:10255000938120E030E040E05FE30E94FFC6D301BA
:102560006D937D938D939C9313970D561F4FF80198
:10257000C082D182E282F38209501040D8018D924C
:102580009D92AD92BC921397F801129212920F9005
:102590000F900F900F90CF91DF911F910F91FF90AF
:1025A000EF90DF90CF90BF90AF909F908F907F90F3
:1025B0006F905F904F903F902F90089580E090E053
:1025C0000E94511181E090E00E94511182E090E060
:1025D0000E945111089520E0039708F421E0822F12
:1025E00008952F923F924F925F926F927F928F92B7
:1025F0009F92AF92BF92CF92DF92EF92FF920F9392
:102600001F93DF93CF93CDB7DEB760970FB6F894E3
:10261000DEBF0FBECDBF8C0149875A876B877C8791
:102620003E872D878FEF90E0089FF001099FF00D06
:10263000189FF00D1124E958F14F8081882359F437
:102640000F2EF0E0CF2EF0E0DF2EF0EAEF2EF1ECCF
:10265000FF2EF02D0AC00F2EF0E0CF2EF0E0DF2E7F
:10266000F0EAEF2EF1E4FF2EF02D8FEF90E0089FBF
:102670009001099F300D189F300D11242157324FC2
:1026800025503F4FD9012D903D904D905C902251A7
:102690003040D9018D919D910D90BC91A02D8D83DD
:1026A0009E83AF83B88729853A854B855C858217E1
:1026B0009307A407B5072CF04FEF5FEF588B4F87B8
:1026C00004C081E090E0988B8F87C201B10120E0C7
:1026D00030E040E050E00E94ACC5882309F44BC1D3
:1026E0008FEF90E0089FF001099FF00D189FF00D0B
:1026F0001124E958F14F808190E0AF85B889FC0141
:10270000AE9FC001AF9F900DBE9F900D112497FF0B
:1027100032C1C8010E9451113CC18FEF90E0089F67
:10272000F001099FF00D189FF00D1124E157F24FB1
:10273000EF50FF4F619071908190919080819181D5
:10274000A281B38189839A83AB83BC83C701B6011D
:10275000A20191010E94FFC62FE632E143E852E454
:102760000E94B0C57B018C01E89417F9C801B7013C
:10277000A40193010E94ACC587FD15C00F2EF0E0A7
:102780006F2EF0E07F2EF0E08F2EF0E09F2EF02DE8
:102790000F2EF0E02F2EF0E03F2EF0E04F2EFFE363
:1027A0005F2EF02D35C0C401B301A80197010E942E
:1027B00047C529813A814B815C810E94B0C53B01AC
:1027C0004C0120E030E040E05FE30E94ACC587FDB3
:1027D00015C00F2EF0E06F2EF0E07F2EF0E08F2E70
:1027E000FFE39F2EF02D0F2EF0E02F2EF0E03F2E76
:1027F000F0E04F2EF0E05F2EF02D0AC060E070E0B8
:1028000080E09FE3A40193010E9447C51B012C01B6
:1028100069817A818B819C81A40193010E94FFC60A
:102820009B01AC01C801B7010E9448C55B016C0166
:10283000C801B701A40193010E94FFC67B018C016E
:1028400069817A818B819C8120E030E040E05FE308
:102850000E94FFC6A40193010E94FFC6A401930138
:102860000E94FFC69B01AC01C801B7010E9448C588
:102870000E9418C60E944BC67B018C01C201B101A7
:10288000A60195010E94FFC69B01AC01C801B701DA
:102890000E9448C50E9418C60E944BC67B018C014D
:1028A000C601B501A60195010E94FFC620E030E0F7
:1028B00040E05FE30E94FFC629813A814B815C8141
:1028C0000E94B0C59B01AC01C801B7010E9448C578
:1028D0000E9418C6EF85F8899F01442737FD40956F
:1028E000542F0E94C7C72D813E814F815885620FAA
:1028F000731F841F951F4F8558894130510551F42E
:1029000029853A854B855C8526173707480759077F
:102910008CF40EC04F8558894F5F5F4F59F429855D
:102920003A854B855C85621773078407950714F415
:10293000CA01B901AD85BE856D937D938D939C933E
:10294000139781E060960FB6F894DEBF0FBECDBF3F
:10295000CF91DF911F910F91FF90EF90DF90CF907B
:10296000BF90AF909F908F907F906F905F904F90AF
:102970003F902F90089529853A854B855C858D8100
:102980009E81AF81B885281739074A075B0709F090
:10299000C4CE80E0D7CF8091A50408958091C10472
:1029A000882339F480914C05882319F420E030E025
:1029B0000AC02091CC043091CD048091A304909161
:1029C000A404280F391FC90108951092A40410927D
:1029D000A3041092CD041092CC040895809192101B
:1029E00091E0892780939210089510929210089593
:1029F0008091921008952091C4043091C5044091B3
:102A0000C6045091C7048091B9049091BA04A09172
:102A1000BB04B091BC04280F391F4A1F5B1FB901CA
:102A2000CA01089580914C05882319F420E030E014
:102A30000BC080914D05882319F421E030E004C0DB
:102A4000813011F422E030E0C90108952091C804DA
:102A50003091C9044091CA045091CB04809138054B
:102A600090913905A0913A05B0913B05280F391F87
:102A70004A1F5B1FB901CA010895813039F08130C6
:102A800018F0823051F406C083E001C082E08093E8
:102A9000C003089581E08093C0030895E091A110E0
:102AA000F091A210309709F0099508958091E10402
:102AB0000895823010F48093C30408958091C30474
:102AC00008958091A60408951F938091C1048823DE
:102AD00011F011E007C080914C05882311F015E03A
:102AE00001C010E08091D704882311F0136004C066
:102AF00080914D05811116608091D6048111186076
:102B00000E946115811110610E945E158111106291
:102B1000812F1F910895FC0110820895FC0180818E
:102B20000895FC0180E880930D1180930E1180932D
:102B30000F11809310111286138608951F93FC01C4
:102B40008081882309F455C070E061507040258170
:102B5000368147815085DA01C901062E04C0B69539
:102B6000A795979587950A94D2F7182F11708181B0
:102B70009281A381B481062E04C0B695A79597953E
:102B800087950A94D2F780FF17C081E090E0A0E01B
:102B9000B0E004C0880F991FAA1FBB1F6A95D2F727
:102BA000822B932BA42BB52B85839683A783B08789
:102BB0001130E9F481E01EC081E090E0A0E0B0E0D7
:102BC00004C0880F991FAA1FBB1F6A95D2F7809572
:102BD0009095A095B09582239323A423B523858354
:102BE0009683A783B087113021F482E003C083E08D
:102BF00001C080E01F910895FC018081882341F18C
:102C0000862F90E001972581368147815085082ED7
:102C100004C056954795379527950A94D2F7922F79
:102C20009170218132814381548104C0569547952A
:102C3000379527958A95D2F720FF06C0913011F479
:102C400081E0089583E00895913011F482E00895C1
:102C500080E00895FC01E45BFF4F80810895FC0152
:102C6000E25BFF4F80810895FC01E15BFF4F8081B3
:102C7000089508951092C11008950895AF92BF92DB
:102C8000CF92DF92EF92FF920F931F935A016B0145
:102C9000CB01BA0120E030E040E053E40E9447C598
:102CA0007B018C0120E030E040E050E00E94FBC658
:102CB00018165CF4C801B70120E030E040E251E4AE
:102CC0000E94ACC51816ACF00AC0C801B70120E0DC
:102CD00030E040E251EC0E94FBC6882354F00F2EF6
:102CE000F0E0AF2EF0E0BF2EF0E0CF2EF3E4DF2EC9
:102CF000F02DB501C6011F910F91FF90EF90DF906D
:102D0000CF90BF90AF900895FC0113A20895FC01ED
:102D1000E60FF11D43870895CF93DF93EC01222343
:102D200019F40E94841612C081E08BA32EA31FA267
:102D30005FA74EA75BA74AA779A768A71DA61CA6F1
:102D40000E94F2B568AB79AB8AAB9BABDF91CF91B8
:102D5000089566E970E044E650E021E00E948C1698
:102D600008957F928F929F92AF92BF92CF92DF92FF
:102D7000EF92FF920F931F93CF93DF934C01742E2A
:102D8000E90181EC90E10E949E15833019F5BE01A6
:102D900080E090E00E9449C67B018C012AE939E974
:102DA00049E15EE30E94FFC60E941DC65B016C0103
:102DB000C801B7012AE939E949E55FE30E94FFC686
:102DC0000E941DC69B01AC01C401B501A901272DBC
:102DD0000E948C16DF91CF911F910F91FF90EF9081
:102DE000DF90CF90BF90AF909F908F907F9008958D
:102DF0006F927F928F929F92AF92BF92CF92DF920B
:102E0000EF92FF920F931F93CF93DF93EC01162F56
:102E1000A42E4901702E6C2C81EC90E1642F0E944D
:102E20009E15982F80915B11882329F080915A116B
:102E3000A81609F08DC0933009F063C01123A9F5DD
:102E4000A0925A1181E080935B110E94F2B56093C9
:102E500056117093571180935811909359111092F5
:102E60005511B70180E090E00E9449C67B018C01BA
:102E70002AE939E949E15EE30E94FFC60E941DC6C6
:102E80005B016C01C801B7012AE939E949E55FE353
:102E90000E94FFC60E941DC69B01AC01CE01B50178
:102EA000A9012FEF0E948C1645C0133019F0113084
:102EB00009F040C0B70180E090E00E9449C67B0164
:102EC0008C012AE939E949E15EE30E94FFC60E94CC
:102ED0001DC65B016C01C801B7012AE939E949E562
:102EE0005FE30E94FFC60E941DC69B01AC01CE019C
:102EF000B501A901272D0E948C1681E080935C11F9
:102F000027C09230B9F480915C11813019F410928D
:102F10005C111EC0882371F480915511882319F427
:102F2000CE010E94841610925B118FA1F401808360
:102F300081E00FC08FA1861558F08091551188232C
:102F400039F4CE010E94841681E0809355116FA25E
:102F500080E0DF91CF911F910F91FF90EF90DF9074
:102F6000CF90BF90AF909F908F907F906F9008957B
:102F70008F929F92AF92BF92CF92DF92EF92FF9289
:102F80000F931F938130910509F0B3C06F5F7F4F9E
:102F900009F0D4C082EE94E00E941F868CEF94E08A
:102FA0000E941F8686E195E00E941F8610925105BF
:102FB0001092500588EE93E0A0E0B0E080935205B7
:102FC00090935305A0935405B09355058AE594E07A
:102FD00090934F0580934E054091B4035091B503F3
:102FE0008AE595E06EE475E02DE430E00CE314E052
:102FF0000E9435AB4091B4035091B5038CEB95E042
:1030000065E373E12DE430E00E9435AB4091B403F9
:103010005091B5038EE196E063E173E12DE430E079
:103020000E9435AB80E896E00E94678981E896E0CF
:103030000E944CA6A1B286E996E06DE270E040E104
:1030400050E020E230E001E110E0E2E1EE2EF12C70
:10305000B3E1CB2ED12CBB24A5E08A2E912C0E946B
:1030600077A2A1B28DE898E06EE270E045E150E011
:1030700024E130E00DE110E0FEE1EF2EF12CEFE174
:10308000CE2ED12CB6E08B2E912C0E9477A2A1B22D
:1030900084E89AE06FE270E042E250E021E230E042
:1030A0000FE010E0ABE2EA2EF12CFCE2CF2ED12CA7
:1030B000E7E08E2E912C0E9477A28BE79CE067E0E0
:1030C0000E94AEA48EE99CE06EE176E00E94F47D61
:1030D00084EA9CE06EE97CE00E94A3100E94F2B5B5
:1030E00060939D1070939E1080939F109093A010FA
:1030F00025C0892B19F56F5F7F4F01F584E89AE0B1
:103100000E94C4898DE898E00E94C48986E996E00F
:103110000E94C4898AE594E090934F0580934E0500
:103120000E94D48186E195E00E94CA888CEF94E0E9
:103130000E94CA8882EE94E00E94CA881F910F9173
:10314000FF90EF90DF90CF90BF90AF909F908F90C7
:10315000089580E090E06FEF7FEF0E94B817089528
:1031600081E090E06FEF7FEF0E94B817089586E945
:1031700096E00E947A8C882389F08DE898E00E947E
:103180007A8C882359F084E89AE00E947A8C90E047
:10319000882309F491E081E0982701C090E0892F0D
:1031A000089541E00E9462AB089542E00E9462AB44
:1031B000089541E00E9462AB089541E00E9462AB35
:1031C000089544E00E9462AB089544E00E9462AB1F
:1031D000089542E00E9462AB089541E00E94B9ABBD
:1031E00008950F931F93CF93DF938FE0689F800123
:1031F0001124065A1F4FC5E4D1E107C0C801BE0122
:103200000E94ED180F5F1F4F219681E1C435D8074A
:10321000A9F7DF91CF911F910F91089541E00E948E
:10322000B9AB089542E00E94B9AB08958093B4030E
:103230001092B50380E090E064EB73E00E941219F5
:10324000089541E00E94B9AB089544E00E94B9ABF3
:10325000089542E00E94B9AB089544E00E94B9ABE2
:103260000895CF93DF93EC0186E996E00E944F8AA0
:10327000882369F48DE898E00E944F8A882339F406
:1032800084E89AE00E944F8A882309F41882DF912B
:10329000CF91089586E996E00E944F8A882371F4C1
:1032A0008DE898E00E944F8A882341F484E89AE0F0
:1032B0000E944F8A882319F081E0089581E00895E3
:1032C000AF92BF92CF92DF92EF92FF920F931F9334
:1032D000DF93CF9300D0CDB7DEB700E010E0A4E2DB
:1032E000EA2EF12CF7EFAF2EF1E0BF2E6E0108941D
:1032F000C11CD11C0A9DC0010B9D900D1A9D900D03
:1033000011248A56994F0E94648A9A838983C7013F
:10331000B6010E9429190F5F1F4F88E190E0E80E67
:10332000F91E0330110531F70F900F90CF91DF9107
:103330001F910F91FF90EF90DF90CF90BF90AF90D3
:1033400008950E9401AD089521E220934F1329E0D2
:103350002093501321E032E0309352132093511305
:10336000109254131092531320E330E0309356130D
:10337000209355131092A7000E94C9B190E08823B2
:1033800009F491E0892F0895FC0180818823C9F018
:10339000628743874093D7038285813021F48FEF82
:1033A0008093D80302C01092D8031092D9031092D0
:1033B000DA0381858093DF0386ED93E060E30E946A
:1033C000A4190895CF93DF93EC018BA1882329F4EE
:1033D00080915411813009F05CC00E94F2B59B01CC
:1033E000AC0188A999A9AAA9BBA9281B390B4A0B2A
:1033F0005B0B6EA57FA56115710501F1CB01A0E006
:10340000B0E0281739074A075B0798F01FA61EA6E9
:1034100088A599A59DA78CA78FA18F5F8FA381E019
:103420008093541181EC90E161E04EEF0E94C41949
:103430002AC0621B730B7FA76EA725C06CA57DA554
:103440006115710501F1CB01A0E0B0E02817390743
:103450004A075B07A0F08EA181508EA3882311F448
:103460001BA204C08AA59BA59FA78EA781EC90E113
:1034700060E04EEF0E94C4191092541104C0621B08
:10348000730B7DA76CA70E94F2B568AB79AB8AABD2
:103490009BABDF91CF910895FC0180818823F1F0EF
:1034A0002185413049F481E090E002C0880F991FE6
:1034B0006A95E2F7282B09C081E090E002C0880FEE
:1034C000991F6A95E2F7809528232187818580934B
:1034D000DF0386ED93E060E30E94A4190895EF9264
:1034E000FF920F931F93CF93DF937C018FE0689F30
:1034F00080011124065A1F4FC5E4D1E107C0C8015D
:10350000BE010E94D1180F5F1F4F219681E1C43583
:10351000D807A9F740E0F70184A9882309F441E01E
:1035200081EC90E162E00E944C1ADF91CF911F91F3
:103530000F91FF90EF900895FC018AE085AB16AAE9
:1035400017AA10AE14AA81E083AF15AE82E081AF56
:1035500012AE16AE17AE14AEEE5BFF4F8083129222
:103560001292E054F04080E883838483858381EC69
:1035700090E162E041E00E944C1A08950F931F937E
:103580008C0181EC90E10E948B15F801118280E89A
:1035900083838483858312A21186128613A2C801B5
:1035A0000E949C1AF801128281E896E061E00E9474
:1035B000F1A481E080939506F80110821F910F918C
:1035C00008950F931F93CF93DF93EC018B018881B4
:1035D00084FF0FC08981882321F085E393E10E9455
:1035E00049BD8A81882329F08B819C81B8010E9482
:1035F00049BDDF91CF911F910F9108950F931F93B4
:10360000CF93DF93EC018B01888183FF0FC0898109
:10361000882321F085E393E10E9449BD8A818823B4
:1036200029F08B819C81B8010E9449BDDF91CF9127
:103630001F910F9108959C0181E08093A7008091D4
:10364000A9008F7B8093A9008091A60080FD06C011
:103650008091A90080648093A9000BC06091F6005E
:103660007091F700C90140E050E00E94FCAB882354
:1036700011F080E008958091A6008E778093A600D7
:103680008091A90080648093A90081E00895CF9380
:10369000DF93EC01809157138B3051F5888188239B
:1036A00039F11FC08E859F85A889B98989839A833E
:1036B000AB83BC838A89C45BDF4F8883CC54D04002
:1036C0008B89C35BDF4F8883CD54D0408C89C25B2C
:1036D000DF4F8883CE54D0408D89C15BDF4F888314
:1036E00007C0CE010C9660E30E941B1B8823D1F615
:1036F000DF91CF9108950F9381E863E041E020E4EA
:1037000030E000E00E9455AC82E063E042E020E45B
:1037100030E00E9455AC0F910895DF93CF93CDB761
:10372000DEB7C851D2400FB6F894DEBF0FBECDBF92
:1037300081E060E0AE01495F5F4F22E10E94D9B2B3
:10374000882309F050C081E0BE016F5F7F4FAE015A
:10375000475E5F4F20E032E00E94C3AF882309F04C
:1037600042C08F8598898C549540E9F589899A895A
:1037700088569240C1F581E00E94F6B2882399F5FF
:103780000E947B1B82E48B838CE08C831D821E82D3
:1037900081E280934F1389E08093501384EF93E08C
:1037A0009093521380935113109254131092531309
:1037B00084E090E090935613809355131092A700E5
:1037C000CE0103960E94C9B1882369F481EC90E18F
:1037D0000E94911581E08093C11084EA9CE068E129
:1037E00071E00E94E11AC85EDD4F0FB6F894DEBFAB
:1037F0000FBECDBFCF91DF910895A82FFB019A0195
:103800008091A803823041F0833019F0813089F42F
:103810000AC08CEB95E002C08AE595E06A2FAF0103
:103820000E94A2A908958EE196E06A2FAF010E943E
:10383000A2A90895E82F9A01AB018091A8038230D4
:1038400041F0833019F0813079F409C08CEB95E0B8
:1038500002C08AE595E06E2F0E941AAA08958EE1B3
:1038600096E06E2F0E941AAA0895E82F9A01AB01E4
:103870008091A803823041F0833019F0813079F4CF
:1038800009C08CEB95E002C08AE595E06E2F0E949E
:10389000F3A908958EE196E06E2F0E94F3A9089592
:1038A000282FAB018091A803823041F0833019F0BA
:1038B000813079F409C08CEB95E002C08AE595E08F
:1038C000622F0E9441AA08958EE196E0622F0E9425
:1038D00041AA0895282FAB018091A803823041F0BE
:1038E000833019F0813079F409C08CEB95E002C087
:1038F0008AE595E0622F0E9462AA08958EE196E023
:10390000622F0E9462AA0895282F462F8091A80353
:10391000823041F0833019F0813079F409C08CEBAA
:1039200095E002C08AE595E0622F0E94CEA9089535
:103930008EE196E0622F0E94CEA90895682F8091B3
:10394000A803823041F0833019F0813069F408C057
:103950008CEB95E002C08AE595E00E94EDA9089500
:103960008EE196E00E94EDA908950F931F93CF93E7
:10397000DF93EC018B01888183FF0FC0898188234D
:1039800021F085E393E10E945DBD8A81882329F0BF
:103990008B819C81B8010E945DBDDF91CF911F9109
:1039A0000F910895EF92FF920F931F93CF93DF93A0
:1039B000EC017A018B01888184FF14C089818823FE
:1039C00031F085E393E122E030E00E9435BD8A8149
:1039D000882341F08B819C81B801A70122E030E06F
:1039E0000E9435BDDF91CF911F910F91FF90EF9015
:1039F00008959C01C397C197E0F486E996E060E0E2
:103A000021E030E040E050E00E947D9F8DE898E0AA
:103A100060E021E030E040E050E00E947D9F84E8DB
:103A20009AE060E021E030E040E050E00E947D9FBD
:103A3000089525363105D8F086E996E061E021E069
:103A400030E040E050E00E947D9F8DE898E061E02A
:103A500021E030E040E050E00E947D9F84E89AE061
:103A600061E021E030E040E050E00E947D9F089559
:103A70004F925F926F927F928F929F92AF92BF927E
:103A8000CF92DF92EF92FF920F931F93CF93DF932A
:103A90000E942A8C882381F566247724C0E0D0E038
:103AA00047EF442E41E0542EC49D8001C59D100D6A
:103AB000D49D100D11240A56194FC8010E945C8C28
:103AC0004B015C01C8010E94338C6B017C01C80171
:103AD0000E946F8CC601880D991D860F971F68166E
:103AE000790608F43C012196C330D105E9F681E856
:103AF00096E0B3010E94FAA4DF91CF911F910F913C
:103B0000FF90EF90DF90CF90BF90AF909F908F90FD
:103B10007F906F905F904F9008952F923F924F92B9
:103B20005F926F927F928F929F92AF92BF92CF924D
:103B3000DF92EF92FF920F931F93DF93CF9300D00A
:103B400000D0CDB7DEB72224332421011A82198296
:103B500049815A8187EF91E0489F9001499F300D3C
:103B6000589F300D11242A56394F3C832B83C901AD
:103B70000E94F189882309F44CC00E942A8C882372
:103B800039F581E896E00E94CFA43B014C018B817E
:103B90009C810E945C8C5B016C018B819C810E94EA
:103BA000338C7B018C018B819C810E946F8CEA0C91
:103BB000FB1C0C1D1D1DE60EF71E081F191FC8015A
:103BC000B701A40193010E94C7C79B01AC011AC0B1
:103BD0008B819C810E945C8C5B016C018B819C8140
:103BE0000E94338C7B018C018B819C810E946F8CA5
:103BF000A80197012A0D3B1D4C1D5D1D260F371F87
:103C0000481F591F221633064406550610F41901A1
:103C10002A01E981FA813196FA83E983339709F021
:103C200097CF2091D2043091D3044091D404509185
:103C3000D504220D331D441D551DB901CA010F9035
:103C40000F900F900F90CF91DF911F910F91FF90E8
:103C5000EF90DF90CF90BF90AF909F908F907F902C
:103C60006F905F904F903F902F9008952F923F92CA
:103C70004F925F926F927F928F929F92AF92BF927C
:103C8000CF92DF92EF92FF920F931F93CF93DF9328
:103C90000E94F2B56624772443014424552457EF4B
:103CA000252E51E0352E429CE001439CD00D529CC4
:103CB000D00D1124CA56D94FCE010E94F189882314
:103CC000F1F0CE010E945C8C5B016C01CE010E9480
:103CD000338C7B018C01CE010E946F8CA80197016F
:103CE0002A0D3B1D4C1D5D1D260F371F481F591FF8
:103CF000621673068406950610F439014A01089489
:103D0000411C511C83E04816510469F60E942A8C1C
:103D1000882391F481E896E00E94FEA4A0E0B0E040
:103D200086159705A805B90538F481E896E00E9444
:103D3000FEA43C01882499240E942A8C882339F40B
:103D40006091A3047091A40480E090E014C060919D
:103D5000B5047091B6048091B7049091B804209195
:103D6000D2043091D3044091D4045091D504621B05
:103D7000730B840B950B0E9449C67B018C01C40117
:103D8000B3010E9449C69B01AC01C801B7010E9462
:103D9000B0C520E030E048EC52E40E94FFC67B0151
:103DA0008C0120E030E040E050E00E94FBC6882318
:103DB0004CF0C801B70120E030E040E05FE30E9432
:103DC00048C508C0C801B70120E030E040E05FE32B
:103DD0000E9447C50E9418C6162F662301F58091E0
:103DE00088118823E1F00E94FE108823C1F484E644
:103DF0008093881180918811DF91CF911F910F914D
:103E0000FF90EF90DF90CF90BF90AF909F908F90FA
:103E10007F906F905F904F903F902F9008951093F8
:103E20008811E8CFAF92BF92CF92DF92EF92FF92CC
:103E30000F931F93DF93CF9300D000D0CDB7DEB7A1
:103E400000E010E076E2E72EF12C67EFA62E61E0AD
:103E5000B62E6E010894C11CD11C0A9DC0010B9D99
:103E6000900D1A9D900D11248A56994F0E94418AF7
:103E700069837A838B839C83C701B6010E942D19C5
:103E80000F5F1F4F88E190E0E80EF91E0330110527
:103E900021F70F900F900F900F90CF91DF911F910E
:103EA0000F91FF90EF90DF90CF90BF90AF9008956B
:103EB0008AE20E94CFB6AA2797FDA095BA2FBC012F
:103EC000CD010E944BC620E030EC4FE754E40E9445
:103ED000B0C520E030E048EC51E40E94FFC60895F0
:103EE0001F93CF93DF93EC01162F888184FF13C0BB
:103EF0008981882331F085E393E14AE050E00E9414
:103F00000EBC8A81882339F08B819C81612F4AE025
:103F100050E00E940EBCDF91CF911F9108951F9336
:103F2000CF93DF93EC01162F888183FF13C0898123
:103F3000882331F085E393E14AE050E00E94FCBB26
:103F40008A81882339F08B819C81612F4AE050E07F
:103F50000E94FCBBDF91CF911F9108951F93CF93D7
:103F6000DF93EC01162F888180FF13C0898188239D
:103F700031F085E393E14AE050E00E94FCBB8A8186
:103F8000882339F08B819C81612F4AE050E00E94A8
:103F9000FCBBDF91CF911F910895FF920F931F9368
:103FA000CF93DF93EC01F62E8A01888180FF10C049
:103FB0008981882321F085E393E10E94FCBB8A81FB
:103FC000882331F08B819C816F2DA8010E94FCBB5E
:103FD000DF91CF911F910F91FF9008951F93CF9381
:103FE000DF93EC01162F888184FF13C08981882319
:103FF00031F085E393E14AE050E00E94FCBB8A8106
:10400000882339F08B819C81612F4AE050E00E9427
:10401000FCBBDF91CF911F9108950F931F93CF9316
:10402000DF93EC018B01888183FF0FC08981882396
:1040300021F085E393E10E9499BC8A81882329F0CD
:104040008B819C81B8010E9499BCDF91CF911F9117
:104050000F9108950F931F93CF93DF93EC018B0182
:10406000888180FF0FC08981882321F085E393E157
:104070000E9499BC8A81882329F08B819C81B80198
:104080000E9499BCDF91CF911F910F9108950F93DA
:104090001F93CF93DF93EC018B01888180FF0FC0CA
:1040A0008981882321F085E393E10E9499BC8A816C
:1040B000882329F08B819C81B8010E9499BCDF91F3
:1040C000CF911F910F9108950F931F93CF93DF937B
:1040D000EC018B01888184FF0FC08981882321F046
:1040E00085E393E10E9499BC8A81882329F08B8122
:1040F0009C81B8010E9499BCDF91CF911F910F91D3
:104100000895DF92EF92FF920F931F93CF93DF9367
:10411000D82E8091CC0C9091CD0C8230910509F471
:104120009FC08330910534F4009769F0019709F03E
:1041300046C128C08330910509F42EC1843691050B
:1041400009F03DC12EC18DE0D81609F43CC19AE0BA
:10415000D91609F438C181E090E09093CD0C80939A
:10416000CC0C9093CF0C8093CE0C1092D00C10926C
:10417000D10C1092D20C1092D30C1092D40C10923D
:10418000D50C21C18091CB0C883631F4E9E6DE16DE
:1041900009F015C18AE00DC08D3629F4F3E7DF166A
:1041A00059F48EE106C0833761F481E6D81609F52B
:1041B00082E38093D00CF2C09DE6D91651F488E2D8
:1041C00046C08E3661F4E0E7DE1609F0F8C08FE1F4
:1041D0003EC0F0E7DF1609F0F2C08BE238C08A3744
:1041E00031F48DE6D81609F0EAC08CE230C083378E
:1041F00031F49DE6D91609F0E2C08AE228C0803782
:1042000031F4E2E7DE1609F0DAC089E220C0823636
:1042100031F4F6E6DF1609F0D2C08CE318C0873619
:1042200031F48FE6D81609F0CAC08DE3C2CF8A36C2
:1042300031F49DE6D91609F0C2C086E408C089367B
:1042400009F0BDC0EDE6DE1609F0B9C087E4809341
:10425000D00C82E090E09093CD0C8093CC0CB3C056
:104260009D2D90539A3020F0FDE2DF1609F065C0D5
:104270008091CB0C8032C1F58091D10C8F5F8093FF
:10428000D10C883248F085E393E168E271E00E9446
:1042900099BC83E090E0DFCFE82FF0E0EE0FFF1F46
:1042A000EE0FFF1FE253F34F10821182128213822E
:1042B0008DE2D81639F48FEF9FEF9093CF0C809357
:1042C000CE0C81C081E090E09093CF0C8093CE0C17
:1042D0008D2D90E0C097AA2797FDA095BA2F8083D7
:1042E0009183A283B3836FC09A3038F56091D10C6B
:1042F000C62FD0E0CC0FDD1FCC0FDD1FC253D34F34
:10430000ED2CFF24E0EDFFEFEE0EFF1E0027F7FC83
:104310000095102F688179818A819B812AE030E0A5
:1043200040E050E00E94C7C7E60EF71E081F191FA5
:10433000E882F9820A831B8346C0F0E2DF1621F08F
:104340008DE0D81609F03FC08091CB0C80538A30A5
:10435000F8F40091D10C0023D9F010E0000F111FE8
:10436000000F111F0253134F2091CE0C3091CF0C30
:10437000442737FD4095542FF80160817181828177
:1043800093810E94C7C7F8016083718382839383FE
:10439000FDE0DF16C1F402C01092D00C84E690E07C
:1043A0005ACF8AE0D81679F48091CB0C8D3059F42D
:1043B0008091D00C1092CD0C1092CC0C05C01092B4
:1043C000CD0C1092CC0C80E0D092CB0CDF91CF9131
:1043D0001F910F91FF90EF90DF900895EF92FF9261
:1043E0000F931F93CF93DF93EC017A018B018881A8
:1043F00083FF14C08981882331F085E393E12AE0AB
:1044000030E00E945EBC8A81882341F08B819C81D0
:10441000B801A7012AE030E00E945EBCDF91CF9195
:104420001F910F91FF90EF900895EF92FF920F93DD
:104430001F93CF93DF93EC017A018B01888184FF76
:1044400014C08981882331F085E393E12AE030E0CC
:104450000E945EBC8A81882341F08B819C81B801D7
:10446000A7012AE030E00E945EBCDF91CF911F914E
:104470000F91FF90EF900895EF92FF920F931F938B
:10448000CF93DF93EC017A018B01888184FF14C004
:104490008981882331F085E393E12AE030E00E94AE
:1044A000D7BB8A81882341F08B819C81B801A70109
:1044B0002AE030E00E94D7BBDF91CF911F910F918E
:1044C000FF90EF900895EF92FF920F931F93382F74
:1044D000562F742FE22F78018EE196E0632F452F3F
:1044E000272F0E2F0E947DA91F910F91FF90EF9013
:1044F0000895EF92FF920F931F93382F562F742F2A
:10450000E22F78018EE196E0632F452F272F0E2FA3
:104510000E947DA91F910F91FF90EF9008958F92B7
:104520009F92AF92BF92CF92DF92EF92FF920F9342
:104530001F93B82EA62E942E822E68018AE595E050
:104540006B2D4A2D292D082D76010E947DA98CEB1B
:1045500095E06B2D4A2D292D0E947DA91F910F9169
:10456000FF90EF90DF90CF90BF90AF909F908F9093
:1045700008950F931F93BC0103EA10E1C8010E9444
:10458000890DC8011F910F9108954F925F927F92FC
:104590008F929F92AF92BF92CF92DF92EF92FF9253
:1045A0000F931F93DF93CF93CDB7DEB7CB57D04098
:1045B0000FB6F894DEBF0FBECDBF782E4B012A0197
:1045C000EC960CAF1DAF2EAF3FAFEC97F8E0CF2EBF
:1045D000D12CCC0EDD1EC6016FE371E00E9441BFFD
:1045E0000E94F2B5AB01BC017E010894E11CF11CF4
:1045F000C7012AE00E9474BFC601B7010E94F0BE45
:1046000066E471E00E94D4BEBC018E01015F1F4FC1
:10461000C8010E9420C084EA9CE0B8010E94B51C39
:10462000C8010E9431C0C7010E942BC0C6010E9470
:1046300031C083E0871520F081E07816B0F509C01D
:1046400084E0781609F473C085E0781609F0FEC09E
:10465000A9C08EE891E00E94B922BC01EDE1CE2E06
:10466000D12CCC0EDD1EC6010E9441BF56E1E52EC5
:10467000F12CEC0EFD1EC701B4014AE00E94A6BF5A
:10468000C601B7010E94F0BE66E471E00E94D4BE8C
:104690008C01C2010E94B922BC01C8010E94D4BE93
:1046A000BC018E010C5D1F4F6DC083E991E00E943B
:1046B000B922BC0142E3A42EB12CAC0EBD1EC50133
:1046C0000E9441BF3BE2C32ED12CCC0EDD1EC601A1
:1046D000B4014AE00E94A6BFC501B6010E94F0BE27
:1046E0006AE471E00E94D4BE8C0129E3E22EF12C31
:1046F000EC0EFD1E672D70E061507040C7014AE06E
:104700000E94A6BFC801B7010E94F0BE66E471E036
:104710000E94D4BE8C01C2010E94B922BC01C80112
:104720000E94D4BEBC018E01005C1F4F7BC088E993
:1047300091E00E94B922BC019EE4C92ED12CCC0E7E
:10474000DD1EC6010E9441BF87E4E82EF12CEC0E6D
:10475000FD1EC701B4014AE00E94A6BFC601B70111
:104760000E94F0BE66E471E00E94D4BE8C01C201DA
:104770000E94B922BC01C8010E94D4BEBC018E01B6
:104780000B5A1F4FC8010E9420C084EA9CE0B80168
:104790000E94B51CC8010E9431C0C7010E942BC0F5
:1047A000C60152C08DE991E00E94B922BC0103E626
:1047B000A02EB12CAC0EBD1EC5010E9441BF1CE550
:1047C000C12ED12CCC0EDD1EC601B4014AE00E94E0
:1047D000A6BFC501B6010E94F0BE64E571E00E946B
:1047E000D4BE8C010E944F86BC01BAE6EB2EF12CA0
:1047F000EC0EFD1EC7014AE00E94A6BFC801B7012A
:104800000E94F0BE66E471E00E94D4BE8C01C20139
:104810000E94B922BC01C8010E94D4BEBC018E0115
:104820000F581F4FC8010E9420C084EA9CE0B801C5
:104830000E94B51CC8010E9431C0C7010E942BC054
:10484000C6010E942BC0C5010E9431C0EC966CAD20
:104850007DAD8EAD9FADEC9728E23BE64EE65EEC7B
:104860000E94ACC5882339F484EA9CE06DE571E0D0
:104870000E94FE1A26C08091A40C83FF22C0809162
:10488000A50C882361F085E393E1EC964CAD5DAD1A
:104890006EAD7FADEC9722E030E00E9435BD809197
:1048A000A60C882371F08091A70C9091A80CEC962F
:1048B0004CAD5DAD6EAD7FADEC9722E030E00E9477
:1048C00035BDC558DF4F0FB6F894DEBF0FBECDBF64
:1048D000CF91DF911F910F91FF90EF90DF90CF90DC
:1048E000BF90AF909F908F907F905F904F90089572
:1048F0000F931F9308E21BE62EE63EEC0E94C522B2
:104900001F910F910895EF92FF920F931F93F82E2E
:10491000E62E8A0185E19EE00E94B922BC0184EA6C
:104920009CE00E94472084EA9CE06F2D0E94AE1F0D
:104930008EE19EE00E94B922BC0184EA9CE00E94C4
:10494000472084EA9CE06E2D0E94AE1F88E29EE024
:104950000E94B922BC0184EA9CE00E94472084EABC
:104960009CE0F801608140E150E00E94CD1F82E3AD
:104970009EE00E94B922BC0184EA9CE00E9447208C
:1049800084EA9CE0F801618140E150E00E94CD1F83
:104990008CE39EE00E94B922BC0184EA9CE00E9464
:1049A000472084EA9CE0F801628140E150E00E94E7
:1049B000CD1F86E49EE00E94B922BC0184EA9CE0FF
:1049C0000E94472084EA9CE0F801638140E150E0C6
:1049D0000E94CD1F80E59EE00E94B922BC0184EABE
:1049E0009CE00E94472084EA9CE0F801648140E159
:1049F00050E00E94CD1F8AE59EE00E94B922BC01D2
:104A000084EA9CE00E944720E090DD04F090DE0400
:104A10000091DF041091E0048091A40C80FF1AC083
:104A20008091A50C882341F085E393E1B801A701AB
:104A30002AE030E00E94D7BB8091A60C882351F079
:104A40008091A70C9091A80CB801A7012AE030E052
:104A50000E94D7BB8091A40C80FF16C08091A50C4A
:104A6000882331F085E393E16DE571E00E9449BD53
:104A70008091A60C882341F08091A70C9091A80CFE
:104A80006DE571E00E9449BD1F910F91FF90EF907D
:104A900008950F931F93CF93DF93EC018B018881CF
:104AA00084FF0FC08981882321F085E393E10E9470
:104AB000FBBA8A81882329F08B819C81B8010E94EE
:104AC000FBBADF91CF911F910F9108950F931F9320
:104AD000CF93DF93EC018B01888183FF0FC0898125
:104AE000882321F085E393E10E943CBB8A818823DF
:104AF00029F08B819C81B8010E943CBBDF91CF9152
:104B00001F910F9108952F923F924F925F926F9253
:104B10007F928F929F92AF92BF92CF92DF92EF924D
:104B2000FF920F931F93DF93CF93CDB7DEB76A97B2
:104B30000FB6F894DEBF0FBECDBF84EA9CE06FE6EF
:104B40007EE00E9466251A8E198EB7EF2B2EB1E0FB
:104B50003B2E298D3A8D229D8001239D100D329D83
:104B6000100D11240A56194FC8010E94FD8B6F8742
:104B7000788B898B9A8BC8010E940D8C6B017C010C
:104B8000C8010E943F8C6B877C878D879E87C801F8
:104B90000E944B8C4B015C01C8010E945C8C6F83AE
:104BA000788789879A87C8010E946F8C2B013C0106
:104BB000C801B701A6010E94F58BC8014F8558892D
:104BC00069897A890E94058CC801B501A4010E94F7
:104BD000398CC8014B855C856D857E850E94458C2E
:104BE000C801B2010E94518CC8016F8178850E9472
:104BF000648C898D9A8D01969A8F898F039709F01D
:104C0000A8CF1E821D828D819E810E944A86ED81E1
:104C1000FE812AE130E0E29F7001E39FF00CF29FF9
:104C2000F00C112482EE94E0E80EF91EC7010E94F8
:104C300063862C01009709F4AAC09A8F898F8C0192
:104C4000000F111F000F111FC8010E94B20B9E8B95
:104C50003C018D8BC8010E94B20B9F8B4C018C8B49
:104C6000C8010E94B20B988F5C018B8BB20161501E
:104C70007040C7010E94888669837A838B839C83F6
:104C800022243324CC24DD2435C0C701698D7A8DDC
:104C90000E9488869B01AC0183010C0D1D1D69815A
:104CA0007A818B819C810E9447C5F8016083718362
:104CB00082839383C701698D7A8D0E94C386F40134
:104CC000EC0DFD1D6083718382839383C701698D21
:104CD0007A8D0E94FE86F501EC0DFD1D90586083D3
:104CE0007183828393830894211C311C24E030E07B
:104CF000C20ED31E898D9A8D01979A8F898F2414A5
:104D000035041CF2C7010E948486C7010E94BF8639
:104D1000C7010E94FA86C701B2010E94CD8800E057
:104D200010E0CC24DD2424C0F301EC0DFD1D4081F6
:104D3000518162817381C7010E946786F401EC0D85
:104D4000FD1D4081518162817381C7010E949A8655
:104D5000F501EC0DFD1D4081518162817381C70118
:104D60000E94D5860F5F1F4FE4E0F0E0CE0EDF1EFD
:104D700004151505CCF28D899E890E945C0C8C89E6
:104D80009F890E945C0C8B89988D0E945C0C2D8100
:104D90003E812F5F3F4F3E832D832330310509F045
:104DA00032CF6A960FB6F894DEBF0FBECDBFCF915B
:104DB000DF911F910F91FF90EF90DF90CF90BF9008
:104DC000AF909F908F907F906F905F904F903F90AB
:104DD0002F9008950F931F93CF93DF93EC018B01D6
:104DE000888184FF0FC08981882321F085E393E1C6
:104DF0000E943CBB8A81882329F08B819C81B80169
:104E00000E943CBBDF91CF911F910F910895EF92CB
:104E1000FF920F931F93E82E84EA9CE06DED72E100
:104E20000E94EA268091A1048823F1F084EA9CE0A4
:104E300063EB72E10E94EA26EE2021F0809191104E
:104E4000882371F58091A004813039F484EA9CE0D4
:104E500060E872E10E94EA261AC084EA9CE066E5F6
:104E600072E10E94EA261CC0E090B803F090B903FA
:104E700000E010E081E896E00E94CFA4E616F70675
:104E80000807190798F080919110882379F481E040
:104E900008C090919110911191E081E0892701C0A3
:104EA00080E01F910F91FF90EF9008950E94F2B55E
:104EB0007B018C0180918D1090918E10A0918F10AC
:104EC000B0919010E81AF90A0A0B1B0B81E896E0E2
:104ED0000E94CFA42091B8033091B90340E050E084
:104EE000621B730B840B950BE616F7060807190770
:104EF000B8F2CFCF0F931F93DF93CF93CDB7DEB729
:104F000027970FB6F894DEBF0FBECDBF8093E104A4
:104F10008091A40C83FF16C08091A50C882331F0EA
:104F200085E393E169EA7EE00E94FBBA8091A60CDA
:104F3000882341F08091A70C9091A80C69EA7EE04B
:104F40000E94FBBA8E010F5F1F4FC8016091E10400
:104F50004AE00E94D7BF8091A40C83FF16C08091C5
:104F6000A50C882329F085E393E1B8010E9490BD48
:104F70008091A60C882349F08091A70C9091A80CF1
:104F8000BE016F5F7F4F0E9490BDCE0101960E94CF
:104F90002BC08091E1048823C9F086E996E040E0C7
:104FA00050E060E070E00E94BF8A8DE898E040E049
:104FB00050E060E070E00E94BF8A84E89AE040E040
:104FC00050E060E070E00E94BF8A03C080E00E9471
:104FD0000B1127960FB6F894DEBF0FBECDBFCF9151
:104FE000DF911F910F9108950F931F93CF93DF933C
:104FF000EC018B01888184FF0FC08981882321F017
:1050000085E393E10E9490BD8A81882329F08B81FA
:105010009C81B8010E9490BDDF91CF911F910F91AB
:1050200008952F923F924F925F926F927F928F924C
:105030009F92AF92BF92CF92DF92EF92FF920F9327
:105040001F93DF93CF9300D000D00F92CDB7DEB780
:10505000D82E6D838091A204882309F455C02D2D8C
:1050600030E087EF91E0AC01249FC001259F900DB7
:10507000349F900D11248A56994F0E9437953B0119
:105080004C0181E896E00E94E3A47C0181E896E06F
:105090000E94EBA41B012C0181E896E00E94E7A48A
:1050A0005C01C401B30120E030E04AEF55E40E9406
:1050B000B0C520E030E04AE754E40E94FFC63B015F
:1050C0004C0100E010E0CC24DD24EA0CFB1C0C1D9C
:1050D0001D1DE20CF31C041D151DC801B7010E9423
:1050E00049C69B01AC01C401B3010E9447C50E949F
:1050F0001DC6AB01BC0181E896E00E94C9A45D8198
:10510000552309F0B4C0B5C00E942A8C882309F049
:105110004DC081E896E00E94CFA47B018C0181E81C
:1051200096E00E94E3A43C0181E896E00E94EBA493
:105130001B012C0181E896E00E94E7A45C012D2D63
:1051400030E087EF91E0FC012E9FC0012F9F900D72
:105150003E9F900D11248A56994F0E94379569837E
:105160007A838B839C8388249924E618F70808099E
:105170001909E218F30804091509CC24DD24EA18FA
:10518000FB080C091D09C801B7010E9449C620E0AF
:1051900030E04AE754E40E94B0C59B01AC0169814C
:1051A0007A818B819C810E94B0C514C00E942A8C98
:1051B000882391F08D2D90E027EF31E0AC01429FE4
:1051C000C001439F900D529F900D11248A56994F14
:1051D0000E9437957B018C0184EA9CE061E37FE0CB
:1051E0000E94492584EA9CE0B801A7010E94D21CD4
:1051F000C801B70120E030E04AE756E40E94FBC650
:10520000882344F084EA9CE067E17FE00E94EA267C
:1052100080E032C05D81552361F1C801B70120E013
:1052200030E04AEF55E40E94FBC6882364F0C801D1
:10523000B70120E030E04AE756E40E94ACC588237D
:1052400014F484E019C0C801B70120E030E04AEF4F
:1052500055E40E94ACC5882374F4C801B70120E06E
:1052600030E04AE755E40E94FBC6181624F488E0B3
:1052700003C081E001C080E10F900F900F900F906C
:105280000F90CF91DF911F910F91FF90EF90DF90E2
:10529000CF90BF90AF909F908F907F906F905F90D6
:1052A0004F903F902F9008950F931F93CF93DF93CC
:1052B000182F062F84EA9CE069EF7EE00E94EA2620
:1052C0000E94F2B58091C1048823B1F5212F30E00E
:1052D00087EF91E0289FE001299FD00D389FD00DE6
:1052E0001124CA56D94FCE010E944F8A882321F536
:1052F000812F61E00E941128182F002321F08823BC
:10530000A9F011E013C0882311F41FEF0FC0CE01E4
:10531000612F0E94F99A84EA9CE062EE7EE00E948E
:10532000492584EA9CE0612F0E94701F812FDF9144
:10533000CF911F910F91089584EA9CE064EB7EE089
:105340000E94EA2610E0F2CF60E00E9454290895FE
:1053500060E00E9411280895EF92FF921F93CF936F
:10536000DF9310E0C0E0D0E081E0E82EF12C8C2F3C
:105370000E94A829813041F4C7010C2E02C0880F79
:10538000991F0A94E2F7182B2196C330D10579F7BB
:10539000812FDF91CF911F91FF90EF90089590E0C2
:1053A00027EF31E0AC01429FC001439F900D529F17
:1053B000900D11248A56994F0E94F6890895EF9214
:1053C000FF921F93CF93DF9310E0C0E0D0E091E015
:1053D000E92EF12C8C2F0E94CF29813041F4C70196
:1053E0000C2E02C0880F991F0A94E2F7182B219601
:1053F000C330D10579F7812FDF91CF911F91FF90B5
:10540000EF9008950F931F93DF93CF930F92CDB733
:10541000DEB76983082F10E087EF91E0AC01049FAD
:10542000C001059F900D149F900D11248A56994F2D
:105430000E94CE96C801880F991F800F911F23E00C
:10544000880F991F2A95E1F78396BE016F5F7F4F02
:105450000E9421190F90CF91DF911F910F91089514
:105460002F923F924F925F926F927F928F929F9274
:10547000AF92BF92CF92DF92EF92FF920F931F9362
:10548000DF93CF93CDB7DEB768970FB6F894DEBF42
:105490000FBECDBF80E090E064EB73E00E94D518B2
:1054A00082E090E069EA73E04AE00E9462AB8AE53C
:1054B00090E068E974E00E94D9188BE590E06AE911
:1054C00074E00E94D9188CE590E069E974E00E94CC
:1054D000D91880919804823010F01092980480912D
:1054E0009A04823010F010929A04809199048230CC
:1054F00010F01092990419821A821D821E821F8256
:10550000188619861A861B861C861D861E861F868F
:10551000188A198A1A8A1B8A1C8A80E090E0A0E007
:10552000B0E08D8B9E8BAF8BB88F1C821B82F9EA0B
:10553000AF2EF4E0BF2ECC24DD24E2E2EE2EF12CDF
:1055400071E1272E312C2C0E3D1E65E1462E512C8B
:105550004C0E5D1E53E0652E712C6C0E7D1E47EFC8
:10556000842E41E0942EC701BE016F5F7F4F0E94E1
:10557000D918C7010196BE016E5F7F4F0E94DD18EA
:10558000C7014097BE016B5F7F4F0E94E118C701C2
:105590000897BE01675F7F4F0E94E118C70104971B
:1055A000BE01635F7F4F0E94E118C7010C97B101F4
:1055B0000E94E118C7010496B2010E94E518C701D4
:1055C0000296B3010E94E918C89C8001C99C100D85
:1055D000D89C100D11240A56194FC80169810E94E8
:1055E000F99A81E191E16C2D49810E948716C801E9
:1055F0006A810E94CE964D895E896F89788DC80137
:105600000E94198A6B817C81C8010E94A88A8091BE
:105610009804882339F04D815E816F817885C801B7
:105620000E94158C80919A04882371F049855A85CF
:105630006B857C85C8010E94F58B4D855E856F85E5
:105640007889C8010E94058C80919904882349F0CB
:1056500089899A89AB89BC89F50180839183A2836A
:10566000B3830894C11CD11C88E190E0E80EF91EB8
:10567000E4E0F0E0AE0EBF1EF3E0CF16D10409F077
:1056800072CF0AE510E0B80165517F4EC8010E9453
:10569000D1180F5F1F4F09361105A9F768960FB68D
:1056A000F894DEBF0FBECDBFCF91DF911F910F9158
:1056B000FF90EF90DF90CF90BF90AF909F908F9032
:1056C0007F906F905F904F903F902F9008958091C2
:1056D0009406882331F080918711882391F01092ED
:1056E000871180919E04873041F080919F0487301C
:1056F00021F08BE79CE062E00AC08BE79CE066E06B
:1057000006C081E0809387118BE79CE064E00E94F3
:1057100087A40895843051F484EA9CE067ED74E135
:105720000E94EA268BE79CE064E014C08230A9F472
:1057300084EA9CE062EC74E10E94EA268091A30472
:105740009091A40401969093A4048093A3048BE702
:105750009CE065E00E9487A40895863011F40E94C1
:10576000672B08958BE79CE060E00E9487A481E8A6
:1057700096E00E94A8A5089586E996E00E944F8AC7
:10578000882361F48DE898E00E944F8A882331F4E1
:1057900084E89AE00E944F8A8823F9F08091A70458
:1057A0008823D9F482E00E944E1586E996E00E9493
:1057B000958AAC0160E070E08FEA91E10E94807F01
:1057C0008FEA91E168E272E32FEF3FEF4FEF5FEF77
:1057D0000E94977F81E08093A70408954F925F9283
:1057E0006F927F928F929F92AF92BF92CF92DF92F1
:1057F000EF92FF920F931F93CF93DF93582E3A01AE
:105800004B01422E222309F042C0282F30E087EFBF
:1058100091E0289F6001299FD00C389FD00C112463
:1058200086E996E0C80ED91EC60164E00E94F99A86
:10583000C6010E94C589E82EC6010E94CA895C0182
:10584000C401B3010E944BC63B014C01FF2400E0A0
:1058500010E0C801B7010E9449C67B018C01CC242D
:10586000B7FCC094DC2CC601B5010E944BC69B015D
:10587000AC01C801B7010E94B0C59B01AC01C401D5
:10588000B3010E94FFC60E9418C63B014C0184EA86
:105890009CE060E67EE00E94492584EA9CE0652D5C
:1058A0000E94EE1F84EA9CE06EE571E00E94642095
:1058B00084EA9CE0B401A3010E941522252D30E06A
:1058C00087EF91E0289FE001299FD00D389FD00DF0
:1058D0001124CA56D94FCE010E94648AA0E0B0E0DC
:1058E000BC01CD010E9449C6AB01BC01CE010E94A2
:1058F000BF8ACE01B401A30121E00E940D9F84EA7A
:105900009CE06CE671E00E946420CE010E94058A52
:10591000AB01BC0184EA9CE00E94D21C84EA9CE0BA
:1059200064E771E00E946420CE010E94148A682F0F
:1059300084EA9CE00E94701F0E94BC2B442021F44A
:10594000CE0161E00E949896DF91CF911F910F9157
:10595000FF90EF90DF90CF90BF90AF909F908F908F
:105960007F906F905F904F90089520E00E94EE2B03
:1059700008950F931F9390E027EF31E0829F8001FD
:10598000839F100D929F100D11240A56194FC801C4
:1059900064E00E94F99AC8010E94648AA0E0B0E025
:1059A000BC01CD010E9449C6AB01BC01C8010E94E7
:1059B000BF8AC8010E94599F0E94BC2BC80161E0A8
:1059C0000E9498961F910F91089586E996E00E9493
:1059D0004F8A8823A1F48DE898E00E944F8A88239B
:1059E00071F484E89AE00E944F8A882341F40E946F
:1059F000B92C81E00E94B92C82E00E94B92C089554
:105A00006F927F928F929F92AF92BF92CF92DF92CE
:105A1000EF92FF920F931F93CF93DF9390E027EFC6
:105A200031E0829FE001839FD00D929FD00D112421
:105A3000CA56D94FCE010E940D8C7B018C01CE013C
:105A40000E94FD8B5B016C01CE010E94FD8B3B012E
:105A50004C01CE010E941D8C30E0EA18FB080C09B5
:105A60001D091E141F04100611060CF431E020E07D
:105A7000661A770A880A990A161417041804190472
:105A80000CF421E0321719F0CE0161E002C0CE0122
:105A900060E00E945896CE0164E00E94F99ACE011F
:105AA0000E94648AA0E0B0E0BC01CD010E9449C61A
:105AB000AB01BC01CE010E94BF8ACE010E94679F4C
:105AC0000E94BC2BCE0161E00E949896DF91CF919D
:105AD0001F910F91FF90EF90DF90CF90BF90AF900C
:105AE0009F908F907F906F90089586E996E00E9436
:105AF0004F8A8823A1F48DE898E00E944F8A88237A
:105B000071F484E89AE00E944F8A882341F40E944D
:105B1000002D81E00E94002D82E00E94002D08955A
:105B20002F923F924F925F926F927F928F929F92AD
:105B3000AF92BF92CF92DF92EF92FF920F931F939B
:105B4000DF93CF9300D000D000D0CDB7DEB749832C
:105B50005A836B837C8327EF31E0829FA001839F70
:105B6000500D929F500D11244A56594F5E834D831C
:105B7000CA010E94FB897B018C0169817A818B813A
:105B80009C8120E030E040E050E00E94FBC6181607
:105B90002CF4A980BA80CB80DC8008C0A980BA80B0
:105BA000CB80DC80D7FAD094D7F8D0948D819E81B9
:105BB0000E94648AA0E0B0E0BC01CD010E9449C609
:105BC0009B01AC01C601B5010E94FBC618162CF062
:105BD000A980BA80CB80DC8029C069817A818B81E1
:105BE0009C8120E030E040E050E00E94ACC588237A
:105BF0008CF48D819E810E94648AA0E0B0E0BC019B
:105C0000CD010E9449C65B016C01D7FAD094D7F848
:105C1000D0940CC08D819E810E94648AA0E0B0E087
:105C2000BC01CD010E9449C65B016C018D819E8142
:105C3000B601A5010E94BF8AC801B70120E030E08B
:105C400040E050E00E94FBC618165CF4C801B701A2
:105C500020E030E040E85FE30E94ACC587FD0BC068
:105C60003BC0C801B70120E030E040E85FEB0E9494
:105C7000FBC6181604F5C601B50120E030E040E08F
:105C800050E00E94FBC6181664F4C601B50120E07E
:105C900030E040E85FE30E94FBC618160CF47DC0BC
:105CA0000AC0C601B50120E030E040E85FEB0E9489
:105CB000ACC587FD5CC0C801B70120E030E040E022
:105CC00050E00E94FBC618163CF01701280157FA55
:105CD000509457F8509402C017012801C601B5012D
:105CE00020E030E040E050E00E94FBC618161CF4B3
:105CF0003501460106C03501460197FA909497F8A0
:105D00009094C801B701A20191010E94B0C57B0126
:105D10008C01C601B501A40193010E94B0C59B018D
:105D2000AC01C801B7010E94ACC5882309F44CC07E
:105D3000C601B50120E030E040E050E00E94FBC623
:105D400018165CF4C601B50120E030E040E85FE3DE
:105D50000E94FBC618160CF137C0C601B50120E041
:105D600030E040E85FEB0E94ACC588236CF5C601CB
:105D7000B50120E030E040E85FE30E94FBC6181662
:105D800064F0C601B50120E030E040E85FE30E9426
:105D9000ACC588231CF410E001C011E08D819E8108
:105DA00061E00E940F8A8D819E81612F20E030E0AA
:105DB00040E050E00E947D9F0E94BC2B84EA9CE062
:105DC00062E87EE00E94662569817A818B819C81F0
:105DD00020E030E040E050E00E94ACC5882339F577
:105DE00086E996E00E94FB8920E030E040E050E048
:105DF0000E94ACC5882311F58DE898E00E94FB89CC
:105E000020E030E040E050E00E94ACC58823B1F4CF
:105E100084E89AE00E94FB8920E030E040E050E016
:105E20000E94ACC5882351F41092DC0407C00E9484
:105E30001011882319F081E08093DC0426960FB6B8
:105E4000F894DEBF0FBECDBFCF91DF911F910F91B0
:105E5000FF90EF90DF90CF90BF90AF909F908F908A
:105E60007F906F905F904F903F902F9008952F926A
:105E70003F924F925F926F927F928F929F92AF92DA
:105E8000BF92CF92DF92EF92FF920F931F93CF9327
:105E9000DF930E94F2B57B018C01809134059091D3
:105EA0003505A0913605B0913705E81AF90A0A0BB5
:105EB0001B0B0E945E86AA2797FDA095BA2F8E1510
:105EC0009F05A007B10708F0E5C044245524AAE1C6
:105ED0002A2E312C429CE001439CD00D529CD00DC7
:105EE0001124CE51DB4FCE010E946386BC0161506C
:105EF0007040CE010E9488867B018C010E942A8C12
:105F0000882371F481E896E00E94CFA40E9449C6DC
:105F10009B01AC01C801B7010E94FFC67B018C0147
:105F2000CE010E946386181619060CF082C060919B
:105F300038057091390580913A0590913B050E9492
:105F400049C63B014C016091D2047091D304809109
:105F5000D4049091D5040E9449C69B01AC01C801AC
:105F6000B7010E9448C59B01AC01C401B3010E9466
:105F7000FBC618160CF450C0CE0160E070E00E9421
:105F800088867B018C016091D2047091D30480914A
:105F9000D4049091D5040E9449C69B01AC01C8016C
:105FA000B7010E9448C59B01AC01C401B3010E9426
:105FB000ACC587FD31C0609138057091390580917D
:105FC0003A0590913B050E9449C65B016C01CE01E8
:105FD0000E946386BC0161507040CE010E94888699
:105FE0007B018C016091D2047091D3048091D40420
:105FF0009091D5040E9449C63B014C01C801B701EC
:10600000A40193010E9448C59B01AC01C601B501E2
:106010000E94FBC6181604F5A0E050E040E060E0E6
:10602000C2012A2F352FE42FF62FA901BF010E94AC
:10603000902D0894411C511C83E04816510409F02E
:1060400049CF0E94F2B56093340570933505809373
:106050003605909337051EC060913805709139055B
:1060600080913A0590913B050E9449C6A401930195
:106070000E9447C5AB01BC01CE010E94948820E07C
:1060800030E04AE754E40E94FFC6A62F572F482F5E
:10609000692FC6CFDF91CF911F910F91FF90EF90A5
:1060A000DF90CF90BF90AF909F908F907F906F9038
:1060B0005F904F903F902F9008959F92AF92BF9224
:1060C000CF92DF92EF92FF920F931F93CF93DF93C4
:1060D000982E10E0CC24DD2407EFA02E01E0B02E96
:1060E000CA9CE001CB9CD00DDA9CD00D1124CA567D
:1060F000D94FCE010E9460968130A9F5CE010E9451
:10610000E089892B81F1CE0164E00E94F99ACE01E9
:106110000E94648AA0E0B0E0BC01CD010E9449C6A3
:10612000AB01BC01CE010E94BF8ACE010E940D8C42
:106130007B018C01CE010E94FD8B20E0E61AF70A5C
:10614000080B190B1E141F04100611060CF421E095
:10615000CE01622F21E030E040E050E00E947D9FC0
:106160000E94BC2B11E00894C11CD11C23E0C21674
:10617000D10409F0B5CF112389F0992079F40E9458
:10618000F2B57B018C010E94F2B56E197F09800B7C
:10619000910B6C52714080409040A8F3C0E0D0E079
:1061A000B7EFEB2EB1E0FB2ECE9D8001CF9D100D01
:1061B000DE9D100D11240A56194FC8010E94659CDE
:1061C00084EA9CE06FE67FE00E944925C8010E94B6
:1061D000C589682F84EA9CE00E94701F2196C33015
:1061E000D10511F784EA9CE064E57FE00E94EA268D
:1061F000DF91CF911F910F91FF90EF90DF90CF90A3
:10620000BF90AF909F90089580E00E945D30089508
:106210008F929F92BF92CF92DF92EF92FF920F9355
:106220001F93CF93DF9380E896E00E940C89B82EED
:1062300086E996E00E94F189882309F06BC08DE819
:1062400098E00E94F189882309F064C084E89AE00C
:106250000E94F189882309F05DC08BE79CE06B2DDB
:106260000E9487A45EC0C89CE001C99CD00DD89C48
:10627000D00D1124CA56D94FCE010E94F18988232E
:10628000F1F1CE010E945C8C6115710581059105CB
:1062900031F1E090A304F090A40400E010E0CE01FE
:1062A0000E945C8C6E157F058007910720F00E948C
:1062B0002A8C882321F10E942A8C882381F0E09087
:1062C000B504F090B6040091B7041091B804CE0163
:1062D0000E945C8C6E157F058007910780F4CE01CB
:1062E0000E94D2A10E942A8C882321F48BE79CE093
:1062F00063E003C08BE79CE06B2D0E9487A40894A9
:10630000C11CD11C83E0C816D10409F0ACCF0E9497
:10631000BC2B07C0CC24DD2487EF882E81E0982E8B
:10632000A2CFDF91CF911F910F91FF90EF90DF905F
:10633000CF90BF909F908F9008958F929F92AF9231
:10634000BF92CF92DF92EF92FF920F931F93DF9352
:10635000CF9300D000D0CDB7DEB7EE24FF2422E1EA
:10636000C22ED12C97EF892E91E0992E5E010894D0
:10637000A11CB11CE89C8001E99C100DF89C100D3B
:1063800011240A56194FC8010E94A296C8010E9402
:106390001D8C69837A838B839C83C601B5010E941F
:1063A00025190894E11CF11C88E190E0C80ED91E63
:1063B00093E0E916F104F1F61092A70481E00E943F
:1063C0004E158FEA91E10E94887F0F900F900F90F9
:1063D0000F90CF91DF911F910F91FF90EF90DF9081
:1063E000CF90BF90AF909F908F9008951F93CF93C1
:1063F000DF93EC0181EC90E164E00E949E15182F80
:10640000833031F40E94F2B56E8F7F8F88A399A3F9
:106410000E944A19882311F4188216C01130A1F481
:106420000E94F2B52E8D3F8D48A159A1621B730BBE
:10643000840B950B615D77408040904028F01AA254
:106440000E949D3183E08883DF91CF911F91089551
:10645000AF92BF92CF92DF92EF92FF920F931F9372
:10646000CF93DF9358E9E52E56E0F52E00E010E0DB
:1064700047EFA42E41E0B42E31E0C32ED12C0A9D6B
:10648000E0010B9DD00D1A9DD00D1124CA56D94F95
:10649000CE010E944F8A8823A9F0CE010E943E9629
:1064A000CE010E942F99882369F09601F7010080A0
:1064B00002C0220F331F0A94E2F78091A804822BB6
:1064C0008093A8040F5F1F4F87EF91E0E80EF91E3D
:1064D00003301105A1F681B39091A804892B81BBEB
:1064E00081E090E00E947FB691B38091A8048095EE
:1064F000892381BB1092A80486E996E00E944F8A06
:10650000882371F48DE898E00E944F8A882341F433
:1065100084E89AE00E944F8A882311F40E949D31FA
:10652000DF91CF911F910F91FF90EF90DF90CF906F
:10653000BF90AF90089586E996E00E944F8A882325
:1065400061F48DE898E00E944F8A882331F484E852
:106550009AE00E944F8A882311F00E949D3186E9BB
:1065600096E00E94448B8DE898E00E94448B84E87A
:106570009AE00E94448B08950E94627E80919E045E
:106580008650823048F460E08091C103882309F48A
:1065900061E088E10E9481B780919F04865082303B
:1065A00048F460E08091C103882309F461E089E147
:1065B0000E9481B780919110863021F48BE79CE096
:1065C00061E003C08BE79CE062E00E9487A408952D
:1065D0008CE060E00E9481B710929D0C08958CE0E1
:1065E00061E00E9481B781E080939D0C08958091C5
:1065F0009D0C882319F00E94E83208950E94EF3222
:1066000008950E94EA10882319F00E94EF3208953D
:106610000E94E83208951F93182F84EA9CE068E0F6
:1066200071E10E94492580E090E040E050E060E0A8
:1066300070E00E94902D81E090E040E050E060E04A
:1066400070E00E94902D82E090E040E050E060E039
:1066500070E00E94902D80E00E947A2710924C05F5
:1066600010924D051092D8041123A1F41092C80481
:106670001092C9041092CA041092CB041092CD0457
:106680001092CC040E94F814882321F00E94F51483
:106690000E9483250E942A8C823021F481E896E0B2
:1066A0000E94A8A50E9401331F91089580E00E94D6
:1066B0000B330895CF93DF9384EA9CE06CE271E1A1
:1066C0000E944925C0E0D0E084EA9CE06CE171E1E1
:1066D0000E94492584EA9CE06C2F0E94701FCE0125
:1066E00040E050E060E070E00E94902D2196C330C1
:1066F000D10551F781E080934D051092400510922D
:10670000410510924205109243050E94F2B5609334
:106710003C0570933D0580933E0590933F050E9494
:106720000133DF91CF910895AF92BF92CF92DF9264
:10673000EF92FF920F931F938091D704882309F063
:1067400063C080914D05882309F05EC00E94EA1065
:10675000882359F40F2EFDECAF2EFCECBF2EFCEC81
:10676000CF2EFDE3DF2EF02D0AC00F2EF6E6AF2E62
:10677000F6E6BF2EF6E6CF2EFFE3DF2EF02D0E94C9
:10678000F2B5209192113091931140919411509152
:106790009511621B730B840B950B615D77408040F4
:1067A000904068F00E94EF320E94F2B5609392111F
:1067B00070939311809394119093951125C00E942A
:1067C000F2B57B018C018091921190919311A0916F
:1067D0009411B0919511E81AF90A0A0B1B0BC60126
:1067E000B50120E030E04AEF54E40E94FFC60E9469
:1067F00018C6882777FD8095982F6E157F0580072E
:10680000910710F40E94E8321F910F91FF90EF90D2
:10681000DF90CF90BF90AF900895FC01EB5BFB4FF2
:1068200090E0662309F491E08081692F0E9481B78E
:1068300008954F925F926F927F928F929F92AF9244
:10684000BF92CF92DF92EF92FF920F931F93CF935D
:10685000DF932C017A018B018FEF90E0489EF001CD
:10686000499EF00D589EF00D1124E458F14FA08080
:10687000B180C280D380A416B506C606D7061CF028
:10688000CFEFDFEF02C0C1E0D0E08FEF90E0489E95
:10689000F001499EF00D589EF00D1124E657F14F7E
:1068A000608171818281938120E030E040E050E09E
:1068B0000E94ACC5882321F0C2010E94511195C0ED
:1068C000CE01880F991F3C01882477FC8094982C76
:1068D000A60CB71CC81CD91CC130D10531F4EA1470
:1068E000FB040C051D055CF408C0CF5FDF4F39F4D5
:1068F000AE14BF04C006D10614F4570168018FEF2F
:1069000090E0489EF001499EF00D589EF00D112434
:10691000E753F24F80E090E020E030E040E050E0CC
:10692000F8972083318342835383F8962083318301
:1069300042835383248F358F468F578F0196349629
:106940008730910569F78FEF90E0489EF001499EEE
:10695000F00D589EF00D1124E157F24FEC51FF4F0E
:106960002083318342835383E45EF0408AE097EDD5
:10697000A3E2BCE382839383A483B583E751FF4FF3
:1069800080819181A281B381E95EF040868F978FEB
:10699000A0A3B1A3680E791E8A1E9B1E62A273A2D9
:1069A00084A295A2EE51FF4F118210823B96A082E5
:1069B000B182C282D382A816B906CA06DB06A9F044
:1069C00081E090E0A0E0B0E0042C04C0880F991FA3
:1069D000AA1FBB1F0A94D2F720918A0D282B20935F
:1069E0008A0DC20161E00E940D34DF91CF911F91A9
:1069F0000F91FF90EF90DF90CF90BF90AF909F905E
:106A00008F907F906F905F904F9008952F923F925C
:106A10004F925F926F927F928F929F92AF92BF92AE
:106A2000CF92DF92EF92FF920F931F93DF93CF935A
:106A3000CDB7DEB728970FB6F894DEBF0FBECDBF37
:106A40008091880D882321F01092880D0E94DE121B
:106A5000F1E76F2EFEE07F2E18861F82D301589635
:106A60001C921E92579720E030E040E050E059968B
:106A70002D933D934D935C935C9710918A0D812FDC
:106A800090E00F8002C0959587950A94E2F780FF09
:106A900069C1ED91FC91FA83E9836F01CC0CDD1C97
:106AA000CC0CDD1C2F8138854FEF50E0249FC001B6
:106AB000259F900D349F900D1124C80ED91E81E999
:106AC0009DE0C80ED91ED6016D917D918D919C914E
:106AD00020E030E040E050E00E94ACC5882341F562
:106AE00081E090E0A0E0B0E00F8004C0880F991F23
:106AF000AA1FBB1F0A94D2F78095812380938A0D29
:106B0000EF81F88527EF31E0E29FC001E39F900D10
:106B1000F29F900D11248A56994F0E94F68988237E
:106B200009F420C18F81988560E00E940D341AC15C
:106B3000D30112968D919D910D90BC91A02D8B83C8
:106B40009C83AD83BE83BC01CD012DEC3CEC4CE4B9
:106B50005DE30E9448C57B018C01F301628373836E
:106B600084839583D601AD90BD90CD90DC90A60135
:106B700095010E94FBC687FF03C089819A8110C0DE
:106B8000C801B701A60195010E9447C5F3016283C0
:106B900073838483958389819A810196918380830D
:106BA000D30112968D909D90AD90BC9015978C015D
:106BB000000F111F000F111FEF81F8852FEF30E03C
:106BC000E29FC001E39F900DF29F900D1124080FEA
:106BD000191F0157124FD8015E966D917D918D91CD
:106BE0009C9191970E944BC66B017C01C501B40139
:106BF000F80122AD33AD44AD55AD0E94FFC69B01F7
:106C0000AC01C701B6010E9448C56B017C010A5A5C
:106C10001F4FC501B401D8012D913D914D915C915B
:106C20000E94FFC6A50194010E94FFC69B01AC0112
:106C3000C701B6010E9448C50E9418C61B012C015D
:106C4000F30187819085A185B28562015101A81A5F
:106C5000B90ACA0ADB0AD7FE08C0D094C094B0941F
:106C6000A094A11CB11CC11CD11CA114B104C1046D
:106C7000D10409F477C0882482159305A405B505CD
:106C800014F4882483942F8138854FEF50E0249F9B
:106C9000F001259FF00D349FF00D1124E958F14FBC
:106CA0008081881671F08B819C81AD81BE81F3015A
:106CB00082839383A483B58329813A81318320839E
:106CC00043C0C601B5010E944BC623E333E343E84A
:106CD00052E40E94FFC67B018C0120E03FEF4FE7AA
:106CE00057E40E94FBC61816ACF0C801B70120E0BB
:106CF00030E040E85FE30E94ACC58823ACF40F2E7F
:106D0000F0E0EF2EF0E0FF2EF0E80F2FFFE31F2F53
:106D1000F02D0AC00F2EF0E0EF2EFFEFFF2EFFE761
:106D20000F2FF7E41F2FF02DD3015996ED92FD920E
:106D30000D931C935C975896BC92AE925797F301B3
:106D400027823086418652862F8138854FEF50E06A
:106D5000249FF001259FF00D349FF00D1124E95878
:106D6000F14F80828F819885019698878F83AFEF4E
:106D7000B0E06A0E7B1E039709F070CE81E080932D
:106D8000840D28960FB6F894DEBF0FBECDBFCF910D
:106D9000DF911F910F91FF90EF90DF90CF90BF9008
:106DA000AF909F908F907F906F905F904F903F90AB
:106DB0002F9008952F923F924F925F926F927F9201
:106DC0008F929F92AF92BF92CF92DF92EF92FF92FB
:106DD0000F931F93CF93DF9390E080918B0D8823C7
:106DE00009F491E090938B0D992309F467C04091C9
:106DF000780D5091790D41155105D9F02091720D02
:106E00003091730D80917E0D90917F0D820F931FB5
:106E10009093730D8093720D8217930750F4415035
:106E200050405093790D4093780D8DE261E00E94BF
:106E300081B740917A0D50917B0D41155105D9F0E4
:106E40002091740D3091750D8091800D9091810D80
:106E5000820F931F9093750D8093740D8217930783
:106E600050F44150504050937B0D40937A0D8EE288
:106E700061E00E9481B740917C0D50917D0D4115DC
:106E8000510509F4B1C02091760D3091770D8091B4
:106E9000820D9091830D820F931F9093770D8093B5
:106EA000760D8217930708F09FC0415050405093D1
:106EB0007D0D40937C0D8FE261E094C08091850D43
:106EC0009091860D01969093860D8093850D885E36
:106ED000934009F07DC01092860D1092850D80912F
:106EE000870D882319F081508093870D00EDC02E07
:106EF00003E0D02E1AEC812E13E0912EC8E8DEE0DC
:106F0000B4ECAB2EB3E0BB2EEE24FF24A1E04A2E5E
:106F1000512C612C712C22242A94322CD601ED9113
:106F2000FC9180819181892BD9F06A817B818C8150
:106F30009D8120E030E040E050E00E94ACC5882315
:106F400079F4D301C2010E2C04C0880F991FAA1F27
:106F5000BB1F0A94D2F72091890D282B2093890D0D
:106F6000D401ED91FD914D018881998191838083B8
:106F7000F601019111916F016A817B818C819D8164
:106F80000E941DC6D8016D937C938FEF90E0E89E20
:106F9000F001E99EF00DF89EF00D1124E958F14F33
:106FA0006081C85FD04088810E9481B7D501ED9192
:106FB000FD915D01318220820894E11CF11CC950D1
:106FC000DE4FB3E0EB16F10409F0A8CF1092840D68
:106FD0008DE260E00E9481B78EE260E00E9481B79E
:106FE0008FE260E00E9481B7DF91CF911F910F91F6
:106FF000FF90EF90DF90CF90BF90AF909F908F90D9
:107000007F906F905F904F903F902F9008951F93C7
:10701000CF93DF93182F863029F4C091BC03D09111
:10702000BD0304C0C091BE03D091BF0380919E04F4
:10703000181711F090E006C088E16091C1030E942A
:1070400081B791E080919F04181731F489E1609134
:10705000C1030E9481B702C0992369F0BE0180E09C
:1070600090E04CEB52E30E94047E0E944C7E8BE742
:107070009CE060E009C0163021F48BE79CE061E001
:1070800003C08BE79CE062E00E9487A4DF91CF9170
:107090001F910895809174118823A1F484E791E1F0
:1070A0000E94C3BA892B71F00E94F2B560937C11E3
:1070B00070937D1180937E1190937F1184E791E10D
:1070C0000E94CDBA80919E04873051F080919F0438
:1070D000873031F08BE79CE062E00E9487A408953E
:1070E00080919110882371F487E0809391100E9421
:1070F000F2B560937C1170937D1180937E11909313
:107100007F1108950E94F2B520917C1130917D117C
:1071100040917E1150917F11621B730B840B950B74
:107120002091BA033091BB0340E050E026173707A7
:107130004807590728F41092911087E00E940738F9
:107140000895FF920F931F93F82E062FE82FF0E07B
:10715000E256FB4F608381E0F816D9F1FF2019F465
:1071600082E00E94F6B318E1002329F4812F60E049
:107170000E94FEB633C006500230E8F0812F60E076
:107180000E94FEB6812F61E00E9481B7FF2021F0AE
:1071900081E0F81619F506C04091C00382E06AEE5E
:1071A0007BE605C04091C00383E066EE7BE650E0DD
:1071B0000E947AB313C0812F61E00E94FEB660E0A6
:1071C0008091C103882309F461E0812F0E9481B777
:1071D00005C083E00E94F6B319E1C6CF1F910F915D
:1071E000FF90089580E060919E040E94A13881E0A4
:1071F00060919F040E94A13890E080919E048430A9
:1072000009F491E080919F04843009F491E0909317
:10721000A1040895882399F080E00E943D1580E044
:1072200064E00E94A13881E064E00E94A1380E94DD
:10723000F23881E08093A2040E94EF32089580E04A
:1072400060E00E94A13881E060E00E94A1380E94C5
:10725000F2381092A2040E94E8320895EF92FF9251
:107260000F931F93CF93DF93EC017A018B018881F9
:1072700084FF14C08981882331F085E393E12AE0FB
:1072800030E00E9422BC8A81882341F08B819C815E
:10729000B801A7012AE030E00E9422BCDF91CF9123
:1072A0001F910F91FF90EF900895EF92FF920F932F
:1072B0001F930E942A8C8230F1F081E896E00E94B0
:1072C000FEA47C0181E896E00E94CFA49B01AC0162
:1072D00000E010E0C801B7010E94C7C7F62E072FD3
:1072E000182FE92E80914C058823A9F484EA9CE0AC
:1072F00064E97FE00EC00E943886F62E072F182F13
:10730000E92E80914C05882331F484EA9CE06CE7F7
:107310007FE00E94492580914C05882371F484EA1E
:107320009CE04F2D502F612F7E2D0E942E3984EA34
:107330009CE061E871E00E94E11A6F2D702F812FAF
:107340009E2D1F910F91FF90EF9008958F929F9225
:10735000AF92BF92CF92DF92EF92FF920F931F9363
:107360000E9455394B015C0181E8C82E86E0D82E79
:10737000C6010E94E7A47C01C6010E94EBA400E0C4
:1073800010E0E80CF91C0A1D1B1DE60EF71E081F75
:10739000191FB701C8011F910F91FF90EF90DF9067
:1073A000CF90BF90AF909F908F900895EF92FF92F3
:1073B0000F931F930E942A8C823079F460913805D4
:1073C0007091390580913A0590913B050E9449C61C
:1073D0007B018C010E9455390EC060913805709177
:1073E000390580913A0590913B050E9449C67B0181
:1073F0008C010E94A6399B01AC016091D20470916E
:10740000D3048091D4049091D504620F731F841F1C
:10741000951F0E9449C69B01AC01C801B7010E949B
:10742000B0C520E030E048EC52E40E94FFC60E9464
:1074300018C6CB011F910F91FF90EF9008950E9405
:107440002A8C823019F40E94553902C00E94A63954
:107450009B01AC018091D2049091D304A091D404FB
:10746000B091D504280F391F4A1F5B1FB901CA010B
:1074700008952F923F924F925F926F927F928F92D8
:107480009F92AF92BF92CF92DF92EF92FF920F93B3
:107490001F93DF93CF9300D000D0CDB7DEB70E940B
:1074A0005E15882309F494C10091A3041091A404EB
:1074B00081E896E00E94FEA40817190709F088C128
:1074C0008DC18091A004882359F480919C10882359
:1074D00039F484EA9CE063E270E10E94EA267EC10E
:1074E00080919E04863039F080919F04863019F097
:1074F00080E090E004C08091B8039091B9039C01B2
:10750000442737FD4095542F29833A834B835C836E
:1075100081E896E00E94CFA47B018C01A090380501
:10752000B0903905C0903A05D0903B056090480571
:107530007090490580904A0590904B0581E896E04F
:107540000E94CFA429813A814B815C812E153F0591
:107550004007510768F4A618B708C808D908621B85
:10756000730B840B950BA616B706C806D90620F038
:1075700080919110882321F08091A004882329F123
:107580008091380590913905A0913A05B0913B055D
:107590008093480590934905A0934A05B0934B0505
:1075A00010929610109297101092981010929910B5
:1075B00010929A1010929B108091A004882329F0B9
:1075C00081E080939C101092A00480919E048630EC
:1075D00021F080919F048630E9F581E00E94072721
:1075E0008823C1F1809197108823A1F5809196108E
:1075F000882379F486E0809391100E94073884EA0A
:107600009CE06BEE7FE00E94EA2681E0809396107A
:10761000E5C08091480590914905A0914A05B09137
:107620004B0529813A814B815C81820F931FA41FF6
:10763000B51F209138053091390540913A05509198
:107640003B05281739074A075B0708F4C7C081E0E4
:1076500080939710109291101092A004809199102D
:10766000882309F049C0809198108823D1F484EAD6
:107670009CE06BED7FE00E944925409138055091D8
:10768000390560913A0570913B0584EA9CE00E94BF
:107690003C2281E896E00E945DA581E080939810ED
:1076A0009DC0E0903805F090390500913A051091A1
:1076B0003B05A0904805B0904905C0904A05D09080
:1076C0004B0581E896E00E94E7A429813A814B812D
:1076D0005C81A20EB31EC41ED51EA0E0B0E0A80EB1
:1076E000B91ECA1EDB1EEA14FB040C051D0508F4B6
:1076F00075C081E08093991080919B10882309F0D8
:107700006DC080919A108823C9F484EA9CE068ECEB
:107710007FE00E94492540913805509139056091DC
:107720003A0570913B0584EA9CE00E943C2281E886
:1077300096E00E94A8A581E080939A1020903805D9
:107740003090390540903A0550903B0560904805CF
:107750007090490580904A0590904B0581E896E02D
:107760000E94E7A47C0181E896E00E94EBA45B0103
:107770006C0181E896E00E94E3A429813A814B8163
:107780005C81260D371D481D591D2A0D3B1D4C1DC2
:107790005D1D00E010E02E0D3F1D401F511FA0E0B9
:1077A000B0E0280F391F4A1F5B1F2216330644061C
:1077B0005506A0F011E010939B1010929C1084EAE3
:1077C0009CE06BEA7FE00E94EA261093931006C0CB
:1077D0008091A104882309F074CE82CE0F900F907F
:1077E0000F900F90CF91DF911F910F91FF90EF902D
:1077F000DF90CF90BF90AF909F908F907F906F90D1
:107800005F904F903F902F900895AF92BF92CF928C
:10781000DF92EF92FF920F931F93CF93DF938091AC
:107820009310882309F4C3C0E0903805F09039051F
:1078300000913A0510913B050E9455392091D204E0
:107840003091D3044091D4045091D504260F371FB2
:10785000481F591F2E153F054007510708F4A7C0C0
:1078600078C0CA9CE001CB9CD00DDA9CD00D1124CD
:10787000CE51DB4FCE010E94638602970CF455C0B7
:1078800060919410709195106F5F7F4F882777FDFE
:107890008095982F0E944BC67B018C01CE010E94DF
:1078A0006386BC0161507040CE010E9488869B01B6
:1078B000AC01C801B7010E94FBC61816B4F155C04F
:1078C000EB0121968091A50C882339F085E393E1A3
:1078D000BE014AE050E00E9485BC8091A60C88233E
:1078E00049F08091A70C9091A80CBE014AE050E0AD
:1078F0000E9485BC84EA9CE062E670E10E94492512
:1079000084EA9CE0B801A7010E94D21C84EA9CE0B2
:107910006DE571E00E94E11AC801B7010E9418C626
:10792000AB01BC018C2D0E94B52C0894C11CD11C4C
:1079300083E0C816D10409F094CF809194109091FF
:107940009510019690939510809394101092931037
:107950002EC084EA9CE06CE870E10E94EA26CC2408
:10796000DD249AE1A92EB12C7CCF60919410709106
:1079700095106F5F7F4F882777FD8095982F0E9425
:107980004BC6AB01BC01CE010E94A3887B018C01D8
:1079900084EA9CE06EE670E10E94492560919410B3
:1079A000709195108091A40C84FD8ACFA3CFDF91B4
:1079B000CF911F910F91FF90EF90DF90CF90BF90EC
:1079C000AF9008950F931F93CF93DF93EC018B013A
:1079D000888184FF13C08981882331F085E393E196
:1079E0004AE050E00E9472BC8A81882339F08B8182
:1079F0009C81B8014AE050E00E9472BCDF91CF91B7
:107A00001F910F910895EF92FF920F931F93CF93C1
:107A1000DF93182F80914D058823E9F0809144056C
:107A200090914505A0914605B091470520914005EC
:107A3000309141054091420550914305820F931FBB
:107A4000A41FB51F8093440590934505A093460558
:107A5000B0934705C3C084EA9CE06BE471E10E94E7
:107A600049250E942A8C682F84EA9CE070E00E94DD
:107A7000E23C84EA9CE06FE371E10E94EA26109206
:107A8000DA041092931010929510109294101092A4
:107A90004405109245051092460510924705109234
:107AA0004D05109248051092490510924A05109212
:107AB0004B051092961010929710109298101092F9
:107AC000991010929A1010929B1010929C10109284
:107AD000A4041092A304112361F41092CD04109217
:107AE000CC041092C4041092C5041092C6041092E3
:107AF000C7040E9455390E94A639112311F40E942F
:107B0000E5140E942A8C882361F481E896E00E94A3
:107B1000CFA40E9455390E94A63980E00E947A279E
:107B200041C081E00E947A2700E010E02AE1E22EC5
:107B3000F12C0E9DE0010F9DD00D1E9DD00D112446
:107B4000CE51DB4FCE010E946386181619062CF524
:107B5000CE0160E070E00E94888620E030E040E0E6
:107B600050E00E94ACC5882389F4CE0140E050E08B
:107B700060E070E00E94948820E030E04AE754E43E
:107B80000E94FFC6AB01BC01C80105C0C80140E0AE
:107B900050E060E070E00E94902D0F5F1F4F0330B7
:107BA000110539F6109238051092390510923A05F0
:107BB00010923B050E94F2B5609330057093310539
:107BC00080933205909333050E94F2B5609334059B
:107BD00070933505809336059093370581E0809347
:107BE0004C0510924D058093C303DF91CF911F91F7
:107BF0000F91FF90EF900895AF92BF92CF92DF92D6
:107C0000EF92FF920F931F930E94F2B55B016C01FC
:107C10008091380590913905A0913A05B0913B05C6
:107C20000097A105B10541F4A0927011B0927111B5
:107C3000C0927211D092731180914D05882349F141
:107C40000E94F2B520913C0530913D0540913E05E2
:107C500050913F05621B730B840B950B609340059D
:107C600070934105809342059093430584EA9CE01C
:107C700069EF70E10E94492540914005509141050E
:107C8000609142057091430584EA9CE00E943C2289
:107C900039C10E94F2B520913005309131054091F3
:107CA000320550913305621B730B840B950B2091A9
:107CB0004405309145054091460550914705621BAA
:107CC000730B840B950B6093380570933905809383
:107CD0003A0590933B050E9400B67B018C010E94FF
:107CE00000B66E197F09800B910B645F7140804074
:107CF0009040A8F3209138053091390540913A051C
:107D000050913B058091D2049091D304A091D4046A
:107D1000B091D504281739074A075B0740F58091D1
:107D2000D904882321F581E08093D60480917011D5
:107D300090917111A0917211B0917311A6019501EA
:107D4000281B390B4A0B5B0BDA01C901855F914097
:107D5000A040B04008F4D6C00E94F732A092701143
:107D6000B0927111C0927211D0927311CBC08091F8
:107D7000A204882319F00E94EF3202C00E94E83268
:107D80001092D6048091C303882351F00E942A8C5C
:107D9000823021F481E896E00E94A8A51092C303E6
:107DA0000E942A8C882331F08091D804882311F412
:107DB0000E94372F0E942A8C823011F00E94393A9B
:107DC0000E942A8C882331F48091D804882311F4EE
:107DD0000E94053C0E94A6399B01AC018091D90408
:107DE000882361F48091D2049091D304A091D404AB
:107DF000B091D504280F391F4A1F5B1F80913805A9
:107E000090913905A0913A05B0913B0528173907A3
:107E10004A075B0708F076C08091A604882329F101
:107E200084EA9CE06FED70E10E94662581E080931A
:107E3000D80480E090E040E050E060E070E00E9414
:107E4000902D81E090E040E050E060E070E00E9422
:107E5000902D82E090E040E050E060E070E00E9411
:107E6000902D80E00E947A274DC084EA9CE06BEC64
:107E700070E10E9466250E945E158823F1F18091D1
:107E8000C8049091C904A091CA04B091CB04209178
:107E900038053091390540913A0550913B05820FE4
:107EA000931FA41FB51F8093C8049093C904A09387
:107EB000CA04B093CB048091CC049091CD0420915E
:107EC000A3043091A404820F931F9093CD04809358
:107ED000CC0481E00E940B3381E08093D9040E949E
:107EE000EE140E94832584EA9CE06CEA70E10E9413
:107EF000662581E00E94033D05C00E94563381E063
:107F00008093DA041F910F91FF90EF90DF90CF9054
:107F1000BF90AF90089580E00E94033D0895CF92F6
:107F2000DF92EF92FF920F931F93CF93DF9385E33E
:107F300093E161E272E10E94FBBA85E393E16DE5B2
:107F400071E00E9449BD85E393E16FE072E10E9418
:107F5000FBBA0E94A639AB01BC0185E393E12AE09C
:107F600030E00E945EBC85E393E16FEF71E10E9417
:107F7000FBBA0E945539AB01BC0185E393E12AE0CD
:107F800030E00E945EBC85E393E162EF71E10E9404
:107F9000FBBA0E941215BC0185E393E14AE050E070
:107FA0000E9485BC85E393E16FED71E10E94FBBA0D
:107FB0000E942615AB01BC0185E393E12AE030E085
:107FC0000E945EBC85E393E16CEC71E10E94FBBA18
:107FD0000E94D639BC0185E393E14AE050E00E945B
:107FE00085BC85E393E16DEB71E10E94FBBA0E94D1
:107FF0002A8C682F85E393E14AE050E00E940EBC92
:1080000085E393E16AEA71E10E94FBBA0E94388637
:10801000AB01BC0185E393E12AE030E00E945EBC45
:10802000EE243AE1C32ED12C92C085E393E16DE9B1
:1080300071E10E94FBBA85E393E16E2D4AE050E0C6
:108040000E94FCBB85E393E165E971E10E943CBBC2
:1080500085E393E16DE571E00E9449BD85E393E11D
:1080600063E871E10E943CBBCC9D8001CD9D100D69
:10807000DC9D100D11240E511B4FFF240DC0C801B3
:10808000BE010E948886AB01BC0185E393E122E03A
:1080900030E00E9435BDF394CF2DD0E0C8010E949E
:1080A0006386C817D9075CF385E393E16DE571E05A
:1080B0000E9449BD85E393E161E771E10E943CBB09
:1080C000FF240DC0C801BE010E94C386AB01BC01E4
:1080D00085E393E122E030E00E9435BDF394CF2D9B
:1080E000D0E0C8010E946386C817D9075CF385E316
:1080F00093E16DE571E00E9449BD85E393E16EE592
:1081000071E10E943CBBFF240DC0C801BE010E946A
:10811000FE86AB01BC0185E393E122E030E00E94E2
:1081200035BDF394CF2DD0E0C8010E946386C817F7
:10813000D9075CF385E393E16DE571E00E9449BDE9
:1081400085E393E16DE571E00E9449BDE394CE2D96
:10815000D0E00E945486C817D9070CF466CFDF918F
:10816000CF911F910F91FF90EF90DF90CF900895E6
:108170008F929F92AF92BF92CF92DF92EF92FF9237
:108180000F931F93CF93DF93843609F4F9C185369B
:1081900070F5803109F458C1813198F48C3009F4BC
:1081A000A9C08D3038F48A3009F452C08B3009F000
:1081B000F0C36CC08E3009F4F9C08F3008F028C1CC
:1081C000C7C0853109F4B5C1863138F4813109F46D
:1081D00094C1843109F0DDC3A4C1873109F4BDC164
:1081E000873108F4B0C1833609F0D3C3C3C18B36DD
:1081F00009F4E5C28C3698F4873609F436C288361D
:1082000038F4853609F4DCC1863609F0C2C3EEC104
:10821000893609F490C28A3608F0ACC259C28B374D
:1082200009F411C38C3750F4893709F4EEC28A3748
:1082300008F0FBC2883709F0ACC3D1C2833809F417
:1082400040C3843809F466C3823809F0A2C315C359
:108250008EE196E00E9477A67C01B701882777FD22
:108260008095982F0E944BC68B019C0185E06AE0A7
:1082700070E04AEC53E00E94C52224E0E216F104CB
:1082800008F0B1C1C7010E944A86ADC18EE196E0F7
:108290000E9477A6EC0197FD2AC00E944F862AE132
:1082A00030E0829F8001839F100D929F100D11245A
:1082B0000E511B4FC8010E948486C8010E94BF86D0
:1082C000C8010E94FA86C801BE010E94CD88BE0185
:1082D000882777FD8095982F0E944BC68B019C01C3
:1082E00085E06BE070E040EB53E00E94C52281E046
:1082F000BE01C0C28EE196E00E94D3A66B017C0154
:108300000E944F862AE130E0829F8001839F100DFA
:10831000929F100D11240E511B4FC8010E948086A0
:108320005C01C801B701A6010E946786C801B501BA
:108330000E9488866B017C01C801B5010E94888675
:108340008B019C0185E06CE070E04DE953E05BC07F
:108350008EE196E00E94D3A66B017C010E944F86BD
:108360002AE130E0829F8001839F100D929F100DC3
:1083700011240E511B4FC8010E94BB865C01C8012D
:10838000B701A6010E949A86C801B5010E94C38662
:108390006B017C01C801B5010E94C3868B019C0161
:1083A00085E06DE070E04AE853E02DC08EE196E094
:1083B0000E94D3A66B017C010E944F862AE130E027
:1083C000829F8001839F100D929F100D11240E51EA
:1083D0001B4FC8010E94F6865C01C801B701A601C7
:1083E0000E94D586C801B5010E94FE866B017C0102
:1083F000C801B5010E94FE868B019C0185E06EE0FC
:1084000070E047E753E00E94C522C701B60124C1CE
:108410008EE196E00E947FA60E9459860E945E86A9
:108420007C01BC0180E090E00E9449C68B019C0168
:1084300085E06FE070E041E653E00E94C52281E0F4
:10844000B7010E946A1CA5C20E944F867C018AE186
:1084500090E0E89EE001E99ED00DF89ED00D112439
:10846000CE51DB4FCE010E94638602971CF1CE01F4
:1084700060E070E00E94C38627EF31E0E29E800159
:10848000E39E100DF29E100D11240A56194F0E9402
:1084900018C6AB01BC01C8010E94F58BCE010E9439
:1084A0006386BC0161507040CE010E94C3860E9469
:1084B00018C616C087EF91E0E89E8001E99E100D76
:1084C000F89E100D11240A56194FC8010E941D8CE8
:1084D000AB01BC01C8010E94F58BC8010E941D8C34
:1084E000AB01BC01C8010E94058C85E060E170E031
:1084F0004AE453E00E94782439C08EE196E00E945D
:10850000A3A60E942F860E9438866B017C010E94E0
:108510004BC68B019C0185E061E170E04BE253E0CA
:10852000F3C10E948B3F85E064E170E04FE053E0CF
:10853000E1CF85E065E170E04CEF52E00E947824E5
:108540000E945A3313C085E066E170E048EE52E0C5
:108550000E9478240E94563309C085E067E170E0EC
:1085600045ED52E00E9478240E94043181E00E948F
:108570009E1C0FC281E00E949E1C0E948F3F09C278
:108580000E944F862AE130E0AC01429FC001439F28
:10859000900D529F900D11248E519B4F0E94638627
:1085A0007C01B701882777FD8095982F0E944BC6E4
:1085B0008B019C0185E064E670E043EC52E011C061
:1085C0000E945E867C01B701882777FD8095982FF1
:1085D0000E944BC68B019C0185E065E670E046EA8F
:1085E00052E00E94C52281E0B70144C18EE196E0CD
:1085F0000E94D3A67B018C010E944F866AE1C62EA1
:10860000D12C9C012C9DC0012D9D900D3C9D900D69
:1086100011248E519B4FB801A7010E94A3884B01E2
:108620005C010E944F86AC014C9DC0014D9D900D98
:108630005C9D900D11248E519B4FB801A7010E94A3
:10864000A3888B019C0185E066E670E041E952E079
:108650000E94C522C501B40120E030E048EC52E49C
:108660000E94FFC60E9418C68FC18EE196E00E944C
:10867000D3A66B017C010E944F865AE1A52EB12C36
:108680009C012A9DC0012B9D900D3A9D900D1124B7
:108690008E519B4FB701A6010E9494888B019C01CB
:1086A00085E067E670E041E852E00E94C5220E9442
:1086B0004F86AC014A9DC0014B9D900D5A9D900D77
:1086C00011248E519B4FB701A6010E949488C4CFFC
:1086D0008EE196E00E94D3A66B017C010E944F863A
:1086E0004AE1A42EB12C9C012A9DC0012B9D900D26
:1086F0003A9D900D11248E519B4FB701A6010E9407
:1087000085888B019C0185E068E670E04FE652E0C9
:108710000E94C5220E944F86AC014A9DC0014B9D1C
:10872000900D5A9D900D11248E519B4FB701A601BB
:108730000E94858891CF0E944F862AE130E0AC01EB
:10874000429FC001439F900D529F900D11248E5166
:108750009B4F0E940E88F82E682F70E080E090E01A
:108760000E9449C68B019C0185E069E670E043E602
:1087700052E01EC00E944F862AE130E0AC01429FC9
:10878000C001439F900D529F900D11248E519B4F1D
:108790000E949787F82E682F70E080E090E00E949A
:1087A00049C68B019C0185E06AE670E045E552E030
:1087B0000E94C52281E06F2D0E94841CEAC00E94A5
:1087C00038860E944BC68B019C0185E06BE670E009
:1087D00040E452E00E94C5220E943886D5C00E9423
:1087E0001215AA2797FDA095BA2FBC01CD010E94B2
:1087F0004BC68B019C0185E068E770E044E352E0E2
:108800000E94C5220E94121533C00E9426150E94A4
:108810004BC68B019C0185E069E770E04EE152E0B8
:108820000E94C5220E942615AFC00E941F3A6B010C
:108830007C010E944BC68B019C0185E06AE770E0D9
:1088400047EF51E061C00E94D639AA2797FDA09555
:10885000BA2FBC01CD010E944BC68B019C0185E063
:108860006BE770E044EE51E00E94C5220E94D639C9
:10887000BC0181E00E94501C8CC08EE196E00E94F9
:1088800077A68C010E944F862AE130E0AC01429F1E
:10889000C001439F900D529F900D11248E519B4F0C
:1088A000B8010E9488860E9418C66B017C010E9454
:1088B0004BC68B019C0185E062E870E04DEC51E015
:1088C00023C08EE196E00E9477A68C010E944F861D
:1088D0002AE130E0AC01429FC001439F900D529FBE
:1088E000900D11248E519B4FB8010E94C3860E94A7
:1088F00018C66B017C010E944BC68B019C0185E070
:1089000063E870E047EB51E00E94C52281E0B701C7
:10891000A6013DC08EE196E00E9477A65C010E9410
:108920004F860AE110E09C01209FC001219F900D1D
:10893000309F900D11248E519B4FB5010E94FE86F1
:108940006B017C010E944F86AC01409FC001419F9A
:10895000900D509F900D11248E519B4FB5010E9498
:10896000FE868B019C0185E064E870E041EA51E0FD
:108970000E94C522C701B6010E9418C624E630E055
:1089800040E050E00E94C7C7AB01BC0181E00E94FB
:108990001A1CDF91CF911F910F91FF90EF90DF9004
:1089A000CF90BF90AF909F908F9008952F923F925D
:1089B0004F925F926F927F928F929F92AF92BF92EF
:1089C000CF92DF92EF92FF920F931F93DF93CF939B
:1089D000CDB7DEB762970FB6F894DEBF0FBECDBF3E
:1089E00087E090E00E94E4AB80E090E064EB73E00D
:1089F0000E94121982E090E069EA73E04AE00E9466
:108A0000B9AB19821A821B821C821D821E821F82B0
:108A1000188619861A861B861C861D861E861F864A
:108A2000188A198A1A8A19EAA12E14E0B12ECC24C8
:108A3000DD24B2E2EB2EF12CA3E02A2E312C2C0EF9
:108A40003D1EF7E04F2E512C4C0E5D1EEBE06E2EBE
:108A5000712C6C0E7D1E7FE0872E912C8C0E9D1E3E
:108A600087EF91E0C89E8001C99E100DD89E100D21
:108A700011240A56194FC8010E94C5898983C8016B
:108A80000E94F6891A82882311F091E09A83C80126
:108A90000E941D8C6B837C838D839E83C8010E9402
:108AA000FD8B6F83788789879A87C8010E940D8C18
:108AB0006B877C878D879E87F50181919191A1912C
:108AC000B1915F018F87988BA98BBA8B81E191E17E
:108AD0006C2D49810E948716C701BE016F5F7F4FD1
:108AE0000E940E19C7010196BE016E5F7F4F0E9462
:108AF0002119C7014097B1010E942519C7010897A4
:108B0000B2010E942519C7010497B3010E942519DB
:108B1000C7010C97B4010E9425190894C11CD11CEF
:108B200088E190E0E80EF91E93E0C916D10409F03F
:108B300097CF0AE510E0B80165517F4EC8010E9449
:108B4000ED180F5F1F4F09361105A9F70E94121F7C
:108B50000E94601962960FB6F894DEBF0FBECDBFBB
:108B6000CF91DF911F910F91FF90EF90DF90CF9009
:108B7000BF90AF909F908F907F906F905F904F903D
:108B80003F902F9008950E94A4AB882339F00E9453
:108B90008AAB079719F40E94302A08950E94D644A0
:108BA00008954F925F926F927F929F92AF92BF9281
:108BB000CF92DF92EF92FF920F931F93DF93CF93A9
:108BC00000D00F92CDB7DEB700E010E037EFE32E14
:108BD00031E0F32E0E9DC0010F9D900D1E9D900D56
:108BE00011248A56994F0E944F8A882309F0B2C0F7
:108BF0008091C104882309F0ADC0C2C0EE24FF24D7
:108C000027EFA22E21E0B22E6E010894C11CD11CC8
:108C100099249394EA9C8001EB9C100DFA9C100D12
:108C200011240A56194FC8010E94F689F601EE0D6B
:108C3000FF1D108281119082C80161E00E94CE96D2
:108C40000894E11CF11C83E0E816F10419F799245B
:108C5000EE24FF2497EF492E91E0592E81E0682EF3
:108C6000712CE49C8001E59C100DF49C100D1124E6
:108C70000A56194FC80160E00E94CE9664E670E083
:108C800080E090E00E9426B689E20E94CFB6AA2733
:108C900097FDA095BA2FBC01CD010E944BC620E0E4
:108CA00030EC4FE754E40E94B0C520E030E040EAE9
:108CB00050E40E94FFC65B016C010E94581F9B019B
:108CC000AC0166E676E686EE9FE30E94B0C59B01A6
:108CD000AC01C601B5010E94FBC6181644F4C301DD
:108CE0000E2C02C0880F991F0A94E2F7982AC80137
:108CF00061E00E94CE9684EA9CE064E871E00E9404
:108D0000642084EA9CE0B7010E94E23C84EA9CE093
:108D10006BE871E00E94642084EA9CE0B601A50142
:108D20000E94D21C0894E11CF11C83E0E816F104B7
:108D300009F097CF86E996E069810E94CE968DE88A
:108D400098E06A810E94CE9684E89AE06B810E9446
:108D5000CE9602C008E0902E892D0F900F900F90B4
:108D6000CF91DF911F910F91FF90EF90DF90CF9007
:108D7000BF90AF909F907F906F905F904F900895BD
:108D80000F5F1F4F0330110509F024CF37CFCF926B
:108D9000DF92EF92FF920F931F93CF93DF9381E8BF
:108DA00096E00E94A8A568EE73E080E090E00E9443
:108DB00026B681E896E00E94A8A568EE73E080E000
:108DC00090E00E9426B6C0E0D0E067EFE62E61E0BA
:108DD000F62ECE9D8001CF9D100DDE9D100D11242D
:108DE0000A56194FC80161E00E94EC89C80161E090
:108DF0000E94CE962196C330D10559F70E94D145E5
:108E0000182F6AEF70E080E090E00E9426B6C0E084
:108E1000D0E0E12EFF2457EFC52E51E0D52EC7013B
:108E20000C2E02C0959587950A94E2F780FF1CC02E
:108E3000CC9D8001CD9D100DDC9D100D11240A5696
:108E4000194FC80160E00E94CE966AEF70E080E0A2
:108E500090E00E9426B6C80161E00E94CE966AEFBB
:108E600070E080E090E004C068EE73E080E090E0A5
:108E70000E9426B62196C330D10589F686E996E090
:108E800060E00E94CE968DE898E060E00E94CE9669
:108E900084E89AE060E00E94CE960E94F2B5C0E0BD
:108EA000D0E047EFE42E41E0F42ECE9D8001CF9D2F
:108EB000100DDE9D100D11240A56194FC80140E017
:108EC00050E06AE775E40E94BF8AC80160E00E9432
:108ED0000F8AC80160E020EE3EE240E050E00E94D0
:108EE0007D9F2196C330D10501F70E94BC2B86E9F6
:108EF00096E00E944F8A8823D1F78DE898E00E947F
:108F00004F8A8823A1F784E89AE00E944F8A882339
:108F100071F786E996E061E020EE3EE240E050E045
:108F20000E947D9F8DE898E061E020EE3EE240E007
:108F300050E00E947D9F84E89AE061E020EE3EE2EE
:108F400040E050E00E947D9F0E94BC2BDF91CF91BA
:108F50001F910F91FF90EF90DF90CF9008954F9267
:108F60005F926F927F928F929F92AF92BF92CF92B9
:108F7000DF92EF92FF920F931F93DF93CF9300D076
:108F80000F92CDB7DEB7882EEE24FF24F7EFAF2E79
:108F9000F1E0BF2E6E010894C11CD11C992493945A
:108FA000EA9C8001EB9C100DFA9C100D11240A56CE
:108FB000194FC8010E94F689F601EE0DFF1D1082BF
:108FC00081119082C80161E00E94CE960894E11C54
:108FD000F11C83E0E816F10419F783E0889E300164
:108FE00011249924E7EF4E2EE1E05E2E28C0E49C88
:108FF0008001E59C100DF49C100D11240A56194FA8
:10900000C80160E00E94CE966BE470E080E090E0E2
:109010000E9426B6C80161E00E94CE96EA0CFB1CB5
:1090200083E0E816F10421F4B094A194B108B3945C
:109030000894C11CD11CC614D704CCF29394981484
:1090400040F471E0A72EB12CCC24DD24EE24FF24C3
:10905000F2CF86E996E069810E94CE968DE898E08D
:109060006A810E94CE9684E89AE06B810E94CE9637
:109070000F900F900F90CF91DF911F910F91FF9064
:10908000EF90DF90CF90BF90AF909F908F907F90A8
:109090006F905F904F900895FF920F931F93CF931F
:1090A000DF93F82E8B01C0E0D0E015C08F2D61E07A
:1090B0000E9481B764E670E080E090E00E9426B6EE
:1090C0008F2D60E00E9481B764E670E080E090E060
:1090D0000E9426B62196C017D10744F3DF91CF91A5
:1090E0001F910F91FF900895FF920F931F93082FE8
:1090F00084EA9CE00E94A910482F90E0202F30E0E5
:1091000082239323892B21F0F02EF094F42202C0C5
:10911000F42EF02A84EA9CE06F2D0E94B4100F2DEB
:1091200010E0C801B4E096958795BA95E1F7817093
:109130000E94F7A41695079516950795802F8170C4
:109140000E9465968F2D1F910F91FF900895CF92E9
:10915000DF92EF92FF920F931F93CF93DF9380E8FC
:1091600096E00E944389EE24FF2400E010E087EFA0
:10917000C82E81E0D82E0C9DE0010D9DD00D1C9DC8
:10918000D00D1124CA56D94FCE010E94F1898823EF
:10919000B9F0E114F10469F0CE010E945C8C9701F2
:1091A000442737FD4095542F6217730784079507AE
:1091B00018F00115110521F4CE010E945C8C7B0191
:1091C0000F5F1F4F03301105B1F61E141F043CF54D
:1091D0008091A3049091A404E816F90620F00E945F
:1091E0002A8C8230B1F40E942A8C8230C1F497011B
:1091F000442737FD4095542F8091B5049091B604D3
:10920000A091B704B091B804281739074A075B0743
:1092100030F08BE79CE061E00E9487A402C00E94CE
:109220000831DF91CF911F910F91FF90EF90DF9068
:10923000CF900895EF92FF920F931F93CF93DF93F8
:10924000EC017A018B01888184FF14C08981882315
:1092500031F085E393E12AE030E00E94C8BB8A81C7
:10926000882341F08B819C81B801A7012AE030E07E
:109270000E94C8BBDF91CF911F910F91FF90EF909B
:1092800008950F931F930BE71CE0C80161E041E5CF
:1092900058E70E949EA4C80162E047EA58E40E9491
:1092A0009EA4C80163E045E158E70E949EA4C8015E
:1092B00064E042EB5BE20E949EA4C80165E04CE6DC
:1092C00059E40E949EA4C80166E04AE458E30E9463
:1092D0009EA41F910F9108958BE79CE060E00E948F
:1092E00087A481E896E00E9425A508952F923F92D9
:1092F0004F925F926F927F928F929F92AF92BF92A6
:10930000CF92DF92EF92FF920F931F93DF93CF9351
:10931000CDB7DEB7A2970FB6F894DEBF0FBECDBFB4
:109320001C01498F5A8F6B8F7C8F8FEF90E0289EA6
:109330009001299E300D389E300D11242753324F55
:109340003A832983F90180E090E020E030E040E0BA
:1093500050E0F8972083318342835383F89620832B
:10936000318342835383248F358F468F578F0196E5
:1093700034968730910569F78FEF90E0289EB00111
:10938000299E700D389E700D11246157724F6C51DB
:109390007F4FDB012D933D934D935C9313976B5F50
:1093A0007F4FDB012D913D914D915C912D8B3E8B3B
:1093B0004F8B588F695E7040FB01268F378F40A31B
:1093C00051A36F507F4FDB01ED90FD900D911D91EA
:1093D0008D919D910D90BC91A02D898B9A8BAB8B1B
:1093E000BC8BC801B70129893A894B895C890E94E5
:1093F000B0C56D877E878F87988BC801B7012D8593
:109400003E854F8558890E94FFC669877A878B877A
:109410009C87698D7A8D8B8D9C8D2D893E894F8996
:10942000588D621B730B840B950B97FF07C09095AB
:109430008095709561957F4F8F4F9F4F0E944BC6CF
:109440006D837E838F839887898D9A8DAB8DBC8D3C
:109450002D893E894F89588D281739074A075B07A0
:109460002CF04FEF5FEF5C834B8304C081E090E012
:109470009C838B838FEF90E0289E8001299E100DA6
:10948000389E100D11240157124F05501F4FD8015F
:109490008D909D90AD90BC900B5F1040C501B401C4
:1094A00020E030E040EA50E40E94FBC618160CF0C1
:1094B00027C1F801E851FF4F8081882329F460E03B
:1094C00070E080EA91EC04C060E070E080EA91E432
:1094D000A50194010E94FFC62FE632E143E852E461
:1094E0000E94B0C56B017C0129893A894B895C894E
:1094F0000E94B0C52B013C01E89477F869897A890C
:109500008B899C8920E030E040E05FE30E94FFC649
:10951000A30192010E94FFC6A30192010E94FFC60F
:109520006D8F7E8F8F8F98A3EB81FC81BF01882781
:1095300077FD8095982F0E944BC64B015C01C701B7
:10954000B601A50194010E94FFC620E030E040E092
:1095500050E00E94ACC58823BCF58FEF90E0289EB8
:109560008001299E100D389E100D11240157124FB5
:10957000D80112964D925D926D927C9215970B5088
:109580001F4FC501B401F80120813181428153810F
:109590000E94FFC60F591040D8016D937D938D93A3
:1095A0009C93139706551040F801C2AED3AEE4AEBB
:1095B000F5AE6D817E818F8198852D8D3E8D4F8D8D
:1095C00058A10E9448C550C06D817E818F819885C9
:1095D0002D8D3E8D4F8D58A10E94ACC588230CF077
:1095E0004BC08FEF90E0289E8001299E100D389E81
:1095F000100D11240157124FD80112964D925D9211
:109600006D927C921597EB81FC81F095E195FF4F6F
:10961000FC83EB83BF01882777FD8095982F0E94FC
:109620004BC60B501F4FD8012D913D914D915C9130
:109630000E94FFC60F591040F80160837183828336
:10964000938306551040D801DA96CD92DD92ED92C3
:10965000FC92DD976D8D7E8D8F8D98A12D813E8141
:109660004F8158850E9447C56D837E838F8398877D
:10967000B1E06B2E712C46C06D817E818F81988503
:109680002D8D3E8D4F8D58A10E9448C56D837E83E0
:109690008F8398878FEF90E0289E6001299ED00CE1
:1096A000389ED00C1124EFE8FDE0CE0EDF1E6D8950
:1096B0007E898F89988D0E944BC67B018C01C501E4
:1096C000B4012D8D3E8D4F8D58A10E94FFC69B0188
:1096D000AC01C801B7010E9447C50E9418C6D60157
:1096E0005E966D937D938D939C939197E4EEF0E05D
:1096F000CE0EDF1ED6014D925D926D927C92139735
:10970000662477246D817E818F81988529853A85AD
:109710004B855C850E94ACC518163CF4BD85B9A389
:10972000EE85EAA34F8458881AC08FEF90E0289EF8
:10973000F001299EF00D389EF00D1124EC57F14FE9
:109740006D817E818F819885208131814281538115
:109750000E94B0C50E9466C769A37AA32C01F301D9
:10976000EE0FFF1FEE0FFF1F8FEF90E0289E70019E
:10977000299EF00C389EF00C1124EE0DFF1DEF56C3
:10978000F24F29A13AA1C901D20180839183A2831A
:10979000B3832B813C81B901882777FD8095982F71
:1097A0000E944BC64B015C018301000F111F000F8B
:1097B000111F0E0D1F1D0B51124FEFE8CE2EEDE0C5
:1097C000DE2ECE0CDF1CF601EB50FF4F20813181E5
:1097D000428153810E94FFC6D8016D937D938D9382
:1097E0009C9313976D817E818F81988529853A8519
:1097F0004B855C850E94FBC61816ACF50894611C6D
:10980000711C8301000F111F000F111F0E0D1F1D72
:109810000F56124F6D817E818F81988529853A85FB
:109820004B855C850E9447C5F601EF50FF4F2081B4
:109830003181428153810E94B0C5F80160837183F8
:1098400082839383F301EE0FFF1FEE0FFF1FEE0DD8
:10985000FF1DEB51F24F80E090E0A0E0B0E080838C
:109860009183A283B3830894611C711CF301EE0FF2
:10987000FF1FEE0FFF1F8FEF90E0289E7001299EC3
:10988000F00C389EF00C1124EE0DFF1DEF56F24F38
:1098900029A13AA1C901D20180839183A283B38314
:1098A0008301000F111F000F111F0E0D1F1D0B5103
:1098B000124FF701EC57F14F2081318142815381E2
:1098C0005058C501B4010E94FFC6D8016D937D9325
:1098D0008D939C93139731E9432E3DE0532E4E0C0C
:1098E0005F1C21E0822E912CF201A080B180C28009
:1098F000D380648D758D868D978D0E944BC67B01BC
:109900008C01C601B501A981BA812D913D914D917E
:109910005C910E94FFC69B01AC01C801B7010E9487
:1099200048C57B018C01E981FA81648D758D868D36
:10993000978D20E030E040E05FE30E94FFC6A60183
:1099400095010E94FFC6A60195010E94FFC69B01DA
:10995000AC01C801B7010E9448C50E9418C6D201D7
:1099600090966D937D938D939C939397C601B501CB
:10997000E981FA81248D358D468D578D0E94FFC671
:109980009B01AC01A981BA816D917D918D919C91D2
:109990000E9448C5E981FA81648375838683978331
:1099A0000894811C911C24E030E0420E531E349632
:1099B000FA83E983681479040CF096CFF3013196A9
:1099C000EE0FFF1FEE0FFF1F8FEF90E0AC01249E04
:1099D000C001259E900D349E900D1124E80FF91FB3
:1099E000E157F24F298D3A8D4B8D5C8D268F378F45
:1099F00040A351A38C010B51124FEE24FF24D80138
:109A00006D917D918D919C9120E030E040E05FE38D
:109A10000E94FFC6F80161937193819391938F0126
:109A20000894E11CF11C6E147F044CF78FEF90E05A
:109A3000289EF001299EF00D389EF00D1124EF585C
:109A4000F14F11821082A2960FB6F894DEBF0FBEBE
:109A5000CDBFCF91DF911F910F91FF90EF90DF90DD
:109A6000CF90BF90AF909F908F907F906F905F90BE
:109A70004F903F902F900895CF93DF93EC018FEF9D
:109A800090E0C89FF001C99FF00DD89FF00D112400
:109A9000E157F24FE351FF4F408351836283738359
:109AA000B291A29192918291481759076A077B0758
:109AB000C1F0CE010E94764981E090E0A0E0B0E0E4
:109AC0000C2E04C0880F991FAA1FBB1F0A94D2F73F
:109AD00020918A0D282B20938A0DCE0161E00E94EF
:109AE0000D34DF91CF9108952F923F924F925F9264
:109AF0006F927F928F929F92AF92BF92CF92DF929E
:109B0000EF92FF920F931F93DF93CF93CDB7DEB702
:109B100060970FB6F894DEBF0FBECDBF9A878987D6
:109B20007C876B8728013901CD86DE86EF86F88A2F
:109B3000662757FD6095762FCB01BA010E944BC670
:109B400020E030E04AE754E40E94B0C57B018C017C
:109B50006D857E858F8598890E944BC66D837E8337
:109B60008F8398872D853E854F855889421A530AE1
:109B7000640A750AC301B2010E944BC69B01AC0185
:109B8000C801B7010E94FFC69B01AC016D817E81B7
:109B90008F8198850E9448C50E9418C61B012C0120
:109BA0008D859E85AF85B889881A990AAA0ABB0A4D
:109BB000C501B4010E944BC69B01AC01C801B701AD
:109BC0000E94FFC69B01AC016D817E818F819885CB
:109BD0000E9448C50E9418C669837A838B839C8340
:109BE0008FEF90E0A985BA85A89FF001A99FF00D9D
:109BF000B89FF00D1124E75CF14F20E030E080E0E9
:109C000090E0A0E0B0E0F89780839183A283B383D3
:109C1000F89680839183A283B383848F958FA68FD8
:109C2000B78F2F5F3F4F34962730310561F78FEFA5
:109C300090E0E985FA85E89F8001E99F100DF89F83
:109C4000100D11240157124F0E561F4FD8012D929F
:109C50003D924D925C921397EB85FC85BF0188275E
:109C600077FD8095982F0E944BC620E030E04AE7B0
:109C700054E40E94B0C520E030E040E05FE30E9481
:109C8000FFC66B017C010C511040D8016D937D9390
:109C90008D939C931397065710408EEA682E712C73
:109CA000600E711E6D857E858F8598896219730996
:109CB000840995090E944BC6A70196010E94B0C570
:109CC000F30160837183828393830A561F4F2D852E
:109CD0003E854F855889D8012D933D934D935C93D4
:109CE00013970C511040F801C082D182E282F382B6
:109CF000085C1F4F69817A818B819C81621B730B89
:109D0000840B950B0E944BC6A70196010E94B0C51B
:109D10004B015C01D8016D937D938D939C931397B8
:109D2000F301608171818281938120E030E040E025
:109D30005FE30E94FFC66B017C01C201B1010E947A
:109D40004BC6A70196010E9447C50E9418C62B0169
:109D50003C0104521040D8016D937D938D939C93E8
:109D600013970C51104080E090E0A0E8BFE3F801A9
:109D700080839183A283B3830C5A1F4FF801C08262
:109D8000D182E282F3820C52104029813A814B81C8
:109D90005C81F80120833183428353830C5110404E
:109DA000F80180839183A283B383085C1F4FD8019D
:109DB0008D929D92AD92BC921397045E1F4FC50188
:109DC000B40120E030E040E05FEB0E94FFC6F80104
:109DD00060837183828393830453104069817A8105
:109DE0008B819C810E944BC66B017C01C501B40133
:109DF00020E030E040E05FE30E94FFC69B01AC0141
:109E0000C701B6010E9448C50E9418C6D8016D93CB
:109E10007D938D939C93139789859A85B301A201B5
:109E20000E943C4D60960FB6F894DEBF0FBECDBFCA
:109E3000CF91DF911F910F91FF90EF90DF90CF9026
:109E4000BF90AF909F908F907F906F905F904F905A
:109E50003F902F9008950F931F93CF93DF93062F7A
:109E6000853009F4BBC0863080F4823009F449C0E3
:109E7000833020F4813009F01DC11AC0833009F409
:109E800062C0843009F016C18AC08A3009F4E1C08A
:109E90008B3038F4863009F4D2C0873009F00AC11B
:109EA000D3C08C3009F4EBC08D3009F003C1ECC095
:109EB00085E393E16BE971E00E9499BC85E393E14E
:109EC00061E070E04AE050E00E9472BC85E393E1FB
:109ED0006FE971E00E9499BC85E393E163E070E073
:109EE0004AE050E00E9472BC85E393E16FE971E0C3
:109EF0000E9499BC85E393E161EA71E00E9499BCFC
:109F0000D3C085E393E16AEA71E00E9499BC10E056
:109F1000B8016F5F7F4F85E393E14AE050E00E9414
:109F200072BC85E393E16FE971E00E9499BC8FEF09
:109F300090E0089FF001099FF00D189FF00D11248B
:109F4000E458F14F21C085E393E16EEA71E00E948D
:109F500099BC10E0B8016F5F7F4F85E393E14AE061
:109F600050E00E9472BC85E393E16FE971E00E94CA
:109F700099BC8FEF90E0089FF001099FF00D189FAA
:109F8000F00D1124E858F14F4081518162817381B5
:109F900085E393E12AE030E00E9422BC85C085E39E
:109FA00093E162EB71E00E9499BCC0E0D0E0809147
:109FB0008A0D90E00C2E02C0959587950A94E2F7E1
:109FC00080FD02C060E301C061E385E393E10E948C
:109FD0001EBB2196C330D10551F766C085E393E1DE
:109FE00066EB71E00E9499BC10E0B8016F5F7F4F93
:109FF00085E393E14AE050E00E9472BC85E393E17F
:10A000006FE971E00E9499BC8FEF90E0089FF0012A
:10A01000099FF00D189FF00D1124E058F14F608159
:10A020007181828193810E941DC69B01AC0185E3F1
:10A0300093E1B9014AE050E00E94EBBB35C085E3F3
:10A0400093E16AEB71E024C085E393E16EEB71E08C
:10A050002FC085E393E163EC71E00E9499BC6091AD
:10A060008D0D70918E0D85E393E14AE050E00E94E2
:10A0700072BC85E393E167EA71E00E9499BC85E3D5
:10A0800093E167EC71E004C085E393E16BEC71E070
:10A090000E9499BC602F70E06F5F7F4F85E393E172
:10A0A0004AE050E00E9472BC85E393E167EA71E008
:10A0B0000E9499BCDF91CF911F910F910895CF938A
:10A0C000DF93EC018FEF90E0C89FF001C99FF00D86
:10A0D000D89FF00D1124E858F14F80819181A28121
:10A0E000B38184179507A607B70729F0CE010E9410
:10A0F0003C4D82E001C083E06C2F0E942B4FDF912A
:10A10000CF9108956F927F928F929F92AF92BF925C
:10A11000CF92DF92EF92FF920F931F93CF93DF9333
:10A1200010928C0D1092CB0C1092CD0C1092CC0C86
:10A130001092860D1092850D8AE08093870D109203
:10A14000840D1092880D8CE061E00E94FEB6C0E0A4
:10A15000D0E08CE061E00E9481B762E370E080E0D3
:10A1600090E00E9426B68CE060E00E9481B762E336
:10A1700070E080E090E00E9426B62196CC30D105B8
:10A1800041F7E9EAFCE011928CE0E93CF807D9F7E5
:10A19000B097F093CA0CE093C90C81E065E171E1DE
:10A1A00041E050E00E947AB30FE81DE028E7E22E7C
:10A1B0002EE0F22E6801C0E0D0E09FEF692E712CF6
:10A1C0000F2EF0E08F2EF0E09F2EF0E0AF2EF0E0AB
:10A1D000BF2EF02DFE01E85BFB4F8081F6018083EE
:10A1E000FE01E55BFB4F8081F6018183FE01EB5BA5
:10A1F000FB4F808161E00E94FEB6CE0160E00E94CC
:10A200000D34C69DF001C79DF00DD69DF00D1124B3
:10A21000E958F14F81E08083F701108211821282A8
:10A2200013821482158216821782118A108A828AFA
:10A23000938AA48AB58ACE0168E873E10E94191155
:10A2400021968FEF90E0C80ED91EE80EF91EC3309C
:10A25000D10509F0BFCFF801808161E00E94FEB610
:10A26000F801818161E00E94FEB6F80180818A30A8
:10A2700029F4809180008A7F8093800001501F4FD5
:10A28000F0E10C381F0739F78091770E60E08111FB
:10A2900061E08091900D0E9481B78091760F60E01F
:10A2A000811161E080918F0E0E9481B780917510BD
:10A2B00060E0811161E080918E0F0E9481B781E0A2
:10A2C00060E00E942B4F8FEA91E149E150E060E0AD
:10A2D00070E00E94807F8FEA91E16AED76E32FEFD4
:10A2E0003FEF4FEF5FEF0E94977FDF91CF911F917C
:10A2F0000F91FF90EF90DF90CF90BF90AF909F9025
:10A300008F907F906F9008952F923F924F925F921F
:10A310006F927F928F929F92AF92BF92CF92DF9275
:10A32000EF92FF920F931F93DF93CF93CDB7DEB7DA
:10A330002A970FB6F894DEBF0FBECDBF85E393E139
:10A340000E943DBE1E821D82282F30E03A87298759
:10A3500022242394A3C285E393E10E94F7BD0E94C7
:10A360008120882309F495C2F090D20CFA948B32A4
:10A3700009F4A8C08C32A8F48F3109F47EC0803271
:10A3800030F48A3019F18E3109F07DC2A7C08932CC
:10A3900009F4CBC08A3208F0A8C0883209F073C231
:10A3A00053C08C3309F4D7C08D3330F48C3281F034
:10A3B000823309F068C2AFC0863409F4FCC1873427
:10A3C00009F449C28D3309F05EC246C181E0ABC0D9
:10A3D0008091D10C813009F056C20F2D10E0C801D8
:10A3E0000E94EB12882309F44EC28FEF90E0089F81
:10A3F000F001099FF00D189FF00D1124E858F14F5E
:10A400001082118212821382C80140E050E060E0A5
:10A4100070E00E943C4DC80140E050E060E070E018
:10A420000E945F5081E090E0A0E0B0E00F2C04C0FB
:10A43000880F991FAA1FBB1F0A94D2F72091890D7C
:10A44000282B2093890D25C28091D10C823009F0F0
:10A450001AC28F2D90E00E94EB12882309F413C2D8
:10A460004091D60C5091D70C6091D80C7091D90CBA
:10A470008F2D90E00E945F500CC28091D10C8230F1
:10A4800009F001C20F2D10E0C8010E94EB128823D1
:10A4900009F4F9C1AFEFB0E00A9FF0010B9FF00D96
:10A4A0001A9FF00D1124E858F14F8091D60C90912D
:10A4B000D70CA091D80CB091D90C80839183A28342
:10A4C000B38327C08091D10C813009F0DCC18F2D7E
:10A4D00090E00E94EB128823E1F4D5C18091D10C69
:10A4E000882309F0D0C184E01EC08091D10C813056
:10A4F00009F0C9C18F2D90E00E94EB12882309F466
:10A50000C2C18F2D90E00E94511186E06F2D0E94F4
:10A510002B4F83E09CC18091D10C882309F0B3C1FB
:10A520000E94DE1287E060E093C18091D10C8230FE
:10A5300009F0A9C18F2D90E00E94EB12882309F445
:10A54000A2C16091D60C7091D70C8F2D90E00E9423
:10A55000191185E07CC180918A0D882309F093C18F
:10A560008091D10C853008F48EC1282F30E0225024
:10A570003040C90183709070892B09F084C1E4EFE9
:10A58000F1E0F0938E0DE0938D0DC90164E070E071
:10A590000E94FAC72B0180E090E0A0E0B0E0809339
:10A5A000010E9093020EA093030EB093040E8093BD
:10A5B000000F9093010FA093020FB093030F8093AD
:10A5C000FF0F90930010A0930110B09302103AED8A
:10A5D000632E3CE0732E18861F822EC0D3013C9060
:10A5E0003A94832D90E00E94EB12882311F411E03D
:10A5F00029C06091D20C7091D30C4091D60C50912F
:10A60000D70CF3010481158126813781C084D18460
:10A61000E284F38484849584A684B784832D90E0B7
:10A620000E94744D2F8138852F5F3F4F38872F83CD
:10A6300080E190E0680E791EAF81B885A415B5055C
:10A640006CF210E020928C0D8AE060E00E942B4FAB
:10A65000112309F41EC117C180918A0D882309F0C6
:10A6600012C18091D10C882309F00DC180918C0D0D
:10A67000882309F408C101E71EE0CC24DD24F80199
:10A68000E057F040608171818281938120E030E069
:10A6900040E050E00E94ACC5882309F477C0EFEF9A
:10A6A000F0E0CE9EC001CF9E900DDE9E900D112455
:10A6B000BC016F5F714FAC014F56524F9C01275C3C
:10A6C000314FFC01E753F24FEE24FF24DB018D9064
:10A6D0009D90AD90BC90DA018D929D92AD92BC920E
:10A6E0001397DB015C968D909D90AD90BC905F9729
:10A6F000DA015C968D929D92AD92BC925F97D901E2
:10A700008D909D90AD90BC90139780829182A28293
:10A71000B3825C968D909D90AD90BC905F97848E37
:10A72000958EA68EB78E0894E11CF11C6C5F7F4F4E
:10A730004C5F5F4F2C5F3F4F3496B7E0EB16F10450
:10A7400029F604541040F80180819181A281B381DF
:10A750000C5B1F4FF80183879487A587B68711820A
:10A76000108281E090E0A0E0B0E00C2C04C0880FE3
:10A77000991FAA1FBB1F0A94D2F720918A0D282B7C
:10A7800020938A0DC60161E00E940D340894C11C1B
:10A79000D11C01501F4FF3E0CF16D10409F06FCF49
:10A7A0000E940635F89427EE33E03093860D20930F
:10A7B000850D78946EC08091D10C823009F063C011
:10A7C0000F2D10E0C8010E94EB12882309F45BC032
:10A7D00019821A821B821C824091D60C5091D70C90
:10A7E0006091D80C7091D90CC8019E012F5F3F4F2A
:10A7F0000E94F112882351F180918A0D90E00F2C74
:10A8000002C0959587950A94E2F780FF18C08FEFF4
:10A8100090E0089FF001099FF00D189FF00D1124A2
:10A82000E458F14F29813A814B815C81808191818B
:10A83000A281B381281739074A075B0739F049819C
:10A840005A816B817C81C8010E943C4D8CE06F2D48
:10A850000E942B4F1EC08091D10C8230A1F48F2D0D
:10A8600090E00E94EB12882371F04091D60C509139
:10A87000D70C6091D80C7091D90C8F2D90E00E946C
:10A8800019348DE0E4CF85E393E16FEC71E00E9431
:10A8900099BCAD81BE811196BE83AD83ED81FE81F1
:10A8A00029853A85E217F3070CF455CD2A960FB6A1
:10A8B000F894DEBF0FBECDBFCF91DF911F910F91F6
:10A8C000FF90EF90DF90CF90BF90AF909F908F90D0
:10A8D0007F906F905F904F903F902F900895AF9230
:10A8E000BF92CF92DF92EF92FF920F931F93DF936D
:10A8F000CF930F92CDB7DEB700E010E063E2E62E13
:10A90000F12C5E010894A11CB11C57EFC52E51E03B
:10A91000D52E1982C701B5010E94DD180C9DC0011A
:10A920000D9D900D1C9D900D11248A56994F6981A3
:10A930000E94CE960F5F1F4F88E190E0E80EF91E4F
:10A940000330110531F744E1F42E8091840D882302
:10A9500011F40E9406350E9484518091870D88234E
:10A96000A1F7F092870D00E010E0602F80918A0D32
:10A9700090E0002E02C0959587950A94E2F780FD3D
:10A980000BC08091890D90E0002E02C095958795AF
:10A990000A94E2F780FF03C083E00E942B4F0F5F11
:10A9A0001F4F0330110509F71092890DCECF0F9379
:10A9B0001F9305E313E1C8010E9444BE64E670E002
:10A9C00080E090E00E9426B6C80140E05BE460E0D1
:10A9D00070E00E9447BE64E670E080E090E00E9474
:10A9E00026B61F910F910895EF92FF920F931F9338
:10A9F000CF93DF930E94F2B56093BD047093BE04C1
:10AA00008093BF049093C00481E08093C10400E070
:10AA100010E0E7EFEE2EE1E0FE2E0E9DE0010F9D2F
:10AA2000D00D1E9DD00D1124CA56D94FCE010E94C3
:10AA3000F189882321F0CE0160E00E94778C0F5FBE
:10AA40001F4F0330110549F78091C204813031F462
:10AA50008CE060E00E9481B71092C20480E896E02A
:10AA60000E940C89882329F08BE79CE061E00E941A
:10AA700087A4DF91CF911F910F91FF90EF900895E0
:10AA80006F927F928F929F92AF92BF92CF92DF92FE
:10AA9000EF92FF920F931F93DF93CF930F92CDB757
:10AAA000DEB7682E7A0170E0FB013297EB37F105D3
:10AAB00010F00C94775FE45BFF4FEE0FFF1F0590E3
:10AAC000F491E02D0994182F115060E0FA01808173
:10AAD000811161E0812F0E94022A812F0E94CF29DB
:10AAE00090E0A0E0B0E0BC01CD010E9449C68B011E
:10AAF0009C01862D62E070E040EE59E023C090E0BA
:10AB0000019727EF31E0829F8001839F100D929F74
:10AB1000100D11240A56194FC801FA0160810E94D4
:10AB2000EC89C8010E94F18990E0A0E0B0E0BC018E
:10AB3000CD010E9449C68B019C01862D63E070E027
:10AB40004FEC59E00E94C52281E00E949E1C0C94AB
:10AB5000775F64E070E040EC59E00E947824862D35
:10AB600090E0019727EF31E0AC01429FC001439F85
:10AB7000900D529F900D11248A56994F0E94A296D3
:10AB800010924C050E94E832DFCF8EE196E0BA01C8
:10AB90000E947FA67C01862D90E0019727EF31E08F
:10ABA000FC01E29FC001E39F900DF29F900D1124E4
:10ABB0008A56994FB7010E94E68900E010E0C8016B
:10ABC000B7010E9449C68B019C01862D65E070E0AB
:10ABD0004DEA59E0B7CFFA0160816983082F10E090
:10ABE0000150104087EF91E09C01029FC001039F3C
:10ABF000900D129F900D11240F5F1F4F8A56994F91
:10AC00000E94F99AC801880F991F800F911F23E0B5
:10AC1000880F991F2A95E1F70A96BE016F5F7F4F53
:10AC20000E940E19043011053CF4662D615081E13B
:10AC300091E149810E948716698170E080E090E08F
:10AC40000E9449C68B019C01862D66E070E048E9B0
:10AC500059E078CF8EE196E0BA010E947FA67C0190
:10AC6000862D90E0019727EF31E0AC01429FC001B3
:10AC7000439F900D529F900D11248A56994FB70112
:10AC80000E94A88A00E010E0C801B7010E9449C6EE
:10AC90008B019C01862D67E070E044E859E00E943A
:10ACA000C5220E94601950CFFA01F0806F2D70E02C
:10ACB00080E090E00E9449C68B019C01862D68E0EF
:10ACC00070E040E759E00E94C522862D90E0019790
:10ACD00027EF31E0AC01429FC001439F900D529F8E
:10ACE000900D11248A56994F6F2D0E94DC962CCF1F
:10ACF00069E070E04EE559E00E947824862D90E0EE
:10AD0000019727EF31E0FC01E29FC001E39F900D26
:10AD1000F29F900D11248A56994F0E949B8B14CF5D
:10AD2000E82EFF240894E108F10887EF91E0E89EFF
:10AD30006001E99ED00CF89ED00C112426E936E083
:10AD4000C20ED31EC6010E941D8C0E944BC68B01F1
:10AD50009C01862D6AE070E04BE459E00E94C52218
:10AD6000C6010E941D8CEE0CFF1CEE0CFF1C49EA74
:10AD700054E0E40EF51EF7016083718382839383B0
:10AD8000E3CE6BE070E04BE359E00E947824862D1F
:10AD900090E0019727EF31E0829F8001839F100DA3
:10ADA000929F100D11240A56194FC8010E94648AFF
:10ADB000A0E0B0E0BC01CD010E9449C6AB01BC01DE
:10ADC000C8010E94BF8AC80164E00E94F99AC801C4
:10ADD0000E94759F0E94BC2BC80161E00E9498965A
:10ADE000B3CE6CE070E04CE259E00E947824862DEE
:10ADF00090E0019727EF31E0829F8001839F100D43
:10AE0000929F100D11240A56194FC8010E94648A9E
:10AE1000A0E0B0E0BC01CD010E9449C6AB01BC017D
:10AE2000C8010E94BF8AC8010E94469FFCC08EE1F3
:10AE300096E0BA010E94D3A66B017C018091E104E7
:10AE4000882331F40E94FE10882311F40C944C5F87
:10AE5000C701B6010E9418C6882777FD8095982FF4
:10AE60000E944BC68B019C01862D6DE070E043E192
:10AE700059E00E94C522862D90E00197B701A601F6
:10AE80000E94902D23C0C8010E94648AA0E0B0E017
:10AE9000BC01CD010E9449C66B017C01C801B7010C
:10AEA000A6010E94BF8AC701B6010E9418C6882762
:10AEB00077FD8095982F0E944BC68B019C01862DB3
:10AEC0006DE070E04DEF58E00E94C5228091E104F2
:10AED000882311F00C94775F0E94FE10882311F0F4
:10AEE0000C94775F31CE8EE196E0BA010E94D3A632
:10AEF0006B017C01862D6EE070E046EE58E0970114
:10AF000086010E94C522862D90E0019727EF31E04F
:10AF1000AC01429FC001439F900D529F900D1124A0
:10AF20008A56994FB701A6010E94198A0E94121FE2
:10AF30000BCEFA01B0808091E1048823A1F1862D27
:10AF400090E0019727EF31E0829F8001839F100DF1
:10AF5000929F100D11240A56194FC8010E94FB89B7
:10AF600020E030E040E85FE30E94ACC58823DCF4D9
:10AF7000C8010E94FB8920E030E040E85FEB0E94BE
:10AF8000FBC6181684F4F1E0BF1631F4C80140E0A6
:10AF900050E060E271E405C0C80140E050E060E2CA
:10AFA00071EC0E94BF8A0894E11CF11C8EE196E0CE
:10AFB000B7010E9487A66B017C010E9449C68B01E4
:10AFC0009C01862D6FE070E044ED58E00E94C522A0
:10AFD000C114D104E104F10491F4862D90E00197AD
:10AFE00027EF31E0AC01429FC001439F900D529F7B
:10AFF000900D11248A56994F61E00E940F8A862D88
:10B0000090E0019727EF31E0FC01E29FC001E39F50
:10B01000900DF29F900D11248A56994F6B2DA70128
:10B0200096010E947D9F0E94BC2B8ECD8EE196E002
:10B03000BA010E94A3A67B018C01862D90E00197A6
:10B0400027EF31E0AC01429FC001439F900D529F1A
:10B05000900D11248A56994FB801A7010E94F58BD3
:10B06000C801B7010E944BC68B019C01862D60E18F
:10B0700070E044EC58E066CD8EE196E0BA010E94A3
:10B08000A3A67B018C01862D90E0019727EF31E08C
:10B09000FC01E29FC001E39F900DF29F900D1124EF
:10B0A0008A56994FB801A7010E94058CC801B701C3
:10B0B0000E944BC68B019C01862D61E170E045EB3F
:10B0C00058E040CDFA014081413081F490E0019791
:10B0D00027EF31E0AC01429FC001439F900D529F8A
:10B0E000900D11248A56994F61E011C0423091F4BD
:10B0F00090E0019727EF31E0FC01E29FC001E39F60
:10B10000900DF29F900D11248A56994F62E00E9493
:10B110000B8B15C0433081F490E0019727EF31E0AD
:10B12000AC01429FC001439F900D529F900D11248E
:10B130008A56994F63E0EBCF80E00E949E1C862DDB
:10B1400090E0019727EF31E0FC01E29FC001E39F0F
:10B15000900DF29F900D11248A56994F0E943F8BBB
:10B1600090E0A0E0B0E0BC01CD010E9449C68B0197
:10B170009C01862D62E170E04FE958E0E3CC90E05D
:10B18000019727EF31E0829F6001839FD00C929F4F
:10B19000D00C112426E936E0C20ED31E8EE196E0D3
:10B1A000BA010E9487A69B01AC01C601B9010E94A9
:10B1B000518CC6010E945C8C0E9449C68B019C0187
:10B1C000862D63E170E04DE858E00E94C522809131
:10B1D0009B04882359F5C60160E070E00E94648CEE
:10B1E00025C090E0019727EF31E0829F8001839F87
:10B1F000100D929F100D11240A56194F8EE196E002
:10B20000BA010E9487A6AB01BC01C8010E942D8C27
:10B21000C8010E94338C0E9449C68B019C01862D77
:10B2200064E170E045E758E00E94C5220E94381DA5
:10B230008BCC90E0019727EF31E0829F8001839FC4
:10B24000100D929F100D11240A56194F8EE196E0B1
:10B25000BA010E9487A6AB01BC01C8010E94398CCB
:10B26000C8010E943F8C0E9449C68B019C01862D1B
:10B2700065E170E04EE558E065CC90E0019727EF7E
:10B2800031E0829F8001839F100D929F100D112449
:10B290000A56194F8EE196E0BA010E9487A6AB01CB
:10B2A000BC01C8010E94458CC8010E944B8C0E94C1
:10B2B00049C68B019C01862D66E170E047E458E0A9
:10B2C00041CC67E170E046E358E00E947824862D87
:10B2D00081500E94002D38CC68E170E045E258E0D2
:10B2E0000E947824862D81500E94B92C2DCC90E0AC
:10B2F000019727EF31E0829F8001839F100D929F7D
:10B30000100D11240A56194F8EE196E0BA010E94E1
:10B3100087A69B01AC01C801B9010E94648C0E9400
:10B32000381DC8010E946F8C0E9449C68B019C0188
:10B33000862D69E170E042E158E004CC6BE170E0F9
:10B340004CEE57E00E947824062D10E0015010408A
:10B3500087EF91E0089F7001099FF00C189FF00C97
:10B36000112446E956E0E40EF51EC7010E949B8BAE
:10B37000C70140E050E060E070E00E94ED8B000FFC
:10B38000111F000F111F07551B4FF801108211826A
:10B3900012821382C70140E050E060E070E00E943A
:10B3A000F58BC70140E050E060E070E049C081509B
:10B3B0000E94A429F82E682F70E080E090E00E949F
:10B3C00049C68B019C01862D6CE170E043ED57E08E
:10B3D0005CC56DE170E040EC57E00E947824862D5A
:10B3E00090E0019727EF31E0829F8001839F100D4D
:10B3F000929F100D11240A56194FC8010E941D8CEE
:10B40000AB01BC01C8010E94F58B9ECB6EE170E0E0
:10B410004EEA57E00E947824862D90E0019727EFAE
:10B4200031E0829F8001839F100D929F100D1124A7
:10B430000A56194FC8010E941D8CAB01BC01C801FE
:10B440000E94058C81CB8EE196E0BA010E94A3A6F2
:10B450006B017C010E944BC68B019C01862D6FE124
:10B4600070E041EA57E00E94C522862D8150B70165
:10B47000A6010E94B52C68CB8EE196E0BA010E942D
:10B48000A3A66B017C010E944BC68B019C01862DFB
:10B4900060E270E043E857E00E94C522862D90E00C
:10B4A000019727EF31E0AC01429FC001439F900D0F
:10B4B000529F900D11248A56994FB701A6010E9400
:10B4C000158C42CB8EE196E0BA010E94A3A66B01D7
:10B4D0007C010E944BC68B019C01862D61E270E0CD
:10B4E00049E657E00E94C522E62DF0E0EE0FFF1F6F
:10B4F000EE0FFF1FEB55FB4FC082D182E282F38239
:10B5000023CB8EE196E0BA010E9477A67C01B701B9
:10B51000882777FD8095982F0E944BC68B019C0150
:10B52000862D68E270E049E557E00E94C522862D2D
:10B5300090E0019727EF31E0FC01E29FC001E39F1B
:10B54000900DF29F900D11248A56994FB7010E94D9
:10B550008C9631C48EE196E0BA010E94D3A66B01AD
:10B560007C01862D69E270E041E457E09701860195
:10B570000E94C522862D90E0019727EF31E0AC01B3
:10B58000429FC001439F900D529F900D11248A56F7
:10B59000994FB701A6010E94689645C48EE196E0D6
:10B5A000BA010E94D3A66B017C01862D6AE270E08D
:10B5B00048E257E0970186010E94C522862D90E05F
:10B5C000019727EF31E0FC01E29FC001E39F900D5E
:10B5D000F29F900D11248A56994FB701A6010E943F
:10B5E0007A9621C4FA01F0806F2D70E080E090E03F
:10B5F0000E9449C68B019C01862D62E370E04DE0FC
:10B6000057E00E94C522F092B006F092A708F0928F
:10B610009E0A6DC490E0019727EF31E0829F6001A0
:10B62000839FD00C929FD00C112426E936E0C20EE5
:10B63000D31EF601828D882309F487CA0E94F2B5D1
:10B640007B018C0181E896E00E94CFA4E61AF70AFC
:10B65000080B190BE0928D10F0928E1000938F1052
:10B660001093901081E0F60184830E94F4546CCA18
:10B6700090E0019727EF31E0829F6001839FD00C1B
:10B68000929FD00C112426E936E0C20ED31EF6019B
:10B69000828D882309F459CAC6010E945C8C611509
:10B6A00071058105910509F41AC4E090A304F09096
:10B6B000A40400E010E0C6010E945C8CE616F706C8
:10B6C0000807190708F00BC40AC001979093A40457
:10B6D0008093A304C6010E94EDA00E94BC2B81E8C8
:10B6E00096E00E94CFA43B014C0181E896E00E94C5
:10B6F000EBA45B016C0181E896E00E94E7A47C0169
:10B7000081E896E00E94E3A400E010E0A0E0B0E051
:10B71000E80EF91E0A1F1B1FEA0CFB1C0C1D1D1D49
:10B72000E614F7040805190538F481E896E00E944C
:10B73000CFA48B019C011BC081E896E00E94EBA482
:10B740006B017C0181E896E00E94E7A48C0181E80E
:10B7500096E00E94E3A420E030E0A0E0B0E0080F13
:10B76000191F2A1F3B1F0C0D1D1D2E1D3F1D8091F3
:10B77000B5049091B604A091B704B091B8048017B5
:10B780009107A207B30768F0801B910BA20BB30BC4
:10B790008093B5049093B604A093B704B093B80413
:10B7A000D3C91092B5041092B6041092B704109247
:10B7B000B804CAC990E0019727EF31E0829F700179
:10B7C000839FF00C929FF00C112426E936E0E20EE4
:10B7D000F31EC7010E94F18990E0A0E0B0E0BC0137
:10B7E000CD010E9449C68B019C01862D64E670E064
:10B7F00043E057E00E94C522C7010E94F1896CC254
:10B8000090E0019727EF31E0829F7001839FF00C59
:10B81000929FF00C112446E956E0E40EF51EC70194
:10B820000E94E089A0E0B0E0BC01CD010E9449C6C1
:10B830008B019C01862D65E670E048EF56E00E9482
:10B84000C522C7010E94E08970C090E0019727EFF0
:10B8500031E0829F7001839FF00C929FF00C1124C5
:10B8600086E996E0E80EF91EC7010E94C58990E0BE
:10B87000A0E0B0E0BC01CD010E9449C68B019C0153
:10B88000862D66E670E04BEE56E00E94C522C701A9
:10B890000E94C58921C290E0019727EF31E0829F85
:10B8A0007001839FF00C929FF00C1124E6E9F6E002
:10B8B000EE0EFF1EC7010E94D08990E0A0E0B0E02C
:10B8C000BC01CD010E9449C68B019C01862D67E613
:10B8D00070E04FED56E00E94C522C7010E94D0895A
:10B8E000FBC190E0019727EF31E0829F7001839FB9
:10B8F000F00C929FF00C112426E936E0E20EF31EC4
:10B90000C7010E94648AA0E0B0E0BC01CD010E94A2
:10B9100049C68B019C01862D68E670E043ED56E038
:10B920000E94C522C7010E94648ABC0181E00E9476
:10B930006A1CDDC2E82EFF24EE0CFF1CEE0CFF1C7F
:10B9400045EA54E0E40EF51EF701608171818281C1
:10B9500093810E944BC68B019C01862D69E670E0A5
:10B9600049EC56E00E94C522F70140815181628175
:10B97000738112C190E0019727EF31E0829F70013F
:10B98000839FF00C929FF00C112426E936E0E20E22
:10B99000F31EC7010E941D8C5B016C01C7010E9450
:10B9A0009D968823B9F0C7010E94CA898C01C701FE
:10B9B0000E94C589682FC80170E00E94FAC79B01E8
:10B9C000442737FD4095542FC601B5010E94C7C7D3
:10B9D0005B016C01C601B5010E944BC68B019C0145
:10B9E000862D6AE670E04BEB56E00E94C52281E0AE
:10B9F000B601A501D2C090E0019727EF31E0829F08
:10BA00007001839FF00C929FF00C112446E956E0E0
:10BA1000E40EF51EC7010E944F8A90E0A0E0B0E05E
:10BA2000BC01CD010E9449C68B019C01862D6BE6AD
:10BA300070E04FEA56E00E94C522C7010E944F8A7B
:10BA40004BC190E0019727EF31E0829F7001839F07
:10BA5000F00C929FF00C112486E996E0E80EF91E96
:10BA6000C7010E94058A8B019C01862D6CE670E05F
:10BA700047EA56E00E94C522C7010E94058A1EC0FF
:10BA800090E0019727EF31E0829F7001839FF00CD7
:10BA9000929FF00C1124E6E9F6E0EE0EFF1EC701BE
:10BAA0000E94418A8B019C01862D6DE670E04FE972
:10BAB00056E00E94C522C7010E94418A20E030E082
:10BAC00048EC52E4B6C190E0019727EF31E0829F45
:10BAD0007001839FF00C929FF00C112426E936E050
:10BAE000E20EF31EC7010E943F8B90E0A0E0B0E0A1
:10BAF000BC01CD010E9449C68B019C01862D6EE6DA
:10BB000070E046E956E00E94C522C7010E943F8BC3
:10BB1000E3C090E0019727EF31E0829F7001839F9F
:10BB2000F00C929FF00C112446E956E0E40EF51E4D
:10BB3000C7010E94FD8B0E944BC68B019C01862D84
:10BB40006FE670E04AE856E00E94C522C7010E94F5
:10BB5000FD8B20C090E0019727EF31E0829F7001BC
:10BB6000839FF00C929FF00C112486E996E0E80E7A
:10BB7000F91EC7010E940D8C0E944BC68B019C01CF
:10BB8000862D60E770E04FE756E00E94C522C701AE
:10BB90000E940D8CAB01BC0181E00E941A1CA7C160
:10BBA00090E0019727EF31E0829F7001839FF00CB6
:10BBB000929FF00C1124E6E9F6E0EE0EFF1EC7019D
:10BBC0000E94338C0E9449C68B019C01862D61E73F
:10BBD00070E04FE656E00E94C522C7010E94338CF8
:10BBE0002CC190E0019727EF31E0829F7001839F85
:10BBF000F00C929FF00C112426E936E0E20EF31EC1
:10BC0000C7010E945C8C0E9449C68B019C01862D55
:10BC100062E770E045E656E00E94C522C7010E9437
:10BC20005C8C0BC190E0019727EF31E0829F70019F
:10BC3000839FF00C929FF00C112446E956E0E40E2D
:10BC4000F51EC7010E943F8C0E9449C68B019C01D2
:10BC5000862D63E770E04EE456E00E94C522C701DE
:10BC60000E943F8CEAC090E0019727EF31E0829F6D
:10BC70007001839FF00C929FF00C112486E996E0EE
:10BC8000E80EF91EC7010E944B8C0E9449C68B0129
:10BC90009C01862D64E770E047E356E00E94C522D0
:10BCA000C7010E944B8CC9C0F82EFA948F2D0E94B8
:10BCB000CF2990E0A0E0B0E0BC01CD010E9449C6D0
:10BCC0008B019C01862D65E770E04FE256E00E94F3
:10BCD000C5228F2D0E94CF29682F81E0DAC08150C4
:10BCE00060E00E941128F82E882311F0FF24F394BD
:10BCF0006F2D70E080E090E00E9449C68B019C01AE
:10BD0000862D66E770E04AE156E0BFC090E00197FB
:10BD100027EF31E0829F7001839FF00C929FF00C1F
:10BD20001124E6E9F6E0EE0EFF1EC7010E946F8CBB
:10BD30000E9449C68B019C01862D67E770E04FE0A9
:10BD400056E00E94C522C7010E946F8C76C08150C8
:10BD500061E00E945429F82E682F70E080E090E0A6
:10BD60000E9449C68B019C01862D68E770E042EF76
:10BD700055E08BC090E0019727EF31E0AC01429F86
:10BD8000C001439F900D529F900D11248A56994FE8
:10BD90000E9492967C01B701882777FD8095982FA5
:10BDA0000E944BC68B019C01862D69E770E046EE30
:10BDB00055E00E94C52281E0B7010E94501C97C047
:10BDC00090E0019727EF31E0FC01E29FC001E39F83
:10BDD000900DF29F900D11248A56994F0E947096F3
:10BDE0006B017C01862D6AE770E046ED55E017C0D7
:10BDF00090E0019727EF31E0AC01429FC001439FE3
:10BE0000900D529F900D11248A56994F0E94829650
:10BE10006B017C01862D6BE770E045EC55E09701E6
:10BE200086010E94C522C701B60120E034E244E742
:10BE300059E40E94FFC60E941DC6AB01BC0181E00F
:10BE40000E94351C54C090E0019727EF31E0FC01BF
:10BE5000E29FC001E39F900DF29F900D11248A563E
:10BE6000994F0E949D96F82E882311F0FF24F39499
:10BE70006F2D70E080E090E00E9449C68B019C012C
:10BE8000862D6CE770E047EB55E00E94C52281E00B
:10BE90006F2D0E94841C2BC0862D90E0019727EF08
:10BEA00031E0829F8001839F100D929F100D11241D
:10BEB0000A56194FC8010E94648AA0E0B0E0BC0194
:10BEC000CD010E9449C69B01AC01C701B6010E9489
:10BED000FBC6181614F00C944E570C9443578091DF
:10BEE000A3049091A404009709F0EFCBF3CB0F903B
:10BEF000CF91DF911F910F91FF90EF90DF90CF9046
:10BF0000BF90AF909F908F907F906F9008953F92D9
:10BF10004F925F926F927F928F929F92AF92BF9259
:10BF2000CF92DF92EF92FF920F931F93DF93CF9305
:10BF3000CDB7DEB7CD54D0400FB6F894DEBF0FBEFC
:10BF4000CDBF3090D7041092D7048091C1048823CC
:10BF500009F0DBC0332009F0D8C00E94E51410922C
:10BF6000DA041092C4041092C5041092C604109210
:10BF7000C7040E94043100E010E027EFE22E21E028
:10BF8000F22E0E94FE10882319F4802F0E94A4290B
:10BF900084EA9CE067E47FE00E9449250E9DC00191
:10BFA0000F9D900D1E9D900D11248A56994F0E9451
:10BFB000C589682F84EA9CE00E94701F0F5F1F4FA5
:10BFC00003301105F1F60E942A8C882309F081C004
:10BFD00081E896E00E94CFA47B018C0181E896E085
:10BFE0000E94EBA43B014C0181E896E00E94E3A48F
:10BFF0005C0181E896E00E94E7A4E618F7080809CA
:10C000001909CC24DD24EA18FB080C091D09A0E05D
:10C01000B0E0E81AF90A0A0B1B0BC801B7010E942D
:10C0200049C620E030E04AE754E40E94B0C55B0115
:10C030006C0120E030E040E05FE30E94FBC6181690
:10C0400054F40F2EF0E0AF2EF0E0BF2EF0E0CF2E34
:10C05000FFE3DF2EF02D6624772497EF492E91E041
:10C06000592E649C4001659C900C749C900C11248A
:10C0700086E996E0880E991EC4010E9437950E94B9
:10C0800018C69B0191E0243F3907E4F4B9018827E1
:10C0900077FD8095982F0E944BC67B018C01C601CD
:10C0A000B50120E030E040E05FE30E94FFC69B0165
:10C0B000AC01C801B7010E94B0C5AB01BC01C4010D
:10C0C0000E94BF8A0894611C711C83E06816710489
:10C0D00041F60E942A8C8230C1F481E896E00E94E9
:10C0E000A8A50E94F2B57B018C010E94F2B56E19E1
:10C0F0007F09800B910B0E9449C620E030E84BEB92
:10C1000054E40E94ACC587FDF0CF8091C104882320
:10C1100009F074C18E010F5F1F4FC80164E871E020
:10C120000E9427BF88E0E82EF12CEC0EFD1EC7010F
:10C13000B8010E9420C0C7016DED71E00E94D4BE1D
:10C14000BC018E01015F1F4FC8010E9420C084EA1C
:10C150009CE0B8010E94F427C8010E9431C0C701C9
:10C160000E9431C0AA24BB2407EF802E01E0902E4C
:10C17000A89C6001A99CD00CB89CD00C112486E925
:10C1800096E0C80ED91EC6010E940D8C7B018C0161
:10C19000C6010E941D8CE61AF70A080B190B84EAE7
:10C1A0009CE0B801A7010E9415220894A11CB11CB3
:10C1B00093E0A916B104E1F616E1E12EF12CEC0EA4
:10C1C000FD1EC701BE016F5F7F4F0E9420C0C701E7
:10C1D00064EE71E00E94D4BEBC018E01035E1F4F6D
:10C1E000C8010E9420C084EA9CE0B8010E94F427A4
:10C1F000C8010E9431C0C7010E9431C000E010E0B8
:10C20000B7EFEB2EB1E0FB2E0E9DC0010F9D900D00
:10C210001E9D900D11248A56994F0E94FD8BAB01F3
:10C22000BC0184EA9CE00E9415220F5F1F4F03307F
:10C23000110551F7A4E2EA2EF12CEC0EFD1EC70108
:10C24000BE016F5F7F4F0E9420C0C7016BEE71E09F
:10C250000E94D4BEBC018E01055D1F4FC8010E9423
:10C2600020C084EA9CE0B8010E94F427C8010E9423
:10C2700031C0C7010E9431C000E010E0F7EFEF2E9F
:10C28000F1E0FF2E0E9DC0010F9D900D1E9D900DA3
:10C2900011248A56994F0E940D8CAB01BC0184EA8F
:10C2A0009CE00E9415220F5F1F4F0330110551F7CC
:10C2B000E2E3EE2EF12CEC0EFD1EC701BE016F5F16
:10C2C0007F4F0E9420C0C70161EF71E00E94D4BE81
:10C2D000BC018E01075C1F4FC8010E9420C084EA88
:10C2E0009CE0B8010E94F427C8010E9431C0C70138
:10C2F0000E9431C000E010E077EFE72E71E0F72EEA
:10C300000E9DC0010F9D900D1E9D900D11248A560B
:10C31000994F0E941D8CAB01BC0184EA9CE00E94F5
:10C3200015220F5F1F4F0330110551F760E4E62E11
:10C33000F12CEC0EFD1EC701BE016F5F7F4F0E9406
:10C3400020C0C7016AEF71E00E94D4BEBC018E011B
:10C35000095B1F4FC8010E9420C084EA9CE0B8011D
:10C360000E94F427C8010E9431C0C7010E9431C059
:10C3700000E010E057EFE52E51E0F52E0E9DC001D4
:10C380000F9D900D1E9D900D11248A56994F0E946D
:10C39000338CAB01BC0184EA9CE00E943C220F5F1D
:10C3A0001F4F0330110551F7332011F10E942A8CE1
:10C3B0008823F1F0EE24FF2447EFC42E41E0D42E71
:10C3C000EC9C8001ED9C100DFC9C100D11240A5674
:10C3D000194FC8010E94F189882319F0C8010E94F1
:10C3E000839F0894E11CF11C83E0E816F10441F7F7
:10C3F0000E94F454CE0101960E942BC0C35BDF4F14
:10C400000FB6F894DEBF0FBECDBFCF91DF911F9165
:10C410000F91FF90EF90DF90CF90BF90AF909F90E3
:10C420008F907F906F905F904F903F9008952F92E4
:10C430003F924F925F926F927F928F929F92AF92B4
:10C44000BF92CF92DF92EF92FF920F931F93DF93F1
:10C45000CF93CDB7DEB72A970FB6F894DEBF0FBEE5
:10C46000CDBF9A878987DC01DB963C90DB97DD9610
:10C470008C90DD97AF5BBF4F9C90A154B040DA9693
:10C48000AC90DA97DC96DC90DC97AE5BBF4F2C90DB
:10C4900012976C91A054B040BA87A98770E080E0F1
:10C4A00090E024E630E040E050E00E94C7C72B0156
:10C4B0003C01E985FA8561AD70E080E090E028EE0E
:10C4C00033E040E050E00E94C7C7460E571E681E8A
:10C4D000791EA985BA85D7968C91D797282F30E0F9
:10C4E000D8968C91F901E80FF11DE536F1056CF055
:10C4F00080E090E0A0E0B0E08D839E83AF83B887BA
:10C5000089839A83AB83BC8315C0B901882777FDE3
:10C510008095982F0E944BC620E030E048EC52E412
:10C520000E94B0C56D837E838F83988769837A83E9
:10C530008B839C83A985BA85D6966C9170E080E048
:10C5400090E020E13EE040E050E00E94C7C77B0160
:10C550008C01E985FA8565A970E080E090E02CE324
:10C5600030E040E050E00E94C7C7E60EF71E081F0B
:10C57000191FC801B70128EE33E040E050E00E94E7
:10C58000C7C7A985BA8552966D937D938D939C9369
:10C590005597DE966C9170E080E090E020E63AEEF0
:10C5A00040E050E00E94C7C7E985FA85668B778B2B
:10C5B000808F918F67AD70E080E090E00E94C7C7E8
:10C5C000A985BA855A966D937D938D939C935D97BB
:10C5D00080E00E94591581E896E0B301A2010E9413
:10C5E000C9A46A2D70E080E090E024E630E040E0ED
:10C5F00050E00E94C7C77B018C01692D70E080E08C
:10C6000090E028EE33E040E050E00E94C7C7E60E1D
:10C61000F71E081F191F81E896E0B7010E94D5A4F4
:10C62000682D70E080E090E024E630E040E050E0EB
:10C630000E94C7C77B018C01632D70E080E090E011
:10C6400028EE33E040E050E00E94C7C7E60EF71E38
:10C65000081F191F81E896E0B801A7010E94D9A41C
:10C66000622D70E080E090E024E630E040E050E0B1
:10C670000E94C7C77B018C016D2D70E080E090E0C7
:10C6800028EE33E040E050E00E94C7C7E60EF71EF8
:10C69000081F191F81E896E0B7010E94DFA4222439
:10C6A0003324E7EFF1E02E9E40012F9E900C3E9E3A
:10C6B000900C112446E956E0840E951EC4010E9498
:10C6C000448BC40162E00E940B8BA985BA85D49685
:10C6D0008C910E94278CE985FA8566897789808DFF
:10C6E000918DA30192010E940DC8C401B9010E945D
:10C6F000518CA985BA855A966D917D918D919C91A9
:10C700005D97A30192010E940DC8C401B9010E9466
:10C71000648CE985FA8584A9882361F56289738927
:10C7200084899589A30192010E940DC879018A012B
:10C73000C801B7010E9449C69B01AC016D817E8191
:10C740008F8198850E94FFC60E941DC65B016C0107
:10C75000C401B601A5010E94398CC401B601A5012E
:10C760000E94458CC401B801A7010E942D8C0E9433
:10C77000381D3BC0A985BA8552966D917D918D91EA
:10C780009C9155970E9449C69B01AC016D817E81A9
:10C790008F8198850E94FFC60E941DC6AB01BC0117
:10C7A000C4010E94398CE985FA856289738984897C
:10C7B00095890E9449C69B01AC0169817A818B8170
:10C7C0009C810E94FFC60E941DC6AB01BC01C40132
:10C7D0000E94458CA985BA8552964D915D916D91C7
:10C7E0007C915597C4010E942D8CC4010E945BA1CD
:10C7F0000894211C311CB3E02B16310409F051CFF1
:10C800000E94F2B5E985FA8566877787808B918BE0
:10C8100081E082830E94875F2A960FB6F894DEBF7C
:10C820000FBECDBFCF91DF911F910F91FF90EF9081
:10C83000DF90CF90BF90AF909F908F907F906F9040
:10C840005F904F903F902F9008954F925F926F921C
:10C850007F928F929F92AF92BF92CF92DF92EF9290
:10C86000FF920F931F93DF93CF93CDB7DEB7299736
:10C870000FB6F894DEBF0FBECDBF4C01DC01199698
:10C880008C91882329F40E945615813009F4CEC476
:10C890000E946415882309F0C9C493C481EC90E117
:10C8A0000E942A1690E0A0E0B0E0BC01CD010E94F9
:10C8B00049C6AB01BC01C4010E943E166E837F8352
:10C8C0008887998781EC90E10E942F1690E0A0E084
:10C8D000B0E0BC01CD010E9449C6AB01BC01C4015E
:10C8E0000E943E166A837B838C839D8381EC90E15A
:10C8F0000E94341690E0A0E0B0E0BC01CD010E949F
:10C9000049C6AB01BC01C4010E943E162B013C018B
:10C910006E817F818885998520E030E040E053E496
:10C920000E94FBC6181624F4F401838187FF11C00E
:10C930006E817F818885998520E030E040E053E476
:10C940000E94ACC5882344F4D40113968C9181389D
:10C9500018F083E0F4018683D40116968C91169723
:10C96000882359F0815016968C9380E090E0A0E0E7
:10C97000B3E48E839F83A887B9876A817B818C818A
:10C980009D8120E030E040E053E40E94FBC6181691
:10C990002CF4D40114968C9187FF10C06A817B819E
:10C9A0008C819D8120E030E040E053E40E94ACC5E2
:10C9B000882344F4F4018481813820F083E0D40199
:10C9C00017968C93F4018781882351F081508783D7
:10C9D00080E090E0A0E0B3E48A839B83AC83BD83D6
:10C9E000C301B20120E030E040E053E40E94FBC606
:10C9F00018162CF4D40115968C9187FF0EC0C30134
:10CA0000B20120E030E040E053E40E94ACC588234E
:10CA100044F4F4018581813820F083E0D401189634
:10CA20008C93F4018085882361F0815080870F2EDC
:10CA3000F0E04F2EF0E05F2EF0E06F2EF3E47F2E5B
:10CA4000F02D6E817F818885998520E030E040E07F
:10CA500053E40E94ACC58823B1F46A817B818C8148
:10CA60009D8120E030E040E053E40E94ACC5882383
:10CA700051F4C301B20120E030E040E053E40E94F1
:10CA8000ACC5882359F0D40119968C911997882345
:10CA900029F481E019968C930E947A27F40163812E
:10CAA00070E0882777FD8095982F0E944BC69B01E8
:10CAB000AC016E817F81888599850E94ACC58823F1
:10CAC00099F1D40192961C92929786E996E01B9672
:10CAD0006C910E94F99A86E996E00E94648A7C0132
:10CAE0006E817F818885998520E030E040E053E4C5
:10CAF0000E9447C520E030E040E05CE30E94FFC6B2
:10CB00005B016C0100E010E0C801B7010E9449C65A
:10CB10009B01AC01C601B5010E94FFC6AB01BC017F
:10CB200080E090E00E94902DF401648170E08827FD
:10CB300077FD8095982F0E944BC69B01AC016A81BE
:10CB40007B818C819D810E94ACC58823C1F1D40179
:10CB50001A968C911A97823090F592961C92929721
:10CB60008DE898E01C966C910E94F99A8DE898E007
:10CB70000E94648A7C016A817B818C819D8120E096
:10CB800030E040E053E40E9447C520E030E040E060
:10CB90005CEB0E94FFC65B016C0100E010E0C80185
:10CBA000B7010E9449C69B01AC01C601B5010E94B4
:10CBB000FFC6AB01BC0181E090E00E94902DF40122
:10CBC000658170E0882777FD8095982F0E944BC67D
:10CBD0009B01AC01C301B2010E94ACC58823A9F13D
:10CBE000D4011A968C91823011F0882371F5F401EA
:10CBF00012A284E89AE065850E94F99A84E89AE096
:10CC00000E94648A7C01C301B20120E030E040E070
:10CC100053E40E9447C520E030E040E05CEB0E9416
:10CC2000FFC65B016C0100E010E0C801B7010E9483
:10CC300049C69B01AC01C601B5010E94FFC6AB010C
:10CC4000BC0182E090E00E94902D6E817F818885FA
:10CC500099850E941DC6D40113966C936A817B81CD
:10CC60008C819D810E941DC6F4016483C301B201C1
:10CC70000E941DC6D40115966C9381EC90E161E091
:10CC80000E949E15A82E81EC90E161E00E94FC15A7
:10CC9000882309F49DC281EC90E168E00E94FC15B4
:10CCA000833009F095C282E0F40180830E94752DE3
:10CCB00081E0D40192968C93B9C28981882339F599
:10CCC000C40160E971E04AE050E021E00E948C1666
:10CCD000EE24FF2477EFC72E71E0D72EEC9C800165
:10CCE000ED9C100DFC9C100D11240A56194FC80123
:10CCF0000E941D8CAB01BC01C8010E94F58B0894F9
:10CD0000E11CF11CB3E0EB16F10441F703C08150C4
:10CD1000F40186AF81EC90E161E00E94FC1588236C
:10CD200009F46AC281EC90E166E00E94FC15833050
:10CD300009F062C282E0D4018C930E94E52C76C295
:10CD40008981882339F5C40160E971E04AE050E047
:10CD500021E00E948C16EE24FF2467EFC62E61E0CE
:10CD6000D62EEC9C8001ED9C100DFC9C100D112426
:10CD70000A56194FC8010E941D8CAB01BC01C801A5
:10CD80000E94058C0894E11CF11CB3E0EB16F10441
:10CD900041F703C08150F40187AFD4011A960C917A
:10CDA000C4016A2D43E09E012F5F3F4F10E054EF16
:10CDB000E52E51E0F52ECC24C3940E94F81688236A
:10CDC000B9F099819130A1F4F4018285813049F064
:10CDD000813018F0823061F408C0D4011A969C9317
:10CDE00007C082E0F401828703C0D4011A961C9226
:10CDF000F40105A9C4016A2D4CE09E012F5F3F4F4D
:10CE000010E0B4EFEB2EB1E0FB2ECC24CA940E94CC
:10CE1000F816882321F08981D401D5968C93F401EA
:10CE200006A9C4016A2D4AE09E012F5F3F4F10E022
:10CE3000A4EFEA2EA1E0FA2ECC24CA940E94F816A0
:10CE4000882321F08981D401D6968C93F40107A917
:10CE5000C4016A2D4BE09E012F5F3F4F10E0F4EFBD
:10CE6000EF2EF1E0FF2EE4E6CE2E0E94F816882386
:10CE700021F08981D401D7968C93F40100ADC401CF
:10CE80006A2D49E09E012F5F3F4F10E074EFE72EBF
:10CE900071E0F72E54E6C52E0E94F816882321F083
:10CEA0008981D401D8968C93F40101ADC4016A2D17
:10CEB0004FE09E012F5F3F4F10E0B4EFEB2EB1E04B
:10CEC000FB2ECC24CA940E94F816882321F0898175
:10CED000D401D9968C93F40102ADC4016A2D4EE0C1
:10CEE0009E012F5F3F4F10E0A4EFEA2EA1E0FA2E43
:10CEF000FAE0CF2E0E94F816882321F08981D40110
:10CF0000DA968C93F40103ADC4016A2D40E19E01D1
:10CF10002F5F3F4F10E0E4EFEE2EE1E0FE2ECC2439
:10CF2000CA940E94F816882321F08981D401DB96E7
:10CF30008C93F40105ADC4016A2D4DE09E012F5F75
:10CF40003F4F10E074EFE72E71E0F72E5AE0C52E48
:10CF50000E94F816882321F08981D401DD968C93F4
:10CF6000C4016A2D47E09E012F5F3F4F00E010E0B3
:10CF7000B8EEEB2EB3E0FB2EA3E0CA2E0E94F8160B
:10CF8000882339F069816150633018F4C4010E942C
:10CF9000F118C4016A2D45E09E012F5F3F4F00E06C
:10CFA00010E0F8EEEF2EF3E0FF2EE3E0CE2E0E942D
:10CFB000F816882339F069816150633018F4C40190
:10CFC0000E946F1A81EC90E161E10E949E1583300E
:10CFD00091F490E0F40184A9882309F491E0D4014C
:10CFE000D4969C9340E0992309F441E081EC90E1D0
:10CFF00062E00E944C1A81EC90E161E10E949E1572
:10D00000833091F490E0F40184A9882309F491E03D
:10D01000D401D4969C9340E0992309F441E081EC3B
:10D0200090E162E00E944C1A86E996E00E941D8C15
:10D030007B018C0186E996E00E94FD8BE616F706DF
:10D0400008071907F1F48DE898E00E941D8C7B0118
:10D050008C018DE898E00E94FD8BE616F706080724
:10D06000190779F484E89AE00E941D8C7B018C01F9
:10D0700084E89AE00E94FD8BE616F7060807190778
:10D0800011F0F40112A281EC90E164E00E949E157F
:10D090008330D9F581EC90E161E00E949E158330E8
:10D0A00041F081EC90E161E00E949E15813009F031
:10D0B000B7C0C4010E949C1AC40160E00E94F1182C
:10D0C000C4010E94A91621C0D40192961C920E940C
:10D0D000F2B5F401668F778F80A391A31083C4010A
:10D0E0000E941762A3C0112381F481E0D4019296BB
:10D0F0008C930E94F2B5F401668F778F80A391A381
:10D1000082E080830E94752D91C06E817F81888529
:10D11000998520E030E040E053E40E94ACC58823CC
:10D12000D9F46A817B818C819D8120E030E040E0F0
:10D1300053E40E94ACC5882379F4C301B20120E016
:10D1400030E040E053E40E94ACC5882329F4D401C8
:10D1500019968C91813039F081EC90E10E948E1506
:10D16000882309F063C0F401118627C0D401139607
:10D170008C911397803859F080E813968C9380E057
:10D1800090E040E050E060E070E00E94902DF401FB
:10D190008481803851F080E8848381E090E040E031
:10D1A00050E060E070E00E94902DD40119968C91BF
:10D1B00019978130D9F519961C9280E00E947A2740
:10D1C00035C081EC90E10E948E15813079F666CBF6
:10D1D000C4016A2D48E09E012F5F3F4F00E010E040
:10D1E00074EFE72E71E0F72ECC24CA940E94F81653
:10D1F000882309F062CD8ECDC4016A2D46E09E01E0
:10D200002F5F3F4F00E010E054EFE52E51E0F52E88
:10D21000CC24CA940E94F816882309F091CDBDCD84
:10D22000F40112A1113009F05ECF4ECF29960FB64E
:10D23000F894DEBF0FBECDBFCF91DF911F910F914C
:10D24000FF90EF90DF90CF90BF90AF909F908F9026
:10D250007F906F905F904F9008951F93182F0E94BA
:10D260009D311092B5041092B6041092B70410923A
:10D27000B8041092A4041092A30486E996E00E94D8
:10D280007D8C8DE898E00E947D8C84E89AE00E9475
:10D290007D8C1092C1041092D8040E949B320E948F
:10D2A000B0A50E940133112341F40E94F814882391
:10D2B00021F00E94F5140E9483251F9108950F9379
:10D2C0001F938C0181E00E942D69F80112821F9149
:10D2D0000F9108952F923F924F925F926F927F929B
:10D2E0008F929F92AF92BF92CF92DF92EF92FF9276
:10D2F0000F931F93CF93DF93EC0180915D118823EF
:10D30000A1F48DE591E10E94C3BA892B71F00E94CE
:10D31000F2B56093671170936811809369119093CF
:10D320006A118DE591E10E94CDBACE010E94B71835
:10D33000882309F480C08A81882329F08091C10460
:10D34000882309F078C0109266111092651181EC63
:10D3500090E164E040E00E944C1A81EC90E163E0CF
:10D36000409165110E944C1A18820BC10E94F2B5BF
:10D370006E8F7F8F88A399A367C0813009F064C046
:10D380000E94F2B52E8D3F8D48A159A1621B730BEF
:10D39000840B950B615D77408040904008F454C049
:10D3A000109266111092651181EC90E164E040E00A
:10D3B0000E944C1A81EC90E163E0409165110E945B
:10D3C0004C1A83E08883CE010E945F69DAC040E096
:10D3D00080916611882309F441E04093661181EC45
:10D3E00090E164E00E944C1A0E94F2B560936711CC
:10D3F000709368118093691190936A110E94C1A47F
:10D4000090916511882359F0992309F0BAC081E001
:10D410008093651181EC90E163E041E009C09923BC
:10D4200009F4AFC01092651181EC90E163E040E037
:10D430000E944C1AA6C081EC90E164E00E949E1507
:10D44000833009F09ACF92CF2A883B884C885D8838
:10D45000EE88FF88088D198DAA8CBB8CCC8CDD8C56
:10D460006E847F84888899880E94F2B5E20CF31C50
:10D47000041D151DEA0CFB1C0C1D1D1DE60CF71CE4
:10D48000081D191DE61AF70A080B190BC801B70188
:10D4900020E83EEE46E350E00E940DC8D22EC801BF
:10D4A000B70120E63AEE40E050E00E940DC88CE360
:10D4B000D89EC0011124281BCE016CE0422F50E001
:10D4C00024EF31E00E94B116CE016AE04D2D50E00C
:10D4D00024EF31E00E94B1164FA9CE016BE050E07D
:10D4E00024EF31E00E94B11648ADCE0169E050E072
:10D4F00024EF31E00E94B11649ADCE016FE050E05B
:10D5000024EF31E00E94B1164AADCE016EE050E04A
:10D5100024EF31E00E94B1164BADCE0160E150E046
:10D5200024EF31E00E94B1164DADCE016DE050E028
:10D5300024EF31E00E94B1164EADCE0168E050E01C
:10D5400024EF31E00E94B1164FADCE0166E050E00D
:10D5500024EF31E00E94B1160E94F2B520916711CC
:10D56000309168114091691150916A11621B730BDF
:10D57000840B950B645F71408040904008F43ECF6F
:10D5800026CFDF91CF911F910F91FF90EF90DF9009
:10D59000CF90BF90AF909F908F907F906F905F9053
:10D5A0004F903F902F900895CF93DF93EC010E940E
:10D5B000F2B520916B1130916C1140916D11509129
:10D5C0006E11621B730B840B950B6A30710581051C
:10D5D000910508F450C00E94F2B560936B117093EE
:10D5E0006C1180936D1190936E1181EC90E10E940B
:10D5F000471B0E941CB381EC90E10E948E15813084
:10D60000D1F489818823B9F481EC90E161E041E0B3
:10D610000E944C1A40E08CA9882309F441E081EC77
:10D6200090E162E00E944C1A1E821F82188680E8F8
:10D630008B838C838D8381EC90E10E948E1589838E
:10D640008881882321F4CE010E94256411C0813095
:10D6500021F4CE010E946A690BC0823021F4CE0110
:10D660000E94F63105C0833019F4CE010E943119B1
:10D67000CE010E94E219DF91CF9108951F93182FD8
:10D680000E94F2B520919D1030919E1040919F1004
:10D690005091A010621B730B840B950B6E5E724051
:10D6A0008040904008F490C00E94F2B560939D10B5
:10D6B00070939E1080939F109093A010E12FF0E044
:10D6C000E256FB4F80818130B1F0883041F4809187
:10D6D000C104813009F078C00E949D3175C082304C
:10D6E00031F0833059F48091C104882321F080E027
:10D6F0000E942D6969C00E94F45466C0843051F4C0
:10D7000084EA9CE062E072E00E94FE1A81E080936D
:10D71000A0045AC0853029F586E996E00E94D08998
:10D7200060E0882309F461E086E996E00E94DC96D7
:10D730008DE898E00E94D08960E0882309F461E0D8
:10D740008DE898E00E94DC9684E89AE00E94D089F7
:10D7500060E0882309F461E084E89AE00E94DC96A6
:10D7600033C0893079F40E949D3186E996E00E94A9
:10D770009B8B8DE898E00E949B8B84E89AE00E9446
:10D780009B8B22C08A3001F50E949D3186E996E08C
:10D790000E941D8CAB01BC0186E996E00E94548A70
:10D7A0008DE898E00E941D8CAB01BC018DE898E0EB
:10D7B0000E94548A84E89AE00E941D8CAB01BC014F
:10D7C00084E89AE00E94548A1F91089581E00E94A3
:10D7D0003E6B089580E00E943E6B0895EF92FF92A9
:10D7E0000F931F93CF93DF93982F8091A5048917F0
:10D7F00009F468C081E0809395069093A50499236D
:10D80000E1F10E942A8C80938C1080E00E94278C8A
:10D81000C0E0D0E0E7EFEE2EE1E0FE2ECE9D8001ED
:10D82000CF9D100DDE9D100D11240A56194FC80111
:10D830000E94F189FE01EC57FE4E8083C80160E032
:10D840000E94EC892196C330D10541F781E896E02A
:10D850000E94FEA4A0E0B0E080938011909381111B
:10D86000A0938211B093831181E896E060E177E2A2
:10D870000E94FAA40E94F45425C080E00E942D6901
:10D8800086E996E0609184110E94EC898DE898E029
:10D89000609185110E94EC8984E89AE0609186117C
:10D8A0000E94EC89609180117091811181E896E06D
:10D8B0000E94FAA41092A4041092A30480918C10E8
:10D8C0000E94278CDF91CF911F910F91FF90EF90D5
:10D8D00008959F92AF92BF92CF92DF92EF92FF9204
:10D8E0000F931F93982EFA01643609F46EC16536C2
:10D8F00070F5673009F4CEC0683098F4643009F4EC
:10D9000076C0653038F4623009F44FC0633009F0F6
:10D91000C3C25EC0653009F485C0663009F0BCC280
:10D920009DC06A3009F400C16B3038F4683009F4E6
:10D93000CDC0693009F0B0C2E4C06C3009F421C137
:10D940006C3008F40AC16D3009F0A6C22AC16B36EA
:10D9500009F4DDC16C3698F4673609F473C1683692
:10D9600038F4653609F445C1663609F095C256C1EA
:10D97000693609F497C16A3608F0B0C17BC16E36CA
:10D9800009F40DC26F3638F46C3609F4D7C16D3620
:10D9900009F082C2ECC1603709F42AC2603708F48A
:10D9A00013C2613709F078C23CC24081411141E0A5
:10D9B00040939506642F70E080E090E00E9449C695
:10D9C0008B019C01892D62E070E049EA55E027C097
:10D9D00081E896E00E94A8A5892D63E070E04BE9FC
:10D9E00055E00E94782481E00E949E1C55C28EE181
:10D9F00096E0BA010E9487A6AB01BC0181E896E0DF
:10DA00000E94D9A481E896E00E94EBA40E9449C636
:10DA10008B019C01892D64E070E044E855E00E9490
:10DA2000C522E1CF8EE196E0BA010E947FA6BC013B
:10DA300081E896E00E94D5A481E896E00E94E7A4E0
:10DA4000A0E0B0E0BC01CD010E9449C68B019C0161
:10DA5000892D65E070E04FE655E0E1CF8EE196E07C
:10DA6000BA010E947FA6BC0181E896E00E94FAA458
:10DA700081E896E00E94FEA4A0E0B0E0BC01CD01E8
:10DA80000E9449C68B019C01892D66E070E04BE540
:10DA900055E0C5CF8EE196E0BA010E947FA6BC0199
:10DAA00081E896E00E94DFA481E896E00E94E3A46A
:10DAB000A0E0B0E0BC01CD010E9449C68B019C01F1
:10DAC000892D67E070E046E455E0A9CF60E08081F1
:10DAD000811161E081E896E00E94F1A481E896E07E
:10DAE0000E94F4A490E0A0E0B0E0BC01CD010E944F
:10DAF00049C68B019C01892D68E070E04AE255E03F
:10DB00008ECF4081411141E040939406642F70E034
:10DB100080E090E00E9449C68B019C01892D69E05C
:10DB200070E042E155E07BCF8EE196E0BA010E94C1
:10DB300087A6AB01BC0181E896E00E94C9A481E8F8
:10DB400096E00E94CFA40E9449C68B019C01892DBA
:10DB50006AE070E04AEF54E062CF80810E94EE6B91
:10DB60000E94CB1490E0A0E0B0E0BC01CD010E9487
:10DB700049C68B019C01892D6BE070E046EE54E0B4
:10DB80004ECF60816093A60470E080E090E00E9438
:10DB900049C68B019C01892D6CE070E041ED54E099
:10DBA0003ECF80810E940A390E94EA1090E0A0E0F6
:10DBB000B0E0BC01CD010E9449C68B019C01892DBA
:10DBC0006DE070E043EB54E02ACF6091950670E081
:10DBD00080E090E00E9449C68B019C01892D64E69B
:10DBE00070E047EA54E00E94C52281E0609195060A
:10DBF00015C10E94C1A490E0A0E0B0E0BC01CD013D
:10DC00000E9449C68B019C01892D65E670E045E9BB
:10DC100054E00E94C5220E94C1A4FEC081E896E0A3
:10DC20000E94EBA40E9449C68B019C01892D66E6E7
:10DC300070E046E854E00E94C52281E896E00E9428
:10DC4000EBA48FC081E896E00E94E7A4A0E0B0E0DA
:10DC5000BC01CD010E9449C68B019C01892D67E65C
:10DC600070E049E754E00E94C52281E896E00E94F6
:10DC7000E7A42FC081E896E00E94FEA4A0E0B0E0F7
:10DC8000BC01CD010E9449C68B019C01892D68E62B
:10DC900070E04DE654E00E94C52281E896E00E94C3
:10DCA000FEA417C081E896E00E94E3A4A0E0B0E0E3
:10DCB000BC01CD010E9449C68B019C01892D69E6FA
:10DCC00070E040E654E00E94C52281E896E00E94A0
:10DCD000E3A4BC0181E00E946A1CDEC081E896E0FA
:10DCE0000E94F4A490E0A0E0B0E0BC01CD010E944D
:10DCF00049C68B019C01892D6AE670E04BE454E033
:10DD00000E94C52281E896E00E94F4A485C060913B
:10DD1000940670E080E090E00E9449C68B019C016F
:10DD2000892D6BE670E04DE354E00E94C5226091BE
:10DD3000940681E070E00E94501CAEC081E896E03D
:10DD40000E94CFA40E9449C68B019C01892D6CE6DC
:10DD500070E04DE254E00E94C52281E896E00E9406
:10DD6000CFA4AB01BC0181E00E94351C95C00E948C
:10DD7000CE14BC0181E00E946A1C0E94CE14A0E077
:10DD8000B0E0BC01CD010E9449C68B019C01892DE8
:10DD90006DE670E04FE154E00E94C5227DC00E9414
:10DDA000CB1490E0A0E0B0E0BC01CD010E9449C6D8
:10DDB0008B019C01892D6EE670E041E154E00E94E8
:10DDC000C5220E94CB1428C06091A60470E080E0B8
:10DDD00090E00E9449C68B019C01892D6FE670E09E
:10DDE00042E054E00E94C52281E06091A60416C082
:10DDF0000E94EA1090E0A0E0B0E0BC01CD010E94DA
:10DE000049C68B019C01892D60E770E04AEE53E022
:10DE10000E94C5220E94EA10682F81E00E94841CA3
:10DE20003BC080914C05882399F10E942A8C88235D
:10DE300079F581E896E00E94E7A46C0181E896E01C
:10DE40000E94EBA47B018C0181E896E00E94E3A490
:10DE50005601CC24DD24A0E0B0E0A80EB91ECA1EF5
:10DE6000DB1EAE0CBF1CC01ED11EC601B5010E9438
:10DE70004BC68B019C01892D61E770E04BED53E0AF
:10DE80000E94C52281E0B601A5010E941A1C04C0AF
:10DE9000AA24BB246501E9CF1F910F91FF90EF9059
:10DEA000DF90CF90BF90AF909F900895EF92FF9238
:10DEB0000F931F930E94F2B57B018C0180918A1110
:10DEC00090918B11A0918C11B0918D11A8019701A7
:10DED000281B390B4A0B5B0B2739310541055105CE
:10DEE00008F466C08091C104882339F08091A504AC
:10DEF000811180E00E942D695BC080914C058823D0
:10DF000019F00E94563361C086E996E00E944F8A5C
:10DF1000882309F05AC08DE898E00E944F8A882330
:10DF200009F053C084E89AE00E944F8A882309F0E0
:10DF30004CC080918A1190918B11A0918C11B0915D
:10DF40008D11A8019701281B390B4A0B5B0BDA01D5
:10DF5000C901885E9340A040B04020F480918911AF
:10DF60008F5F01C081E08093891184EA9CE06CE1BD
:10DF700072E00E94642084EA9CE0609189110E9412
:10DF8000701F80918911833098F08091A2048823BA
:10DF900011F481E001C080E00E940A3910928911D9
:10DFA00064E670E080E090E00E9426B60E94D754BC
:10DFB000E0928A11F0928B1100938C1110938D11C5
:10DFC0001F910F91FF90EF9008950E949D31F0CF27
:10DFD0000E94B0A50E949D311092C1040E9401339D
:10DFE0000895CF92DF92EF92FF920F931F93CF93FA
:10DFF000DF93EB01873609F43DC4883608F082C010
:10E00000843109F461C28531E8F58A3009F4AFC181
:10E010008B30E0F4853009F42AC1863050F4833027
:10E0200009F400C1843008F012C1823009F0BBC687
:10E03000EFC0873009F43AC1873008F42EC1883028
:10E0400009F453C1893009F0AEC682C18F3009F49A
:10E0500008C2803150F48D3009F4D4C18E3008F0FC
:10E06000E8C18C3009F09FC6B8C1813109F40DC2F6
:10E07000813108F4FFC1823109F410C2833109F003
:10E0800092C615C28D3109F401C38E31C8F48831AE
:10E0900009F464C2893138F4863109F438C2873111
:10E0A00008F049C21EC28A3109F46DC28A3108F4EF
:10E0B00060C28B3109F49DC28C3109F074C6D6C29E
:10E0C000823309F445C3833368F48F3109F400C304
:10E0D0008F3108F4E5C2803209F412C3813209F0AD
:10E0E00062C626C3843609F468C3853620F48333B8
:10E0F00009F059C645C3853609F465C3863609F06B
:10E1000052C686C38B3709F4B5C48C3708F040C0BB
:10E11000813709F422C48237E0F48C3609F4C3C392
:10E120008D3650F4893609F4ACC3893608F4A5C39A
:10E130008B3609F038C6ADC38E3609F4F5C38E367A
:10E1400008F4DEC38F3609F4F6C3803709F02BC616
:10E15000FFC3863709F433C4873768F4833709F47B
:10E1600006C4833708F4FEC3843709F408C485372E
:10E1700009F019C608C4883709F439C4883708F487
:10E1800033C4893709F447C48A3709F00CC658C428
:10E19000843809F460C58538C8F48F3709F4E2C4BF
:10E1A000803838F48D3709F4B3C48E3708F0C5C40D
:10E1B00095C4813809F411C5813808F4E7C4823860
:10E1C00009F420C5833809F0EEC531C5883C09F44F
:10E1D000A9C5893C68F4863809F465C5863808F411
:10E1E0004EC58C3809F474C5863909F0DCC585C57F
:10E1F0008D3F09F4B6C58E3F20F48C3F09F0D3C59E
:10E20000A7C58E3F09F4BBC58F3F09F0CCC5BFC57C
:10E2100080E062E070E040ED5DE00E9478240E94C2
:10E22000875F21C080E063E070E040EC5DE00E9429
:10E2300078248091C1048823B1F081E08093D704D1
:10E240000E942A8C882379F00E94E86F0CC080E03D
:10E2500064E070E04FEA5DE00E94782480E00E9474
:10E260002D691092D70481E00E949E1C9CC580E01D
:10E2700065E070E04CE95DE00E94782480916F11C8
:10E28000882331F40E94E83281E080936F11EBCF54
:10E290000E94EF3210926F11E6CF60E08881811109
:10E2A00061E080E896E00E94BA89DDCF8AE0E9EA81
:10E2B000F3E0DF011D928A95E9F780E090E0FE012E
:10E2C000E80FF91F2081222321F0FC01E755FC4FC4
:10E2D000208301968B30910591F782E090E069EA06
:10E2E00073E04AE00E94B9ABBECF6881623010F49F
:10E2F00080E018C06093B4031092B5038EE196E0FD
:10E3000070E00E945AA66091B4037091B5038AE54B
:10E3100095E00E945AA680E090E064EB73E00E94D2
:10E32000121981E00E949E1C6091B4037091B503A4
:10E33000882777FD8095982F0E944BC68B019C0102
:10E3400080E068E070E04AE85DE00E94C5222BC5ED
:10E350008881833020F080E00E949E1C84CF882337
:10E3600019F40E9456897FCF0E9482897CCF80E079
:10E370006AE070E042E75DE00E947824C0E0D0E00F
:10E3800087EFE82E81E0F82ECE9D8001CF9D100D05
:10E39000DE9D100D11240A56194FC8010E94648A8F
:10E3A000A0E0B0E0BC01CD010E9449C6AB01BC01B8
:10E3B000C8010E94BF8AC80164E00E94F99AC8019E
:10E3C0000E94759FC80161E00E9498962196C33013
:10E3D000D105D1F60E94BC2B46CFE8808E2D0E943D
:10E3E0003D150E94F238FF2400E010E0C801B7019B
:10E3F0000E9449C68B019C0180E06CE070E041E521
:10E400005DE0D8C11881098180E0612F0E94A138A8
:10E4100081E0602F0E94A1380E94F238143011F080
:10E42000043021F481E08093A2041DCF1092A20455
:10E430001ACF90E08881811191E0892F0E940B1101
:10E440000E94101190E0A0E0B0E0BC01CD010E945C
:10E4500049C68B019C0180E06EE070E049E35DE01D
:10E46000A9C18EE196E00E947FA69093B9038093A4
:10E47000B80308C08EE196E00E947FA69093BB038C
:10E480008093BA030E94F238EECE8EE196E00E94AD
:10E490007FA69093BD038093BC03F4CF8EE196E0FA
:10E4A0000E947FA69093BF038093BE03EBCF188199
:10E4B000113019F41093C103D6CE112319F4109220
:10E4C000C103D1CE80E0D0CE8EE196E00E9487A637
:10E4D0006093CE047093CF048093D0049093D104C2
:10E4E000C2CE8EE196E00E9487A66093D20470931C
:10E4F000D3048093D4049093D5040E9449C68B0121
:10E500009C0180E065E170E043E25DE053C18881F9
:10E510000E94278C0E942A8C90E0A0E0B0E0BC0111
:10E52000CD010E9449C68B019C0180E066E170E04C
:10E530004CE05DE03FC1E8808E2D0E947A27FF24E9
:10E5400000E010E0C801B7010E9449C68B019C01A0
:10E5500080E067E170E045EF5CE02CC188810E94BB
:10E56000591580E068E170E04DED5CE00E94782490
:10E570007ACE80E069E170E04CEB5CE00E947824A8
:10E580000E94752D70CEC0E0D0E007EFE02E01E0D4
:10E59000F02ECE9D8001CF9D100DDE9D100D11241B
:10E5A0000A56194FC8010E941D8CAB01BC01C8015D
:10E5B0000E94F58B84EA9CE064E372E00E940D20E7
:10E5C00084EA9CE06C2F0E948F1F84EA9CE06CE33D
:10E5D00072E00E940D20C8010E94FD8BAB01BC01BE
:10E5E00084EA9CE00E94EE212196C330D10589F691
:10E5F0003ACEC0E0D0E017EFE12E11E0F12ECE9D33
:10E600008001CF9D100DDE9D100D11240A56194F6B
:10E61000C8010E941D8CAB01BC01C8010E94058C81
:10E6200080E06BE170E044E95CE00E94782484EAD9
:10E630009CE065E472E00E940D2084EA9CE06C2F6F
:10E640000E948F1F84EA9CE06CE472E00E940D201F
:10E65000C8010E940D8CAB01BC0184EA9CE00E94C1
:10E66000EE212196C330D10551F6FDCD688160932E
:10E67000C20370E080E090E00E9449C68B019C01DB
:10E6800080E06CE170E041E85CE094C080E06DE126
:10E6900070E045E65CE00E9478240E948325E3CD8B
:10E6A0008881809398048AE590E068E974E00E948C
:10E6B0000E196091980470E080E090E00E9449C6D5
:10E6C0008B019C0180E06EE170E04BE45CE0BDC238
:10E6D000888180939A048BE590E06AE974E00E9457
:10E6E0000E1960919A0470E080E090E00E9449C6A3
:10E6F0008B019C0180E06FE170E04AE25CE0B9C20E
:10E700008881809399048CE590E069E974E00E9427
:10E710000E196091990470E080E090E00E9449C673
:10E720008B019C0180E060E270E040E15CE0B5C2FA
:10E7300068816093B70370E080E090E00E9449C672
:10E740008B019C0180E061E270E045EF5BE0BAC2C2
:10E7500090E08881811191E0892F0E94F7100E943A
:10E76000FE1090E0A0E0B0E0BC01CD010E9449C6DF
:10E770008B019C0180E062E370E04EED5BE01AC02B
:10E7800080E00E94F71090E08881811191E0892F4C
:10E790000E9401110E94081190E0A0E0B0E0BC01CD
:10E7A000CD010E9449C68B019C0180E063E370E0CB
:10E7B0004BEC5BE00E94C52256CD81E04DE450E079
:10E7C00060E070E0B7C18091D804882319F0B4E00C
:10E7D000FB2E10C08091D604882319F0A3E0FA2EF6
:10E7E00009C08091C104882319F0F2E0FF2E02C015
:10E7F000F090D7046F2D70E080E090E00E9449C651
:10E800008B019C0180E065E670E04EEB5BE070C23E
:10E810000E94FB140E9449C68B019C0180E066E6C1
:10E8200070E04BEA5BE00E94C5220E94FB147B0172
:10E830008C018091A40C83FF1AC08091A50C8823C1
:10E8400041F085E393E1B801A7012AE030E00E949E
:10E85000D7BB8091A60C882351F08091A70C909192
:10E86000A80CB801A7012AE030E00E94D7BB0E94A3
:10E87000FB145DC10E94C1A485C281E06091B60312
:10E8800083C281E069EA73E04AE050E00E94FD1B28
:10E890008AC20E94581F6B017C0180E06BE670E029
:10E8A0004AE95BE01EC089E20E94CFB6AA2797FD25
:10E8B000A095BA2FBC01CD010E944BC620E030ECE0
:10E8C0004FE754E40E94B0C520E030E040EA50E455
:10E8D0000E94FFC66B017C0180E06CE670E049E8B5
:10E8E0005BE0970186010E94C522C701B60120E0C6
:10E8F00030E048EC52E40E94FFC60E941DC617C1DA
:10E900006091C00370E080E090E00E9449C68B01F6
:10E910009C0180E06DE670E04EE65BE00E94C5225F
:10E9200081E06091C00330C270919E0460E08091EC
:10E930009F0490E009C088E10E94B4B7182F89E1D4
:10E940000E94B4B7712F60E0682B792B81E014C26C
:10E950006091B8037091B9030EC06091BA037091D1
:10E96000BB0309C06091BC037091BD0304C06091FA
:10E97000BE037091BF0381E00E946A1C14C281E053
:10E980006091C10301C26091D2047091D30480915F
:10E99000D4049091D5040E9449C68B019C0180E06B
:10E9A00065E770E040E65BE00E94C5224091D2043A
:10E9B0005091D3046091D4047091D504BAC00E94E0
:10E9C0002A8C90E0A0E0B0E0BC01CD010E9449C6D5
:10E9D0008B019C0180E066E770E044E55BE00E940B
:10E9E000C5220E942A8CCEC10E94F210CBC1609138
:10E9F000E10470E080E090E00E9449C68B019C0138
:10EA000080E068E770E044E45BE00E94C52281E0BA
:10EA10006091E104B9C10E945E1590E0A0E0B0E011
:10EA2000BC01CD010E9449C68B019C0180E069E7D1
:10EA300070E044E35BE00E94C5220E945E15A2C123
:10EA40000E94101190E0A0E0B0E0BC01CD010E9456
:10EA500049C68B019C0180E06AE770E042E25BE01E
:10EA60000E94C5228091E104882309F09CC10E9484
:10EA700010117FC10E94361E90E0A0E0B0E0BC0102
:10EA8000CD010E9449C68B019C0180E06BE770E0DC
:10EA900045E15BE00E94C5220E94361E182F80913E
:10EAA000A40C83FF18C08091A50C882339F085E35E
:10EAB00093E1612F4AE050E00E940EBC8091A60CC9
:10EAC000882349F08091A70C9091A80C612F4AE00F
:10EAD00050E00E940EBC0E94361E54C10E94D145D7
:10EAE000182F80E06CE770E040E05BE00E94782443
:10EAF00084EA9CE00E94A910882339F085E393E121
:10EB0000612F42E050E00E940EBC81E0612F3CC1C9
:10EB10000E948D1D0E9449C68B019C0180E06DE71B
:10EB200070E04BEE5AE00E94C5220E948D1DAB01A1
:10EB3000BC0181E00E94351C36C10E94ED10F82E08
:10EB4000882311F0FF24F3946F2D70E080E090E0B3
:10EB50000E9449C68B019C0180E06EE770E044EDA5
:10EB60005AE0C6C06091C20370E080E090E00E946D
:10EB700049C68B019C0180E06FE770E049EC5AE0E8
:10EB80000E94C52281E06091C203FEC086E996E042
:10EB90000E944F8A682F811161E0F62E8DE898E07F
:10EBA0000E944F8A882311F0FF24F39484E89AE0AE
:10EBB0000E944F8A882311F0FF24F3946091C203CE
:10EBC00070E080E090E00E9449C68B019C0180E0EB
:10EBD00060E870E043EB5AE08BC00E94AC29F82E4D
:10EBE000882311F0FF24F3946F2D70E080E090E013
:10EBF0000E9449C68B019C0180E061E870E042EA16
:10EC00005AE076C00E94DF2990E0A0E0B0E0BC01AD
:10EC1000CD010E9449C68B019C0180E062E870E052
:10EC200049E85AE00E94C5220E94DF29ABC06091EA
:10EC3000980470E080E090E00E9449C68B019C013E
:10EC400080E063E870E047E75AE00E94C52281E077
:10EC50006091980499C060919A0470E080E090E01F
:10EC60000E9449C68B019C0180E064E870E04EE59B
:10EC70005AE00E94C52281E060919A0485C06091AB
:10EC8000990470E080E090E00E9449C68B019C01ED
:10EC900080E065E870E04CE45AE00E94C52281E023
:10ECA0006091990471C068816093B70370E080E05F
:10ECB00090E00E9449C68B019C0180E066E870E00C
:10ECC00049E35AE00E94C52281E06091B7035CC02D
:10ECD0000E946415F82E682F70E080E090E00E949A
:10ECE00049C68B019C0180E06CE870E044E25AE088
:10ECF0000E94C52281E06F2D47C00E94FE1090E067
:10ED0000A0E0B0E0BC01CD010E9449C68B019C018E
:10ED100080E066E970E045E15AE00E94C5220E9469
:10ED2000FE1027C00E9444827C01B701882777FD2E
:10ED30008095982F0E944BC68B019C0180E068EC67
:10ED400070E047E05AE00E94C52281E0B70114C09C
:10ED500060E08881811161E084EA9CE00E94B0104B
:10ED600008C060E08881811161E084EA9CE00E9433
:10ED7000AC10682F81E070E00E94501C14C08881A4
:10ED80000E947448682F81E00E94841C0CC080E0BF
:10ED90006FEF70E040EF59E00E94782481E00E941C
:10EDA0009E1C0E94C746DF91CF911F910F91FF904B
:10EDB000EF90DF90CF9008950F931F93CF93DF9341
:10EDC000082F162FEA010E94F2B56093DD047093BC
:10EDD000DE048093DF049093E004043018F40130E3
:10EDE000E8F405C0043091F10530D9F535C00E9432
:10EDF000FE10882371F48091E104813051F41436BF
:10EE000040F41E3031F0173121F0123311F013337A
:10EE100041F5812FBE010E94F16F26C00E94FE10B5
:10EE2000882371F48091E104813051F4143640F468
:10EE3000812F8350823020F0163011F01D3089F47C
:10EE4000802F612FAE010E9440550EC084E0612FDB
:10EE5000AE010E94696C08C0812FBE010E94B840BB
:10EE600003C080E00E949E1CDF91CF911F910F9103
:10EE7000089593E09093A8030E94DC760895EF92A2
:10EE8000FF920F931F93F82EE62E8A0182E0809363
:10EE9000A8030E94F2B56093DD047093DE048093B2
:10EEA000DF049093E00484EA9CE061E07EE00E944D
:10EEB0002A208F2D6E2DA8010E9483248F2D6E2D68
:10EEC000A8010E94DC761F910F91FF90EF900895AA
:10EED000EF92FF920F931F93F82EE62E8A0181E0A6
:10EEE0008093A8030E94F2B56093DD047093DE0462
:10EEF0008093DF049093E00484EA9CE06CE07EE081
:10EF00000E942A208F2D6E2DA8010E9483248F2D10
:10EF10006E2DA8010E94DC761F910F91FF90EF905B
:10EF20000895CF93DF93EA01653009F45BC0663042
:10EF300070F46230F9F0633020F4613009F072C08F
:10EF400016C06330D9F0643009F06CC01AC0683064
:10EF500009F45AC0693020F4673009F063C051C029
:10EF6000693009F454C06A3009F05CC053C00E9493
:10EF7000F45458C080E00E942D6954C00E94E86F8C
:10EF800051C084EA9CE06CEE7DE00E94FE1A48814C
:10EF9000423008F447C04093B4031092B50380E0B8
:10EFA00090E064EB73E00E9412196091B4037091D9
:10EFB000B5038EE196E00E945AA66091B403709169
:10EFC000B5038AE595E00E945AA60E94FE108823A8
:10EFD00019F081E00E949E1C8CE065E070E00E94C8
:10EFE0004C4820C083E08093A80384EA9CE064E559
:10EFF00072E00E940D2081E00E94F71081E00E94E3
:10F000009E1C0E948B3F0EC00E9456330BC00E9474
:10F010005A3308C08EE196E00E9454A6BC0181E0FC
:10F020000E946A1CDF91CF9108950E942A8C882348
:10F0300091F486E996E00E944F8A813089F18DE84B
:10F0400098E00E944F8A813059F184E89AE00E944A
:10F050004F8A813029F180E896E00E940C8988234C
:10F06000D1F08BE79CE061E00E9487A480919A0632
:10F07000813041F080919108813021F08091880A9F
:10F08000813071F484EA9CE066E472E10E94EA2631
:10F090000E94E86F08958BE79CE060E00E9487A4DF
:10F0A0000895EF92FF920F931F93CF93DF9384EA1B
:10F0B0009CE06CEA74E10E94EA268091D7048823E0
:10F0C00041F084EA9CE064E974E10E94EA260E942F
:10F0D000E86F0E942A8C882399F481E896E00E94C8
:10F0E000FEA4892B41F10091A3041091A40481E8AE
:10F0F00096E00E94FEA480179107E8F491E01CC0FE
:10F100000E942A8C8823B9F086E996E00E947A8CC6
:10F11000811181E0082F8DE898E00E947A8C882385
:10F1200009F400E084E89AE00E947A8C882309F4CC
:10F1300000E090E002C090E000E08091A604882307
:10F1400009F0B7C0992319F4002309F4B9C00E944B
:10F150002A8C882309F4C1C10E948D1D2091B90415
:10F160003091BA044091BB045091BC04621B730BF4
:10F17000840B950B16161706180619060CF0ADC170
:10F1800084EA9CE060E774E10E94EA260E948D1DFB
:10F190002091B9043091BA044091BB045091BC0451
:10F1A000621773078407950709F47EC00E948D1DBE
:10F1B000AB01BC0184EA9CE00E941A494091B90469
:10F1C0005091BA046091BB047091BC0484EA9CE045
:10F1D0000E941A4984EA9CE065E574E10E94492591
:10F1E0000E948D1DAB01BC018091B9049091BA04BD
:10F1F000A091BB04B091BC04481B590B6A0B7B0B5C
:10F2000084EA9CE00E942E3984EA9CE06CE374E17D
:10F210000E94EA2649C00E942A8C823021F481E8AB
:10F2200096E00E94A8A50E945E158823B9F18091FE
:10F23000CC049091CD042091A3043091A404820FBA
:10F24000931F9093CD048093CC048091C40490913B
:10F25000C504A091C604B091C7042091B5043091B3
:10F26000B6044091B7045091B804820F931FA41FB5
:10F27000B51F8093C4049093C504A093C604B093B3
:10F28000C70481E00E942D690E94EE140E9483252C
:10F2900081E08093D9040E94F45406C080E00E946B
:10F2A0002D6981E08093DA0484EA9CE067E074E1F0
:10F2B000C8C0992311F4002319F081E08093D80489
:10F2C0008091A104882349F08091A004882329F427
:10F2D00084EA9CE06BEC73E1B4C080919E048630BC
:10F2E00029F080919F04863009F0FDC081E00E94E2
:10F2F0000727882309F4F7C086E0809391100E94C5
:10F30000073884EA9CE066E973E19BC00E94F2B58D
:10F310007B018C0180918D1090918E10A0918F10A7
:10F32000B0919010E81AF90A0A0B1B0B81E896E0DD
:10F330000E94CFA4E616F7060807190748F4809143
:10F340009506882329F08091A204882309F4D3C06C
:10F3500084EA9CE06EE773E10E94EA26C091A30470
:10F36000D091A4048091A40C84FF18C08091A50CB6
:10F37000882339F085E393E1BE014AE050E00E9422
:10F38000EBBB8091A60C882349F08091A70C90914B
:10F39000A80CBE014AE050E00E94EBBB84EA9CE06E
:10F3A0006FE971E00E946420C0E0D0E007EF11E057
:10F3B00084EA9CE067E773E10E94492584EA9CE0C7
:10F3C0006C2F0E94EE1F84EA9CE069E672E00E94C6
:10F3D0006420C09FC001C19F900DD09F900D11244B
:10F3E0008A56994F0E941D8CAB01BC0184EA9CE0B7
:10F3F0000E942E3984EA9CE06FE971E00E9464204B
:10F400002196C330D105A1F684EA9CE06DE571E058
:10F410000E94E11A809195068823B1F48BE79CE065
:10F4200062E00E9487A40E94F2B560938D107093F1
:10F430008E1080938F109093901084EA9CE062E489
:10F4400073E10E94EA2657C084EA9CE064E273E11B
:10F450000E94EA260E94C1A4082F8091A40C84FF78
:10F460001AC08091A50C882341F085E393E1602FB9
:10F4700070E04AE050E00E9485BC8091A60C882391
:10F4800051F08091A70C9091A80C602F70E04AE099
:10F4900050E00E9485BC0E94C1A4882361F584EAE3
:10F4A0009CE06CEF72E10E94EA268BE79CE060E052
:10F4B0000E9487A4109291101092A0040E94F2B5AD
:10F4C00060938D1070938E1080938F109093901096
:10F4D00081E896E00E945DA50EC00E945E1588231B
:10F4E00009F0A1CE98CE80E896E00E940C8988238E
:10F4F00009F42ECF0BCFDF91CF911F910F91FF9089
:10F50000EF900895AF92BF92CF92DF92EF92FF9269
:10F510000F931F930E94F2B57B018C012091B504DB
:10F520003091B6044091B7045091B80421153105CB
:10F530004105510541F460938E1170938F118093B2
:10F540009011909391118091BD049091BE04A0916F
:10F55000BF04B091C00459016A01A81AB90ACA0AC5
:10F56000DB0AD601C5018E0D9F1DA01FB11F809320
:10F57000B5049093B604A093B704B093B804E09296
:10F58000BD04F092BE040093BF041093C004009722
:10F59000A105B10541F08093B9049093BA04A093FA
:10F5A000BB04B093BC048091C204813019F480E0A4
:10F5B0000E942D6980E896E00E940C898823E9F07A
:10F5C0002091CE043091CF044091D0045091D104C9
:10F5D000211531054105510581F08091B5049091C7
:10F5E000B604A091B704B091B804281739074A07A8
:10F5F0005B0718F480E00E942D6980E896E00E9485
:10F600000C89882349F40E940F89882329F08BE70D
:10F610009CE061E00E9487A42091B5043091B6047B
:10F620004091B7045091B8048091D2049091D304D2
:10F63000A091D404B091D504281739074A075B0775
:10F6400020F48091D904882339F08BE79CE00E9454
:10F650008AA41092D60422C081E08093D6048091BF
:10F660008E1190918F11A0919011B0919111A801DC
:10F670009701281B390B4A0B5B0BDA01C901855F27
:10F680009140A040B04050F00E94F732E0928E11BD
:10F69000F0928F1100939011109391111F910F917F
:10F6A000FF90EF90DF90CF90BF90AF900895EF92D2
:10F6B000FF920F931F93CF93DF938EE196E00E940A
:10F6C000BEAA8AE595E00E94BEAA8CEB95E00E9456
:10F6D000BEAA0E94F2B520919A1130919B114091DF
:10F6E0009C1150919D11621B730B840B950B653619
:10F6F00071058105910508F456C088E20E94B4B7EF
:10F70000019759F40E94F2B560939E1170939F1176
:10F710008093A0119093A11133C080919D04882300
:10F7200079F50E94F2B520919E1130919F11409180
:10F73000A0115091A111621B730B840B950B695B97
:10F740007B4080409040E0F082E00E94AF4784EA36
:10F750009CE06CE672E00E94642086E996E068E036
:10F760000E94F99A8DE898E068E00E94F99A84E88E
:10F770009AE068E00E94F99A81E080939D04B2C00B
:10F7800080919D04882329F00E9482500E946F542A
:10F79000A9C00E94F2B560939A1170939B11809357
:10F7A0009C1190939D110E94F2B520919611309179
:10F7B00097114091981150919911621B730B840B12
:10F7C000950B655F71408040904050F00E94F2B50B
:10F7D000609396117093971180939811909399115B
:10F7E0008091DC04882339F10E94F2B52091DD0478
:10F7F0003091DE044091DF045091E004621B730BF2
:10F80000840B950B695E734080409040A0F086E9C0
:10F8100096E00E944F8A882361F48DE898E00E9468
:10F820004F8A882331F484E89AE00E944F8A882323
:10F8300011F00E949D3100E010E027EFE22E21E060
:10F84000F22E0E9DE0010F9DD00D1E9DD00D1124B6
:10F85000CA56D94FCE010E944F8A882319F0CE0193
:10F860000E94CF980F5F1F4F0330110551F7809111
:10F87000C104882359F00E9494330E94827A00E0E8
:10F8800010E097EFE92E91E0F92E09C080914C0528
:10F890008823A9F30E9494330E94FC3DF0CF0E9D73
:10F8A000E0010F9DD00D1E9DD00D1124CA56D94FD9
:10F8B000CE010E949D96882361F0CE010E944F8A5E
:10F8C000882339F4CE0160E00E949896CE010E9410
:10F8D000659C0F5F1F4F0330110509F781E191E12E
:10F8E0000E94D46ADF91CF911F910F91FF90EF900A
:10F8F0000895EF92FF920F931F93CF93DF9385E3C9
:10F9000093E140E05BE460E070E00E9447BE64E6A3
:10F9100070E080E090E00E9426B663E876E080E048
:10F9200090E00E94EA8184EA9CE06DE772E00E9428
:10F93000E11A8CE061E00E94FEB680E061E00E9486
:10F94000FEB680E061E00E9481B78AE260E00E943A
:10F95000FEB689E260E00E94FEB60E9441498BE754
:10F960009CE060E00E9487A460E070E08AE795E494
:10F970000E94108760E070E48CE996E40E94198789
:10F9800080E896E061E00E94BA8989EF9CE10E94DC
:10F99000078981E896E048E750E060E070E00E9467
:10F9A000D9A481E896E060E070E00E94DFA481E8DD
:10F9B00096E060E070E00E94D5A481E896E06AE8F5
:10F9C0007BE20E94C4A483E193E140E051EE60E059
:10F9D00070E00E945AB86091B4037091B5038EE153
:10F9E00096E00E945AA68EE196E068E677E70E94CC
:10F9F00065A98EE196E06FE872E20E9471A98EE13E
:10FA000096E061E977E70E946BA98EE196E060E0FD
:10FA10000E944FA66091B4037091B5038AE595E00A
:10FA20000E945AA68AE595E06FE377E70E9465A9F0
:10FA30008AE595E069E772E20E9471A98AE595E09E
:10FA400061E977E70E946BA98AE595E061E00E9491
:10FA50004FA66091B4037091B5038CEB95E00E94C2
:10FA60005AA68CEB95E069E377E70E9465A98CEBD9
:10FA700095E063E672E20E9471A98CEB95E061E982
:10FA800077E70E946BA98CEB95E061E00E944FA69E
:10FA90008EE196E066E179E10E9469A68AE595E04B
:10FAA00066E179E10E9469A68CEB95E066E179E177
:10FAB0000E9469A600E010E037EFE32E31E0F32E5C
:10FAC0000E9DE0010F9DD00D1E9DD00D1124CA5634
:10FAD000D94FCE0161E00E94EC89CE0168E873E164
:10FAE0000E946A8A0115110559F4CE0168E873E194
:10FAF0000E94A88ACE0140E050E46CE975E40AC097
:10FB0000CE0168EB7BE00E94A88ACE0140E050E87D
:10FB10006BE375E40E94BF8ACE0140E050E66AE6DE
:10FB200076E40E94198ACE0160E00E94CE96CE0152
:10FB300060E070E00E94E689CE0165E00E940B8BD8
:10FB4000CE0140E050E060E070E00E94F58BCE0115
:10FB500040E050E060E070E00E94058CCE0160E083
:10FB600070E00E948C96CE0140E050E060E87FE3B8
:10FB70000E946896CE0140E050E060E87FE30E947A
:10FB80007A960115110519F4CE0164E002C0CE0188
:10FB900060E10E94F99ACE0160E00E9458960F5FE2
:10FBA0001F4F0330110509F08BCF81E191E10E94D5
:10FBB000BE1A0E94C3458CE065E070E00E944C488C
:10FBC00081E066E57FE642E050E00E947AB382EE93
:10FBD00094E063E070E00E944186DF91CF911F9135
:10FBE0000F91FF90EF900895FC011382128282E53D
:10FBF00094E091838083758364830895FC018481FC
:10FC000095810E9416A708956115710581059105DA
:10FC100069F481E090E0A0E0B0E08093A2119093BD
:10FC2000A311A093A411B093A51108C06093A211D1
:10FC30007093A3118093A4119093A5115093A711D1
:10FC40004093A611809170008E7F80937000809108
:10FC5000B0008C7F8093B0008091B100877F80934B
:10FC6000B1008091B6008F7D8093B60080917000C6
:10FC70008D7F809370008091B10084608093B1008B
:10FC80008091B1008C7F8093B10086E090E09093EA
:10FC9000AE118093AD1108951092A8111092A91180
:10FCA0001092AA111092AB111092AC118091AD116B
:10FCB0009091AE118093B200E0E7F0E08081816026
:10FCC00080830895E0E7F0E080818E7F808308954F
:10FCD0008091A8119091A911A091AA11B091AB1196
:10FCE0000196A11DB11D8093A8119093A911A09315
:10FCF000AA11B093AB118091A8119091A911A09174
:10FD0000AA11B091AB112091A2113091A311409191
:10FD1000A4115091A51182179307A407B50710F1FC
:10FD20008091AC118823F1F481E08093AC11809133
:10FD3000A8119091A911A091AA11B091AB11821BA9
:10FD4000930BA40BB50B8093A8119093A911A093CA
:10FD5000AA11B093AB11E091A611F091A7110995EA
:10FD60001092AC1108951F920F920FB60F920BB61E
:10FD70000F9211242F933F934F935F936F937F9331
:10FD80008F939F93AF93BF93EF93FF938091AD11A8
:10FD90009091AE118093B2000E94687EFF91EF9126
:10FDA000BF91AF919F918F917F916F915F914F9193
:10FDB0003F912F910F900BBE0F900FBE0F901F9091
:10FDC00018951F920F920FB60F920BB60F92112437
:10FDD0002F933F934F935F936F937F938F939F9353
:10FDE000AF93BF93EF93FF93E091B311F091B411F0
:10FDF0000995FF91EF91BF91AF919F918F917F9165
:10FE00006F915F914F913F912F910F900BBE0F908B
:10FE10000FBE0F901F901895FC01A3E0440F551FD3
:10FE2000661F771FAA95D1F7403080E0580781E020
:10FE3000680780E0780714F481E010C033E075951E
:10FE40006795579547953A95D1F7403080E0580728
:10FE500081E0680780E078071CF482E0828339C083
:10FE600023E075956795579547952A95D1F74030CA
:10FE700080E0580781E0680780E0780714F483E0A9
:10FE8000EDCF92E075956795579547959A95D1F77F
:10FE9000403080E0580781E0680780E0780714F47C
:10FEA00084E0DCCF82E075956795579547958A95F4
:10FEB000D1F7403080E0580781E0680780E078079C
:10FEC00014F485E0CBCF85E082834FEF5FEF60E0F5
:10FED00070E08FB78383F8945183408350938700F9
:10FEE0004093860083818FBF80918100887F8093BB
:10FEF0008100809181009281892B809381000895F7
:10FF00001092800020E1209381000E940C7F0895D0
:10FF1000EFE6F0E080818E7F80830895E1E8F0E0F5
:10FF20002081DC0112968C91282B208308950F9359
:10FF30001F93CF93DF93EC018B0112161306140667
:10FF4000150624F4BA01A9010E940C7F1D830C83BD
:10FF500081E080936F00CE010E948E7FDF91CF9170
:10FF60001F910F910895F999FECF72BD61BDF89A66
:10FF700080B50895F999FECF1FBA72BD61BD40BD2D
:10FF80000FB6F894FA9AF99A0FBE0895282F909117
:10FF900014129F5F943408F090E080911512891735
:10FFA000E1F33FB7F89480911112882341F0E92FD3
:10FFB000F0E0EA5EFD4E2083909314121DC081E0B4
:10FFC00080931112209312121092131282E088BBB8
:10FFD00080917100826080937100809190008F7396
:10FFE0008068809390008091940090919500409655
:10FFF00090939900809398003FBF0895862F0E94A8
:020000021000EC
:10000000C67F81E090E008951F920F920FB60F9285
:100010000BB60F9211242F933F934F935F936F93DF
:100020007F938F939F93EF93FF9340911112509181
:100030001212209198003091990060910D127091E8
:100040000E12809113121FC0260F371F952F91702B
:1000500056954F5F9817B9F0992321F08091900041
:10006000806C04C0809190008F73806880939000B2
:10007000309399002093980090931312509312128A
:10008000409311123BC04930F8F2493039F48AE00C
:100090008093111280919000806C28C0809114127E
:1000A000E09115128E1769F4109211128091900050
:1000B0008F7380939000809171008D7F8093710089
:1000C0001DC081E080931112EF5FE43408F0E0E09E
:1000D000E0931512F0E0EA5EFD4E808180931212EB
:1000E00010921312809190008F738068809390001B
:1000F000260F371F3093990020939800FF91EF91BE
:100100009F918F917F916F915F914F913F912F912F
:100110000F900BBE0F900FBE0F901F9018958091FF
:1001200011128823E1F708950E948F8008951F928D
:100130000F920FB60F920BB60F9211241F932F93AD
:100140003F934F935F936F937F938F939F93AF935F
:10015000BF93EF93FF932091960030919700909179
:100160000912992341F0809191008F7B8093910037
:100170001092091208C080919100806480939100D0
:1001800080E88093091270910812772331F5992342
:1001900009F06CC080910B1290910C12820F931F8A
:1001A00090939B0080939A0084E088BB80917100BB
:1001B00084608093710080910D1290910E12280F2F
:1001C000391F96958795280F391F30931012209369
:1001D0000F1281E08093081249C040910F12509194
:1001E000101210910912E0910D12F0910E1260910F
:1001F0000A12AA27BB27AE1BBF0BC901841B950B94
:1002000097FD2CC06695612B7F5F8A0F9B1F79300D
:1002100018F44E0F5F1FF4CF60930A1280917100A3
:100220008B7F809371009091B7119F5F903508F09C
:1002300090E08091B611981739F0E92FF0E0E8547A
:10024000FE4E60839093B711809191008F7B8093D5
:100250009100109209121092081208C060930A12BD
:100260005093101240930F1270930812FF91EF9168
:10027000BF91AF919F918F917F916F915F914F91BE
:100280003F912F911F910F900BBE0F900FBE0F90BB
:100290001F9018951F920F920FB60F920BB60F92E8
:1002A00011242F938F939F93EF93FF93809171006D
:1002B0008B7F80937100809191008F7B8093910060
:1002C0009091081280910912805820910A1203C05F
:1002D0002695282B9F5F9930D8F320930A1290918E
:1002E000B7119F5F903508F090E08091B611981794
:1002F00039F0E92FF0E0E854FE4E20839093B711D7
:1003000010920812809191008F7B8093910010923F
:100310000912FF91EF919F918F912F910F900BBE3A
:100320000F900FBE0F901F9018958091B711E0911C
:10033000B6118E1719F42FEF3FEF0EC02E2F2F5F3F
:10034000203508F020E0E22FF0E0E854FE4E8081F6
:100350002093B611282F30E0C90108958091B7117C
:10036000E091B6118E1719F4EFEFFFEF06C0F0E041
:10037000E854FE4E8081E82FF0E0CF01089590917F
:10038000B7118091B611292F30E0482F50E098170F
:1003900010F4205B3F4F241B350BC9010895809159
:1003A000B6118093B71108950F931F9301E710E0E2
:1003B000F80180818B7F808380818F7D80830E9484
:1003C000CF810E948F80F80180818D7F80831F9173
:1003D0000F9108959B01AC012D3A8BE1380780E025
:1003E000480780E0580730F4109271001092900096
:1003F00081E814C063E056954795379527956A952F
:10040000D1F72D3A8BE1380780E0480780E05807A4
:10041000D0F5109271001092900082E880939100C4
:1004200030930E1220930D12CA01B90125E230E07B
:1004300040E050E00E94C7C752E0969587957795B7
:1004400067955A95D1F770930C1260930B1287E160
:1004500062E00E94FEB686E161E00E9481B786E11B
:1004600061E00E94FEB6109208121092B71110922D
:10047000B61110921112109214121092151280E2FD
:1004800088BB809371000895DF93CF9300D0CDB7E0
:10049000DEB72091581330915913CE0101962115E2
:1004A000310519F48256934102C0821B930B9A8343
:1004B000898389819A810F900F90CF91DF91089560
:1004C0002F923F924F925F926F927F928F929F9264
:1004D000AF92BF92CF92DF92EF92FF920F931F9352
:1004E000DF93CF93CDB7DEB766970FB6F894DEBF34
:1004F0000FBECDBF69877A878B879C872D873E8704
:100500004F87588BE98AFA8A0B8B1C8BC601B50181
:100510002FA438A849A85AA82DA92D8B3EA93E8BF7
:1005200029853A854B855C850E9447C55B016C0136
:100530006BA57CA58DA59EA52D853E854F855889EB
:100540000E9447C5A60195010E94B0C53B014C0120
:10055000C801B701A80197010E9448C57B018C0121
:10056000C401B30120E030E040E450EC0E94FFC63B
:100570009B01AC01C801B7010E9448C5A2019101CD
:100580000E9448C59058A60195010E94B0C56D8390
:100590007E838F839887C401B30120E030E040E080
:1005A00050EC0E94FFC69B01AC0169897A898B8956
:1005B0009C890E9448C5A20191010E9448C5A601DC
:1005C00095010E94B0C5A60195010E94B0C52B01FE
:1005D0003C012D893E89C9019A8389831C821B8233
:1005E00022243324AFC0E981FA8160817181828144
:1005F000938129853A854B855C850E9447C57B019F
:100600008C01CFA8D8ACC20CD31CA30192010E94CC
:10061000FFC69B01AC016D817E818F8198850E9410
:1006200048C59B01AC01C801B7010E94FFC69B01F0
:10063000AC0169897A898B899C890E9448C59B0194
:10064000AC01C801B7010E94FFC69B01AC016D85DA
:100650007E858F8598890E9448C5F60160837183E5
:10066000828393836D817E818F8198859B01AC010C
:100670000E9448C55B016C01E981FA81608171814A
:100680008281938129853A854B855C850E9447C587
:100690007B018C0189AC9AAC820C931C20E030E089
:1006A00040E450E40E94FFC6A30192010E94FFC6ED
:1006B0009B01AC01C601B5010E9448C59B01AC017C
:1006C000C801B7010E94FFC69B01AC0169897A8904
:1006D0008B899C890E9448C5F40160837183828361
:1006E00093830BAD1CAD020D131DE981FA8161915D
:1006F000719181919191FA83E98329853A854B859E
:100700005C850E9447C520E030E040EC50E40E9448
:10071000FFC6A30192010E94FFC69B01AC01C60166
:10072000B5010E9448C5F801608371838283938379
:100730002B813C812F5F3F4F3C832B8384E090E0F3
:10074000280E391EEB81FC812BA93CA9E217F30787
:100750000CF449CF66960FB6F894DEBF0FBECDBF3E
:10076000CF91DF911F910F91FF90EF90DF90CF908D
:10077000BF90AF909F908F907F906F905F904F90C1
:100780003F902F9008954F925F926F927F928F9239
:100790009F92AF92BF92CF92DF92EF92FF920F9310
:1007A0001F93CF93DF935C012B0169017A0138011C
:1007B00082E0A816B104A4F500D000D080916013A7
:1007C00090916113EDB7FEB7928381838FE992E038
:1007D000948383830E94FC0D809160139091611338
:1007E000EDB7FEB79283818381EA92E0948383839D
:1007F0000E94FC0D8091601390916113EDB7FEB7DC
:10080000928381838FEB92E0948383830E94FC0D1B
:100810000F900F900F900F9081E090E00E9487C89A
:10082000F8012081318137FD05C0C50101972817E6
:1008300039073CF0C501019795958795F3019183A0
:100840008083F30100811181F801EE0FFF1FEE0F8D
:10085000FF1FE40DF51DC701B601208131814281E2
:1008600053810E94ACC588230CF063C001151105AB
:1008700009F4D8C00130110519F1F8013197EE0FD4
:10088000FF1FEE0FFF1FE40DF51D60817181828156
:100890009381A70196010E94ACC5181634F001504F
:1008A0001040F30111830083BDC0C701B601F201FE
:1008B00024813581468157810E94ACC5181624F0E9
:1008C000F30111821082AEC05EEFA52E5FEFB52E50
:1008D000A00EB11EC1E0D0E0CA15DB0521F4F30182
:1008E000C083D1839FC0C50101968C0F9D1F62E01C
:1008F00070E00E94FAC7972E062F172FF801EE0F0F
:10090000FF1FEE0FFF1FE40DF51D608171818281D5
:100910009381A70196010E94ACC518162CF0802F78
:10092000992D9C01E901D8CF58010894A108B1087C
:10093000D3CF48010894811C911CF401EE0FFF1FD6
:10094000EE0FFF1FE40DF51D60817181828193819F
:10095000A70196010E94ACC588230CF063C0E50195
:1009600022970C171D0709F45DC08DEF9FEFA80EAD
:10097000B91E0A151B0599F00E5F1F4FF801EE0F07
:10098000FF1FEE0FFF1FE40DF51DC701B60120810B
:100990003181428153810E94ACC5181624F0F301C5
:1009A000918280823FC0FE01EE0FFF1FEE0FFF1FFE
:1009B000E40DF51D6081718182819381A70196010B
:1009C0000E94ACC5181624F4E801CA15DB0521F411
:1009D000F301D183C08326C0C50101968C0F9D1FF2
:1009E00062E070E00E94FAC7972E062F172FF801D9
:1009F000EE0FFF1FEE0FFF1FE40DF51D60817181EB
:100A000082819381A70196010E94ACC518162CF033
:100A1000802F992D9C01E901D8CF58010894A10895
:100A2000B108D3CFDF91CF911F910F91FF90EF903D
:100A3000DF90CF90BF90AF909F908F907F906F90FE
:100A40005F904F9008952F923F924F925F926F92D6
:100A50007F928F929F92AF92BF92CF92DF92EF924E
:100A6000FF920F931F93DF93CF93CDB7DEB76697B7
:100A70000FB6F894DEBF0FBECDBF98878F837A87FD
:100A800069875C874B873E872D87188B0F87DA8AAB
:100A9000C98ABC8AAB8A9E8A8D8AC80162E070E0EE
:100AA0000E94FAC77A836983FC82EB821E821D82D0
:100AB00022243324A3C0AB81BC812D913D914D9163
:100AC0005C918F81988569857A858E010F5F1F4FB4
:100AD0000E94C383A981BA818D01000F111F000FED
:100AE000111F1196AA0FBB1FAA0FBB1FEDB7FEB7B0
:100AF00072970FB6F894FEBF0FBEEDBF4DB65EB64F
:100B00000894411C511CE985FA85E00FF11F6081B2
:100B1000718182819381EB85FC85E00FF11F20813B
:100B2000318142815381ED85FE850E0F1F1FF80133
:100B3000E080F18002811381E985FA85EA0FFB1FCD
:100B4000A080B180C280D380EB85FC85EA0FFB1FBB
:100B50006080718082809380EDB7FEB7618272827F
:100B600083829482ED85FE85AE0FBF1F6D907D90D0
:100B70008D909C90D20114966D927D928D929C9254
:100B80001797E1E0F0E01996FC93EE931897EB814C
:100B9000FC811B96FC93EE931A97E989FA89E20D82
:100BA000F31D1D96FC93EE931C97EB89FC89E20DD7
:100BB000F31D1F96FC93EE931E97ED89FE89E20DBF
:100BC000F31D5196FC93EE9350970E9460822D8105
:100BD0003E812F5F3F4F3E832D838B819C81049606
:100BE0009C838B83A4E0B0E02A0E3B1EEDB7FEB7DA
:100BF00072960FB6F894FEBF0FBEEDBF2D813E81F9
:100C00008F859889281739070CF455CF66960FB64B
:100C1000F894DEBF0FBECDBFCF91DF911F910F9132
:100C2000FF90EF90DF90CF90BF90AF909F908F900C
:100C30007F906F905F904F903F902F900895FC01B0
:100C400011861086138612861586148611821082EC
:100C5000138212821582148217821682089560937D
:100C60001104709312048093130490931404089554
:100C700060911104709112048091130490911404F6
:100C8000089590935E1280935D127093601260934A
:100C90005F12089590935B1280935A120895809189
:100CA0005A1290915B12089580915F129091601298
:100CB0000895909308048093070408958091070491
:100CC000909108040895FC01868197810895DC01C4
:100CD0008D919C911197880F991F880F991F1896D5
:100CE000ED91FC911997E80FF91F408351836283BE
:100CF00073838D919C91119701968D939C93089588
:100D0000FC01808191810895FC0111821082089577
:100D1000660F771F660F771FDC011896ED91FC9127
:100D20001997E60FF71F2081318142815381B90164
:100D3000CA010895DC0180915C128823D9F01296D3
:100D40008D919C911397880F991F880F991F1A9660
:100D5000ED91FC911B97E80FF91F4083518362834B
:100D6000738312968D919C911397019613969C9381
:100D70008E9312970895FC01828193810895FC015E
:100D8000138212820895660F771F660F771FDC01AA
:100D90001A96ED91FC911B97E60FF71F2081318188
:100DA00042815381B901CA010895DC0180915C122E
:100DB0008823D9F014968D919C911597880F991FCF
:100DC000880F991F1C96ED91FC911D97E80FF91F54
:100DD000408351836283738314968D919C91159700
:100DE000019615969C938E9314970895FC01848127
:100DF00095810895FC01158214820895660F771F6E
:100E0000660F771FDC011C96ED91FC911D97E60F94
:100E1000F71F2081318142815381B901CA010895B0
:100E200060930D0470930E0480930F04909310044C
:100E300008956093090470930A0480930B049093BF
:100E40000C0408956F927F928F929F92AF92BF92FF
:100E5000CF92DF92EF92FF920F931F93DF93CF9386
:100E600000D000D0CDB7DEB76C014A015B01FC01B8
:100E700060847184F301E080F18002811381CB01F1
:100E8000BA01A80197010E94ACC58823BCF0F60105
:100E9000808191810197880F991F880F991F680E93
:100EA000791EF301E080F18002811381C501B40154
:100EB000A80197010E94FBC618162CF4E982FA8259
:100EC0000B831C8304C089829A82AB82BC82F601A8
:100ED000608571854285538524853585A2E1AA2EDA
:100EE000B12CAC0CBD1CD60156968681978101E0D1
:100EF00010E07E010894E11CF11CEEE0F0E0CE0E63
:100F0000DF1E4D010E9423850F900F900F900F90D0
:100F1000CF91DF911F910F91FF90EF90DF90CF90D5
:100F2000BF90AF909F908F907F906F9008958F9219
:100F30009F92AF92BF92CF92DF92EF92FF920F9368
:100F40001F93CF93DF936C01DC0116968D919C91DA
:100F500017970197880F991F880F991F1896ED9181
:100F6000FC911997E80FF91F60817181828193814B
:100F700020E030E04AE754E40E94B0C520E030E0D1
:100F800040E85FE30E9447C54B015C01C0E0D0E050
:100F9000BE01882777FD8095982F0E944BC6A5013A
:100FA00094010E94FFC6AB01BC01C6010E942287CA
:100FB000F601E688F788008D118DC801B70120E0A1
:100FC00030E040E050E00E94FBC6181624F017FB0A
:100FD000109517F91095C801B701209109043091B7
:100FE0000A0440910B0450910C040E94FBC6181691
:100FF00014F480E006C02196F3E0C83EDF0741F616
:1010000081E0DF91CF911F910F91FF90EF90DF90E2
:10101000CF90BF90AF909F908F9008958F929F92A6
:10102000AF92BF92CF92DF92EF92FF920F931F93F6
:10103000CF93DF936C01DC0116968D919C911797ED
:101040000197880F991F880F991F1896ED91FC91B1
:101050001997E80FF91F608171818281938120E0E7
:1010600030E04AE754E40E94B0C520E030E040E8B8
:101070005FE30E9447C54B015C01C0E0D0E0BE01C8
:10108000882777FD8095982F0E944BC6A501940173
:101090000E94FFC6AB01BC01C6010E942287F60177
:1010A000E288F38804891589C801B70120E030E09F
:1010B00040E050E00E94FBC6181624F017FB109584
:1010C00017F91095C801B70120910D0430910E0455
:1010D00040910F04509110040E94FBC6181614F49E
:1010E00080E006C02196F3E0C83EDF0741F681E0CC
:1010F000DF91CF911F910F91FF90EF90DF90CF90F4
:10110000BF90AF909F908F9008950F931F938C0185
:101110000E942287F80126893789408D518DB901B7
:10112000CA011F910F9108950F931F938C010E9484
:101130002287F8012289338944895589B901CA0176
:101140001F910F9108950F931F938C010E94228786
:10115000F8012685378540895189B901CA011F9157
:101160000F910895CF93DF93EC0180915C12882357
:1011700071F0888599850E945C0C8A859B850E9408
:101180005C0C8C859D850E945C0C10925C12DF913A
:10119000CF9108950E94B2880895CF93DF93EC0118
:1011A00077FD2EC07F836E83623071054CF10E9403
:1011B000B2888E819F81880F991F880F991F0E9486
:1011C000B20B888799878E819F81880F991F880F1E
:1011D000991F0E94B20B8A879B878E819F81880FFF
:1011E000991F880F991F0E94B20B8C879D871982C7
:1011F00018821B821A821D821C8281E080935C12FD
:10120000DF91CF91089581E08093611208959093CA
:101210006312809362120895FC0180810895809189
:10122000611210926112811181E00895809164121F
:10123000882319F080B1847002C08CB1807188233A
:1012400059F40E9400B66093651270936612809301
:1012500067129093681208950E9400B6209165125B
:10126000309166124091671250916812E0916212BB
:10127000F0916312309731F0621B730B840B950B66
:10128000CB0109950895FC018081882371F086E2E5
:1012900060E00E9481B765E070E080E090E00E942D
:1012A00026B686E261E00E9481B7089580916412BB
:1012B0000E94F6B3089580E00E94F6B386E261E0F2
:1012C0000E94FEB686E261E00E9481B70895FC01AB
:1012D000108282E060E00E94FEB684E260E00E943C
:1012E000FEB686E260E00E94FEB682E061E00E9407
:1012F00081B784E261E00E9481B786E261E00E94EA
:1013000081B708950F931F93082F01500230F8F40E
:10131000809164120E94F6B310926412002319F0B7
:1013200081E080936412002311F014E201C012E006
:10133000812F60E00E94FEB6812F61E00E9481B79C
:10134000802F66E179E841E050E00E947AB31F9176
:101350000F91089586E260E00E94FEB686E261E0A9
:101360000E9481B780E063E079E842E050E00E94AB
:101370007AB30895FC016083662319F00E945B89AB
:1013800008950E94AA8908950895FC01EE5EFE4F1B
:1013900080810895FC01EC50FE4F80819181089579
:1013A000FC01EF55FF4F80810895FC01EC5DFE4F7D
:1013B0000190F081E02D309711F0862F0995089566
:1013C000FC01ED5EFE4F808191810895FC01ED5E90
:1013D000FE4F718360830895FC01E356FF4F6083E5
:1013E0000895FC01E356FF4F80810895FC01E25609
:1013F000FF4F80810895FC01EE50FF4F2081318125
:1014000042815381B901CA010895FC01E251FF4FA5
:101410002081318142815381B901CA010895FC01C3
:10142000EC55FF4F60830895FC01EC55FF4F808120
:101430000895EF92FF920F931F93CF93DF93EC01E8
:101440007A018B01CB01BA0120E030E040E050E0AE
:101450000E94ACC5181674F4CA50DF4FC801B7011A
:1014600020E030E048E452E40E94B0C5688379830C
:101470008A839B83DF91CF911F910F91FF90EF9013
:101480000895FC01EA50FF4F608171818281938150
:1014900020E030E048E452E40E94FFC60895FC01D9
:1014A000E156FF4F80810895FC01EF53FF4F4083C9
:1014B0005183628373830895FC01EF53FF4F608172
:1014C0007181828193810895FC01E656FF4F8081EE
:1014D0009181089587E26031780781F083E168386F
:1014E000780761F08FE0603A780741F087E0603D6F
:1014F000780721F083E0683E7807B1F49B0140E073
:1015000050E060E472E48FE090E00E940DC83093F8
:1015100016042093150480E29EE4B9010E94E6C7F8
:1015200070931804609317040895809115049091A6
:1015300016040895209115043091160440E050E0FF
:1015400060E472E48FE090E00E942FC8C901089522
:101550000F931F93CF93DF93EC018B010E949A8A24
:101560008017910738F00115110521F0C656DF4F9D
:1015700019830883DF91CF911F910F910895AF9246
:10158000BF92CF92DF92EF92FF920F931F93CF9370
:10159000DF93EC017A018B01CB01BA0120E030E04E
:1015A00040E050E00E94FBC618161CF45701680189
:1015B00006C057016801D7FAD094D7F8D094CE016D
:1015C0000E949A8AA0E0B0E0BC01CD010E9449C609
:1015D0009B01AC01C601B5010E94FBC6181634F090
:1015E000CE50DF4FE882F9820A831B83DF91CF91CF
:1015F0001F910F91FF90EF90DF90CF90BF90AF9031
:101600000895FC01E354FF4F2081318142815381D1
:10161000B901CA0108951F93CF93DF93EC01162FF0
:101620000E944F8A882339F5113049F4CA5DDE4F94
:1016300080EE9EE899838883C652D14019C012304B
:1016400049F4CA5DDE4F82E89EE88993999389EF59
:101650009FE80AC0133079F4CA5DDE4F82E89EE845
:101660008993999383EC90E999838883C852D140F8
:10167000CB5EDE4F1883DF91CF911F910895FC015F
:10168000EB5EFE4F80810895FC01E354FF4F108212
:101690001182128213827C9610821182128213822E
:1016A0003C9680E090E0A0E0B0E080839183A2834C
:1016B000B383389711921192119211921082118274
:1016C000128213820895CF93DF93EC01FC01E3545F
:1016D000FF4F2081318142815381CB01AA2797FDA1
:1016E000A095BA2F820F931FA41FB51F80839183EB
:1016F000A283B383CF55DF4F8881C15AD04088235E
:1017000019F4709561957F4FFE01E650FF4F2081DF
:10171000318142815381CB01AA2797FDA095BA2F31
:10172000820F931FA41FB51F80839183A283B3836D
:10173000DF91CF910895CF93DF93EC01FC01E2504C
:10174000FF4F2081318142815381211531054105AF
:10175000510581F0C650DF4F88819981AA81BB81F4
:10176000CA5FD040281B390B4A0B5B0B20833183A7
:1017700042835383BE0166507F4FFB01208131813C
:1017800042815381FE01EE5FFE4F80819181A281F3
:10179000B381821B930BA40BB50B80839183A2832F
:1017A000B383FB012081318142815381FE01EA5FD5
:1017B000FE4F80819181A281B381821B930BA40B88
:1017C000B50B80839183A283B383FB0110821182C6
:1017D00012821382DF91CF910895FC01E250FF4FF6
:1017E00040835183628373830895FC01EE5FFE4F53
:1017F00040835183628373830895FC01EE5FFE4F43
:1018000060817181828193810895FC01EA5FFE4FBE
:1018100040835183628373830895FC01EA5FFE4F26
:1018200060817181828193810895FC01E650FF4FB0
:1018300040835183628373830895FC01E650FF4F18
:101840002081318142815381B901CA010895809379
:101850006A12089580916A120895FC01468757879D
:10186000608B718B0895FC016685778580899189ED
:101870000895FC01428B538B648B758B0895FC019A
:1018800062897389848995890895FC01468B578BF9
:10189000608F718F0895FC0166897789808D918DA5
:1018A0000895FC01E65FFE4F9B0140E050E020837D
:1018B0003183428353830895FC01E65FFE4F6081CC
:1018C0007181828193810895FC01E25FFE4F9B014B
:1018D00040E050E020833183428353830895FC012C
:1018E000E25FFE4F60817181828193810895FC01E6
:1018F00061A70895FC0181A50895FC01EB55FF4FF8
:1019000010820895CF92DF92EF92FF920F931F9370
:10191000CF93DF93EB016A01E880F9800A811B8194
:10192000C801B7012DEB37E346E855E30E94ACC58B
:1019300018169CF08DEB97E3A6E8B5E388839983AE
:10194000AA83BB830F2EF0E0EF2EF4E2FF2EF4E724
:101950000F2FF9E41F2FF02D0EC060911704709126
:10196000180480E090E00E9449C6A80197010E94F7
:10197000B0C57B018C01C801B7010E941DC6F601EC
:10198000EB53FF4F608371838283938361157105ED
:101990008105910541F481E090E0A0E0B0E0808312
:1019A0009183A283B38385EC90E0C80ED91EF60123
:1019B00061917191819191916F010E9449C69B0142
:1019C000AC01C801B7010E9447C520E030E04AE7FA
:1019D00054E40E94FFC60E941DC6F6017183608315
:1019E000685E734010F011821082DF91CF911F91D9
:1019F0000F91FF90EF90DF90CF9008952F923F923C
:101A00004F925F926F927F928F929F92AF92BF920E
:101A1000CF92DF92EF92FF920F931F93DF93CF93BA
:101A200000D00F92CDB7DEB7FC012B015B834A8358
:101A30001901E080F18002811381DA016D907D90BF
:101A40008D909C90C801B701A40193010E94ACC580
:101A5000181684F4EA81FB816088718882889388F3
:101A6000C801B701A40193010E94ACC518160CF07F
:101A700007C11CC1AA81BB819096AD90BD90CD904D
:101A8000DC909397F20160817181828193810E9441
:101A90001DC66A157B058C059D0540F4C801B7017C
:101AA000A40193010E94ACC5882351F4C601B5017D
:101AB0000E9449C6D2016D937D938D939C93139799
:101AC00019822FC0C801B701A40193010E94ACC5BF
:101AD000882311F0B1E024C0C601B5010E9449C6B7
:101AE000F2016083718382839383F1E0F98319C0EB
:101AF000C801B70120E030E040E85FE30E94ACC5D8
:101B0000882319F082E089830CC0C601B5010E94C8
:101B100049C6D2016D937D938D939C931397B2E048
:101B2000B983F20160817181828193810E941DC617
:101B300029EDC22ED12CC20CD31CD6016D937D93FE
:101B40008D939C93139785EEA82EB12CA20CB31CF9
:101B5000F501E080F180028113816D917D918D917D
:101B60009C910E9449C69B01AC01D2016D917D916F
:101B70008D919C910E9447C59B01AC01C801B701A2
:101B80000E9448C5F50160837183828393836081DD
:101B900071818281938120E030E040E85FE30E9420
:101BA000FBC68823E4F0D5016D917D918D919C91C8
:101BB00020E030E040E85FE30E9447C5F501608324
:101BC000718382839383F60180819181A281B381A5
:101BD0000196A11DB11D80839183A283B383F981F6
:101BE000F130F1F0F13020F0F23009F075C030C082
:101BF00089ED90E0280E391ED1012D913D914D9136
:101C00005C91EA81FB8180A191A1A2A1B3A1821B79
